:100000000C94A9150C94D4150C94D4150C94D415F7
:100010000C94D4150C94D4150C94D4150C94D415BC
:100020000C94D4150C94D4150C94D4150C94D415AC
:100030000C94D4150C94AD7A0C94D4150C94D4155E
:100040000C94D4150C94C6860C9410D00C94D41532
:100050000C94832E0C94D4150C94D4150C94D415B4
:100060000C94D4150C94D4150C943FC80C94D4154E
:100070000C94D4150C94D4150C94D4150C94D4155C
:100080000C94D4150C94D4150C94D415084AD73B71
:100090003BCE016E84BCBFFDC12F3D6C74319ABD57
:1000A00056833DDA3D00C77F11BED9E4BB4C3E917B
:1000B0006BAAAABE000000803F05A84CCDB2D44E6A
:1000C000B93836A9020C50B9918688083CA6AAAA6C
:1000D0002ABE000000803F4D383420582059205A55
:1000E00020450043616E6E6F7420656E74657220EA
:1000F0007375626469723A20004D3234004D3233B8
:10010000202573006175746F25692E670065727212
:100110006F722077726974696E6720746F206669E8
:100120006C65004E6F74205344207072696E746960
:100130006E67005344207072696E74696E67206246
:10014000797465200044656C6574696F6E20666122
:10015000696C65642C2046696C653A200046696CC0
:10016000652064656C657465643A006F70656E2027
:100170006661696C65642C2046696C653A2000579D
:10018000726974696E6720746F2066696C653A20C5
:10019000002E0A006F70656E206661696C65642CC4
:1001A0002046696C653A20002E0A006F70656E204B
:1001B0006661696C65642C2046696C653A2000466E
:1001C000696C652073656C656374656400205369B0
:1001D0007A653A200046696C65206F70656E6564CB
:1001E0003A20006F70656E206661696C65642C2032
:1001F00046696C653A20004E6F77206672657368B9
:100200002066696C653A20004E6F7720646F696ED6
:10021000672066696C653A20002220706F730022A7
:1002200020706172656E743A2200535542524F55E8
:1002300054494E452043414C4C20746172676574AB
:100240003A22004B494C4C45442E20007472796987
:100250006E6720746F2063616C6C207375622D670C
:10026000636F64652066696C6573207769746820C4
:10027000746F6F206D616E79206C6576656C732E7E
:10028000204D4158206C6576656C2069733A0053A7
:10029000442063617264206F6B006F70656E526FF3
:1002A0006F74206661696C656400766F6C756D654E
:1002B0002E696E6974206661696C65640053442020
:1002C000696E6974206661696C0046696C616D6570
:1002D0006E742073657474696E67733A2044697331
:1002E00061626C65640020204D323030204400464D
:1002F000696C616D656E742073657474696E677383
:100300003A0020430020440020490020204D333093
:10031000312050005049442073657474696E6773CE
:100320003A0020460020420020204D313435204D37
:100330003120480020460020420020204D31343535
:10034000204D302048004D6174657269616C2068F1
:10035000656174757020706172616D65746572732A
:100360003A00205A0020590020204D3230362058C3
:1003700000486F6D65206F666673657420286D6D2B
:10038000293A00204500205A002058002042002031
:10039000540020204D323035205300416476616E88
:1003A000636564207661726961626C65733A20539B
:1003B0003D4D696E20666565647261746520286DC7
:1003C0006D2F73292C20543D4D696E207472617617
:1003D000656C20666565647261746520286D6D2F9B
:1003E00073292C20423D6D696E696D756D207365B2
:1003F000676D656E742074696D6520286D73292C96
:1004000020583D6D6178696D756D205859206A6579
:10041000726B20286D6D2F73292C20205A3D6D6141
:1004200078696D756D205A206A65726B20286D6D34
:100430002F73292C2020453D6D6178696D756D20E5
:1004400045206A65726B20286D6D2F73290020543A
:100450000020520020204D32303420500041636390
:10046000656C65726174696F6E733A20503D70728D
:10047000696E74696E672C20523D72657472616397
:100480007420616E6420543D74726176656C002046
:100490004500205A0020590020204D32303120588C
:1004A000004D6178696D756D20416363656C65729F
:1004B0006174696F6E20286D6D2F7332293A0020A8
:1004C0004500205A0020590020204D32303320585A
:1004D000004D6178696D756D206665656472617443
:1004E000657320286D6D2F73293A00204500205A2E
:1004F0000020590020204D39322058005374657077
:10050000732070657220756E69743A004861726478
:10051000636F6465642044656661756C742053651F
:100520007474696E6773204C6F6164656400457212
:10053000726F722077726974696E6720746F2045DC
:100540004550524F4D21004572726F723A006563FB
:10055000686F3A0020496E76616C69642065787432
:100560007275646572200053544F505045442E20DC
:10057000005072696E7465722073746F7070656478
:100580002064756520746F206572726F72732E20FF
:1005900046697820746865206572726F7220616E9A
:1005A0006420757365204D39393920746F20726568
:1005B00073746172742E202854656D706572617455
:1005C0007572652069732072657365742E2053659A
:1005D0007420697420616674657220726573746139
:1005E0007274696E6729005072696E746572206852
:1005F000616C7465642E206B696C6C2829206361C2
:100600006C6C656421004B494C4C45442E20002005
:10061000746F6F206C6F6E67206578747275736984
:100620006F6E2070726576656E7465640020636F0E
:100630006C6420657874727573696F6E2070726572
:1006400076656E746564006F6B00526573656E64E9
:100650003A2000536C6565702E2E2E00FFFFFF00C0
:1006600000AF430080AC430000CD430000A0400039
:1006700000A04000000040000000000000A0C000FA
:10068000000000000000000000A0C000000000000A
:1006900000AF430000AA430000CD43334420507212
:1006A000696E7465722072656164792E005265739B
:1006B000756D696E67207072696E74005761697438
:1006C00020666F7220757365722E2E2E004E6F207D
:1006D0006D6F76652E00456E642066696C65206CD2
:1006E00069737400426567696E2066696C65206C89
:1006F000697374002569206D696E2C20256920734B
:100700006563004B494C4C45442E20002042403A42
:100710000020403A00202F00205400202F002042CB
:100720003A00202F0020543A006F6B004865617436
:10073000696E6720646F6E652E003F0020573A0097
:1007400020453A00543A0048656174696E672E2E60
:100750002E0042656420646F6E652E0020423A00D0
:1007600020453A00543A0042656420486561746946
:100770006E672E003344205072696E746572204F8C
:1007800066662E004649524D574152455F4E414DD7
:10079000453A4D61726C696E2056313B2053707240
:1007A000696E7465722F6772626C206D6173687513
:1007B0007020666F722067656E36204649524D572D
:1007C0004152455F55524C3A68747470733A2F2FFA
:1007D0006769746875622E636F6D2F4D61726C6905
:1007E0006E4669726D776172652F4D61726C696ECC
:1007F0002050524F544F434F4C5F56455253494F30
:100800004E3A312E30204D414348494E455F5459B0
:1008100050453A3344205072696E746572204558D1
:100820005452554445525F434F554E543A3120552A
:100830005549443A30303030303030302D3030305F
:10084000302D303030302D303030302D30303030B1
:1008500030303030303030300A00205A3A002059E1
:100860003A0020436F756E7420583A200020453AB4
:1008700000205A3A0020593A00583A007A5F6D69D0
:100880006E3A2000795F6D696E3A2000785F6D697D
:100890006E3A20004D31343520533C696E646578E2
:1008A0003E206F7574206F662072616E6765202828
:1008B000302D31290053657474696E67205472615C
:1008C00076656C20416363656C65726174696F6EF7
:1008D0003A200053657474696E67205265747261C2
:1008E000637420416363656C65726174696F6E3A0D
:1008F000200053657474696E67205072696E7420AD
:10090000416363656C65726174696F6E3A20005370
:10091000657474696E67205072696E7420616E64CC
:100920002054726176656C20416363656C65726109
:1009300074696F6E3A20004F66667365742061704B
:10094000706C6965642E004572723A20546F6F2096
:100950006661722100546F6F206661722066726F4B
:100960006D207265666572656E636520706F696E75
:100970007400220A00556E6B6E6F776E20636F6D88
:100980006D616E643A202200256920686F7572736C
:10099000202569206D696E7574657300446F6E65FE
:1009A000207072696E74696E672066696C65004BB1
:1009B000494C4C45442E200053544F505045442E32
:1009C00020005072696E7465722073746F70706568
:1009D000642064756520746F206572726F72732E67
:1009E0002046697820746865206572726F72206194
:1009F0006E6420757365204D39393920746F20720B
:100A00006573746172742E202854656D706572610F
:100A1000747572652069732072657365742E205336
:100A200065742069742061667465722072657374E0
:100A3000617274696E6729004E6F204C696E652083
:100A40004E756D62657220776974682063686563AE
:100A50006B73756D2C204C617374204C696E653A14
:100A600020004E6F20436865636B73756D20776956
:100A70007468206C696E65206E756D6265722C20DD
:100A80004C617374204C696E653A2000636865633D
:100A90006B73756D206D69736D617463682C204C88
:100AA000617374204C696E653A20004C696E652054
:100AB0004E756D626572206973206E6F74204C6193
:100AC0007374204C696E65204E756D6265722B31B2
:100AD0002C204C617374204C696E653A20004D31B6
:100AE0003130006F6B00446F6E6520736176696E04
:100AF000672066696C652E004D3239002020506CED
:100B0000616E6E6572427566666572427974657370
:100B10003A20002046726565204D656D6F72793A06
:100B20002000417567203330203230313700436F69
:100B30006D70696C65643A2000286E6F6E652C20BC
:100B400064656661756C7420636F6E666967290001
:100B5000207C20417574686F723A200041756720CF
:100B6000333020323031372031373A34353A343867
:100B700000204C61737420557064617465643A2080
:100B80000020312E312E3620646576004D61726C66
:100B9000696E0020536F66747761726520526573C9
:100BA000657400205761746368646F6720526573D1
:100BB0006574002042726F776E206F7574205265E5
:100BC000736574002045787465726E616C2052659F
:100BD00073657400506F776572557000584C414FC3
:100BE00044002200656E7175657565696E67202227
:100BF0000020746F6F206C6F6E672065787472755B
:100C000073696F6E2070726576656E74656400201E
:100C1000636F6C6420657874727573696F6E207091
:100C2000726576656E746564007C3C3E5E2B3D3F6C
:100C30002F5B5D3B2C2A225C0045303A20005A3A5B
:100C40002000593A2000583A20004D53312C4D5382
:100C5000322050696E730A004D38342058205920D4
:100C60005A20450024F404D9201BC40C5C0E9804BF
:100C7000C4095F0265077101F405F900FB04B300C4
:100C800048048700C1036900580355000303450069
:100C9000BE023A008402310053022A0029022500D4
:100CA00004022000E4011C00C8011900AF01170074
:100CB00098011400840113007101100061011000FB
:100CC00051010E0043010D0036010B002B010B00FA
:100CD00020010B00150109000C01090003010800A7
:100CE000FB000800F3000800EB000700E40006002A
:100CF000DE000600D8000600D2000600CC00050089
:100D0000C7000500C2000500BD000400B9000400D2
:100D1000B5000400B1000400AD000400A900040007
:100D2000A5000300A20003009F0004009B00030035
:100D30009800030095000200930003009000030058
:100D40008D0002008B000300880002008600020074
:100D500084000300810002007F0002007D00020089
:100D60007B0002007900020077000100760002009B
:100D70007400020072000100710002006F000200A6
:100D80006D0001006C0002006A00010069000200B1
:100D900067000100660001006500010064000200B8
:100DA0006200010061000100600001005F000200BC
:100DB0005D0001005C0001005B0001005A000100C1
:100DC00059000100580001005700010056000100C1
:100DD00055000100540001005300000053000100C1
:100DE0005200010051000100500001004F000100BD
:100DF0004E0000004E0001004D0001004C000100BB
:100E00004B0000004B0001004A00010049000100B6
:100E100048000000480001004700010046000000B3
:100E200046000100450000004500010044000100AB
:100E300043000000430001004200000042000100A6
:100E40004100000041000100400001003F0000009F
:100E50003F0001003E0000003E0001003D00000098
:100E60003D0001003C0000003C0000003C0001008F
:100E70003B0000003B0001003A0000003A00010086
:100E8000390000003900010038000000380000007F
:100E90003800010037000000370001003600000074
:100EA000360000003600010035000000350000006B
:100EB000350001003400000034000000340001005F
:100EC0003300000033000000330001003200000056
:100ED000320000003200010031000000310000004B
:100EE000310001003000000030000000300001003F
:100EF0002F0000002F0000002F0000002F00010035
:100F00002E0000002E0000002E0001002D00000029
:100F10002D0000002D0000002D0001002C0000001D
:100F20002C0000002C0000002C0001002B00000011
:100F30002B0000002B0000002B0001002A00000005
:100F40002A0000002A0000002A00010029000000F9
:100F500029000000290000002900000029000100EC
:100F600028000000280000002800000028000000E1
:100F700028000100270000002700000027000000D3
:100F800027000000270001002600000026000000C6
:100F900026000000260000002600010025000000B9
:100FA00025000000250000002500000025000000AD
:100FB000250001002400000024000000240000009F
:100FC0002400000024000100230000002300000092
:100FD0002300000023000000230000002300000085
:100FE0002300010022000000220000002200000077
:100FF0002200000022000000220001002100000069
:10100000210000002100000021000000210000005C
:10101000210000002100010020000000200000004D
:101020002000000020000000200000002000000040
:1010300020000000200001001F0000001F00000031
:101040001F0000001F0000001F0000001F00000024
:101050001F0001001E0000001E0000001E00000016
:101060001E00000024F4D43050C38E20C2A24017CA
:10107000828B7011127A910D816CD90AA861E108F6
:10108000C7586607615143061E4B5D05C145A7045D
:101090001A411104093D9803713931034036DB02CE
:1010A00065339102D4305402802E1D02632CEE0170
:1010B000752AC501B028A001102781018F25640180
:1010C0002B244B01E0223401AC211F018D200D01A6
:1010D000801FFC00841EED00971DDF00B81CD200AD
:1010E000E61BC600201BBC00641AB200B219A8009F
:1010F0000A19A0006A189900D117910040178B00B7
:10110000B516840031167E00B31579003A157300C8
:10111000C7146F0058146A00EE136600881363004A
:1011200025135E00C7125B006C12570015125400A5
:10113000C111510070114F0021114B00D610490010
:101140008D1047004610440002104200C00F4000BE
:10115000800F3E00420F3C00060F3B00CB0E3800D4
:10116000930E37005C0E3500270E3400F30D32006D
:10117000C10D3100900D3000600D2E00320D2D009C
:10118000050D2C00D90C2B00AE0C2900850C290074
:101190005C0C2700350C27000E0C2600E80B240001
:1011A000C40B2400A00B23007D0B23005A0B21004D
:1011B000390B2100180B2000F80A1F00D90A1E0065
:1011C000BB0A1E009D0A1D00800A1D00630A1C0048
:1011D000470A1B002C0A1B00110A1A00F7091A0003
:1011E000DD091900C4091900AB091900920917009B
:1011F0007B091800630917004C0916003609160010
:10120000200916000A091500F5081500E008140069
:10121000CC081400B8081400A408140090081300A7
:101220007D0812006B0813005808120046081200CF
:1012300034081100230811001208110001081100E0
:10124000F0071000E0071000D0071000C0071000E2
:10125000B0070F00A107100091070E0083070F00D1
:1012600074070F0065070E0057070E0049070E00B0
:101270003B070D002E070E0020070D0013070D0081
:1012800006070D00F9060C00ED060D00E0060C0047
:10129000D4060C00C8060C00BC060C00B0060C00FE
:1012A000A4060B0099060C008D060B0082060B00AD
:1012B00077060B006C060B0061060A0057060B0050
:1012C0004C060A0042060A0038060A002E060A00EA
:1012D00024060A001A060A001006090007060A007A
:1012E000FD050900F4050900EB050900E205090008
:1012F000D9050900D0050900C7050900BE05090088
:10130000B5050800AD050800A50509009C05080005
:10131000940508008C050800840508007C05080079
:10132000740508006C050700650508005D050700E9
:10133000560508004E050700470507004005080050
:1013400038050700310507002A05070023050700B7
:101350001C050600160507000F0507000805060016
:1013600002050700FB040600F5040700EE04060072
:10137000E8040600E2040700DB040600D5040600CA
:10138000CF040600C9040600C3040600BD0406001D
:10139000B7040600B1040500AC040600A60406006C
:1013A000A00405009B0406009504050090040600B7
:1013B0008A04050085040500800406007A040500FF
:1013C00075040500700405006B0405006604050043
:1013D000610405005C040500570405005204050083
:1013E0004D04050048040500430405003E040400C4
:1013F0003A04050035040500300404002C040500FF
:1014000027040400230405001E0404001A04040039
:1014100016040500110404000D040400090405006D
:101420000404040000040400FC030400F8030400A6
:10143000F4030400F0030400EC030400E8030400D8
:10144000E4030400E0030400DC030400D803040008
:10145000D4030400D0030400CC030400C803030039
:10146000C5030300656E6473746F707320686974DC
:101470003A205A00205A3A00656E6473746F707394
:10148000206869743A20590020593A00656E6473E7
:10149000746F7073206869743A20580020583A00BD
:1014A000656E6473746F7073206869743A200045C8
:1014B00072723A204D494E54454D502042454400E9
:1014C0004D494E54454D5020747269676765726589
:1014D00064004572723A204D415854454D502042A7
:1014E0004544004D415854454D502074726967671A
:1014F0006572656400626564002C2073797374659D
:101500006D2073746F707065642120486561746527
:10151000725F49443A2000544845524D414C205294
:10152000554E4157415900546865726D616C2052A7
:10153000756E61776179004B494C4C45442E200013
:10154000202D20496E76616C69642065787472750F
:10155000646572206E756D62657220210070012CC9
:101560000190012701B0012201C0011D01F0011805
:10157000011002130130020E016002090190020401
:1015800001C002FF000003FA004003F5008003F0F1
:1015900000D003EB002004E6007004E100E004DC6E
:1015A000004005D700C005D2004006CD00D006C8D7
:1015B000008007C3003008BE00F008B900C009B4BD
:1015C00000B00AAF00B00BAA00D00CA500000EA01E
:1015D00000500F9B00C01096005012910000148C18
:1015E00000C0158700B0178200B0197D00D01B78AD
:1015F00000001E730040206E0090226900F02464F9
:101600000040275F0090295A00E02B5500102E5013
:101610000020304B0010324600E033410090353C52
:10162000001037370070383200A0392D00B03A284A
:1016300000A03B2300603C1E00103D1900903D14AB
:1016400000103E0F00703E0A00C03E0500003F0043
:101650000048656174696E67206661696C65640045
:1016600048656174696E67206661696C65640045F0
:1016700072723A204D494E54454D50004D494E54DA
:10168000454D5020747269676765726564004572E4
:10169000723A204D415854454D50004D41585445E3
:1016A0004D5020747269676765726564004B6420F1
:1016B0000023646566696E65202044454641554CAB
:1016C000545F004B69200023646566696E652020C5
:1016D00044454641554C545F004B702000236465DF
:1016E00066696E65202044454641554C545F005064
:1016F0004944204175746F74756E652066696E6922
:1017000073686564212050757420746865206C616D
:101710007374204B702C204B6920616E64204B64E5
:1017200020636F6E7374616E74732066726F6D20C8
:1017300062656C6F7720696E746F20436F6E6669A7
:101740006775726174696F6E2E680050494420415C
:1017500075746F74756E65206661696C65642120AF
:1017600074696D656F75740020403A006F6B20548A
:101770003A006F6B20423A00504944204175746F23
:1017800074756E65206661696C6564212054656DB1
:10179000706572617475726520746F6F2068696717
:1017A0006800204B643A2000204B693A2000204B0F
:1017B000703A200020436C61737369632050494480
:1017C00020002054753A2000204B753A2000206DEF
:1017D00061783A2000206D696E3A200020643A203A
:1017E0000020626961733A200000000000000000E0
:1017F00000000000007FFFE000000000000000008B
:10180000000000007000E000000000000000000088
:10181000000000630C6000000000000000000000F9
:101820000000470E20000000000000000000000043
:10183000004F0F200000000000000000000000002A
:101840005F0FA00000000000000000000000005E2C
:1018500007A07F80000000000000004104004060FD
:1018600020FFC00000000000000020820040F020A7
:10187000FFC00000000000000020820040F020FFB8
:10188000C0000000000000004104004060207F8094
:10189000000000000000008208005E07A07F8000BA
:1018A0000000000000010410005F0FA0FFC0000056
:1018B00000000000010410004F0F20FFC0000000D6
:1018C00000000000820800470E20FFC0000000005A
:1018D000000000410400630C603F000000000000B5
:1018E00000000000007000E01E000000000000008A
:1018F00001FFFF807FFFE00C0000000000000001FE
:10190000FFFF800000000000000000000000000059
:1019100000007FFFE0000000000000000000000069
:10192000007000E000000000000000000000000067
:1019300061F86000000000000000000000000041AD
:10194000F82000000000000000000000000040F04F
:1019500020000000000000000000000000406020A7
:101960000000000000000000000000005801A07FFF
:1019700080000000000000004104005C63A0FFC084
:10198000000000000000002082005EF7A0FFC00001
:101990000000000000002082005EF7A0FFC00000F1
:1019A00000000000004104005C63A07F8000000094
:1019B000000000008208005801A07F8000000000A5
:1019C000000001041000406020FFC0000000000083
:1019D000000104100040F020FFC0000000000000E3
:1019E0000082080041F820FFC00000000000000055
:1019F00041040061F8603F000000000000000000AA
:101A000000007000E01E0000000000000001FFFF69
:101A1000807FFFE00C0000000000000001FFFF805D
:101A20000000002D2D2D2E2D2D002D2D2D002D2DC6
:101A30002D002D2D2D002D2D3A2D2D0009200009D2
:101A400020001FFFFFFFFFFFFF600000000001FFFD
:101A5000400000000000FF8000000000007F83CFF6
:101A600000000C303F87FF80000C301F867980001B
:101A70000C000F8C30C7838C30E78C30CFC7CC3153
:101A8000F38C30DCECEC33B98C30D86C6C33198CC3
:101A900030D06C0C33198C30D86C0C33198C30DC92
:101AA0006C0E3B198C30CF7C079F198C30C77C03A0
:101AB0008F194000000000000260000000000006D6
:101AC0001FFFFFFFFFFFF84D323100496E69742E92
:101AD0002053442063617264004E6F20534420639E
:101AE000617264004D3231004368616E6765205356
:101AF000442063617264005072696E742066726F74
:101B00006D2053440053746F70207072696E7400BE
:101B1000526573756D65207072696E7400506175E1
:101B20007365207072696E7400436F6E74726F6CAF
:101B300000507265706172650054756E6500496E83
:101B4000666F2073637265656E005072696E7420F3
:101B500066726F6D205344005072696E7420667215
:101B60006F6D20534400022E2E000152656672658F
:101B70007368004D61696E004D3234004D32332080
:101B8000257300526573746F7265206661696C73AA
:101B90006166650046696C616D656E74004D6F74B9
:101BA000696F6E0054656D70657261747572650061
:101BB0004D61696E0046696C2E204469612E2031AA
:101BC0000046696C2E204469612E2031004F666604
:101BD000004F6E20004520696E206D6D3300436F0D
:101BE0006E74726F6C004573746570732F6D6D0049
:101BF0004573746570732F6D6D005A7374657073DF
:101C00002F6D6D005A73746570732F6D6D0059736D
:101C1000746570732F6D6D005973746570732F6DDB
:101C20006D005873746570732F6D6D005873746513
:101C300070732F6D6D00412D74726176656C00417B
:101C40002D74726176656C00412D726574726163EA
:101C50007400412D7265747261637400416D617826
:101C6000206500416D6178206500416D6178207AC2
:101C700000416D6178207A00416D617820790041E2
:101C80006D6178207900416D6178207800416D6147
:101C9000782078005654726176206D696E00565433
:101CA000726176206D696E00566D696E00566D69C1
:101CB0006E00566D6178206500566D617820650074
:101CC000566D6178207A00566D6178207A00566DE5
:101CD0006178207900566D6178207900566D6178C1
:101CE000207800566D617820780056652D6A6572FF
:101CF0006B0056652D6A65726B00567A2D6A6572A7
:101D00006B00567A2D6A65726B005678792D6A657C
:101D1000726B005678792D6A65726B00416363655A
:101D20006C00416363656C00436F6E74726F6C008E
:101D3000507265686561742041425320636F6E661E
:101D4000005072656865617420504C4120636F6E6D
:101D500066005049442D43005049442D43005049EA
:101D6000442D44005049442D44005049442D49001D
:101D70005049442D49005049442D50005049442DAC
:101D800050002008204661637400200820466163EB
:101D900074002008204D6178002008204D617800F3
:101DA0002008204D696E002008204D696E004F66A6
:101DB00066004F6E20004175746F74656D7000464B
:101DC000616E2073706565640046616E2073706596
:101DD00065640042656400426564004E6F7A7A6C07
:101DE00065004E6F7A7A6C6500436F6E74726F6C2B
:101DF0000042656400426564004E6F7A7A6C65004B
:101E00004E6F7A7A6C650046616E2073706565640A
:101E10000046616E2073706565640054656D706581
:101E20007261747572650042656400426564004EBB
:101E30006F7A7A6C65004E6F7A7A6C650046616ED7
:101E40002073706565640046616E2073706565641B
:101E50000054656D706572617475726500436F6FD3
:101E60006C646F776E0050726568656174204142E2
:101E700053005072656865617420504C41004D38C4
:101E8000340044697361626C6520737465707065B9
:101E90007273004D6F7665206178697300536574C5
:101EA00020686F6D65206F666673657473004732D6
:101EB00038004175746F20686F6D65004D61696E03
:101EC0000050726568656174204142532042656428
:101ED00000507265686561742041425320416C6C0A
:101EE0000050726568656174204142532031005092
:101EF000726570617265005072656865617420502A
:101F00004C412042656400507265686561742050E0
:101F10004C4120416C6C00507265686561742050C2
:101F20004C4120310050726570617265004D6F76D2
:101F30006520302E316D6D004D6F766520316D6DF1
:101F4000004D6F76652031306D6D005072657061A7
:101F50007265004578747275646572004D6F7665C0
:101F6000205A004D6F76652059004D6F76652058D8
:101F7000004D6F76652061786973004578747275DD
:101F8000646572005A0059005800466C6F77203023
:101F900000466C6F77203000466C6F7700466C6FA0
:101FA000770046616E2073706565640046616E203F
:101FB00073706565640042656400426564004E6F3D
:101FC0007A7A6C65004E6F7A7A6C6500537065653D
:101FD00064005370656564004D61696E004D343274
:101FE000380000060900FE070192032120FFFF08C8
:101FF000FF07FF000000060000010707060200803F
:10200000808080800080030202060105A0A00507F1
:10201000070600005050F850F8505005070706001A
:10202000002078A07028F020050707060000C0C82F
:1020300010204098180507070600006090A040A8EF
:102040009068020303060104C040800307070601ED
:102050000020408080804020030707060100804068
:10206000202020408005050506000120A870A8203A
:102070000505050600012020F820200203030602C2
:10208000FFC04080050101060003F80202020602BB
:1020900000C0C005050506000108102040800507A6
:1020A0000706000070888888888870030707060183
:1020B0000040C040404040E005070706000070882F
:1020C00008708080F8050707060000F81020100847
:1020D00008F005070706000010305090F8101005B2
:1020E0000707060000F880F0080888700507070653
:1020F0000000708080F0888870050707060000F8EF
:10210000081020202020050707060000708888702E
:1021100088887005070706000070888878080870AE
:10212000020505060200C0C000C0C0020606060285
:10213000FFC0C000C0408004070706000010204018
:1021400080402010050303060002F800F80407078A
:10215000060100804020102040800507070600008F
:102160007088081020002005070706000070880806
:1021700068A8A870050707060000708888F8888896
:1021800088050707060000F08888F08888F00507B2
:1021900007060000708880808088700507070600A9
:1021A00000F08888888888F0050707060000F88016
:1021B00080F08080F8050707060000F88080F08036
:1021C0008080050707060000708880B88888700541
:1021D0000707060000888888F888888801070706AE
:1021E000020080808080808080050707060000381C
:1021F0001010101090600507070600008890A0C01E
:10220000A09088050707060000808080808080F805
:1022100005070706000088D8A8888888880507076A
:102220000600008888C8A898888805070706000067
:1022300070888888888870050707060000F08888FD
:10224000F080808005070706000070888888A890C5
:1022500068050707060000F08888F0A09088050749
:1022600007060000788080700808F0050707060060
:1022700000F820202020202005070706000088887D
:1022800088888888700507070600008888888888FD
:1022900050200507070600008888888888A8500510
:1022A0000707060000888850205088880507070621
:1022B000000088888850202020050707060000F8C5
:1022C0000810204080F8030707060100E0808080A6
:1022D0008080E00505050600018040201008030706
:1022E00007060100E02020202020E005030306006F
:1022F00004205088050101060000F80202020602CF
:1023000005804005050506000070087888780507F7
:10231000070600008080B0C88888F0050505060023
:10232000007080808870050707060000080868981C
:102330008888780505050600007088F88070050714
:10234000070600003048E040404040050606060011
:10235000FF7088887808700507070600008080B045
:10236000C888888801070706020080008080808076
:10237000800308080601FF200020202020A0400440
:102380000707060000808090A0C0A0900307070602
:102390000100C04040404040E0050505060000D077
:1023A000A8A8A8A8050505060000B0C88888880563
:1023B000050506000070888888700506060600FF7F
:1023C000F08888F080800506060600FF7888887807
:1023D0000808050505060000B0C8808080050505D1
:1023E00006000070807008F00407070600004040F7
:1023F000E040404030050505060000888888986860
:10240000050505060000888888502005050506009A
:10241000008888A8A85005050506000088502050AF
:10242000880506060600FF88888878087005050577
:10243000060000F8102040F80307070601002040BE
:102440004080404020010707060200808080808095
:10245000808003070706010080404020404080053F
:102460000202060002689000000006000000000062
:10247000060000000000060000000000060000004A
:10248000000006000000000006000000000006003A
:102490000000000006000000000006000000000030
:1024A000060000000000060000000000060000001A
:1024B000000006000000000006000000000006000A
:1024C0000000000006000000000006000000000000
:1024D00006000000000006000000000006000000EA
:1024E00000000600000000000600000000000600DA
:1024F00000000000060000000000060000000000D0
:1025000006000000000006000000000006000000B9
:1025100000000600000000000600000000000600A9
:10252000000000000600000000000600000000009F
:10253000060000010707060200800080808080807E
:102540000507070600002070A8A0A870200507074F
:10255000060000304040E04050A805050506000098
:102560008870507088050707060000885020F82002
:10257000F820010707060200808080008080800527
:1025800008080600003048205050209060030101E8
:10259000060107A0050707060000F888B8B8B88844
:1025A000F8050707060001700878887800F8050527
:1025B000050600012850A05028050303060001F875
:1025C000080802020206020640800507070600000E
:1025D000F888A88898A8F8050101060006F8040400
:1025E00004060003609090600507070600002020A5
:1025F000F8202000F804050506000360902040F054
:10260000030505060003E020E020E00202020602C6
:102610000640800508080600FF8888888898E880BA
:1026200080050707060000789898781818180202A5
:1026300002060202C0C00202020602FF4080030539
:102640000506000340C04040E00507070600017092
:102650008888887000F8050505060001A0502850FC
:10266000A00507070600008890A858B808080507C5
:10267000070600008890B84898203805080806002A
:1026800000C040C048D838080805070706000020E9
:102690000020408088700508080600004020007077
:1026A00088F888880508080600001020007088F85F
:1026B00088880508080600002050007088F888887F
:1026C0000508080600006890007088F888880508EA
:1026D000080600005000708888F8888805080806F9
:1026E00000002050207088F8888805070706000041
:1026F0003860A0B8E0A0B80508080600FF70888020
:102700008088702060050808060000402000F880DE
:10271000F080F8050808060000081000F880F08036
:10272000F8050808060000205000F880F080F80541
:1027300007070600005000F880F080F8030808063C
:102740000100804000E0404040E00308080601002E
:10275000204000E0404040E003080806010040A09F
:1027600000E0404040E0030707060100A000E04011
:102770004040E0050707060000704848E8484870F8
:1027800005080806000068900088C8A89888050811
:1027900008060000402070888888887005080806B0
:1027A00000001020708888888870050808060000DE
:1027B000205000708888887005080806000068901E
:1027C000007088888870050808060000500070882E
:1027D0008888887005050506000188502050880506
:1027E00008080600FF1070A8A8A8A87040050808EF
:1027F0000600004020888888888870050808060040
:102800000010208888888888700508080600002045
:1028100050008888888870050808060000500088E5
:1028200088888888700508080600001020885020D5
:102830002020200509090600FFC04070484870406C
:1028400040E00408080601FF609090A09090E080AE
:102850000508080600004020007008788878050800
:10286000080600001020007008788878050808061F
:1028700000002050007008788878050808060000DD
:1028800068900070087888780507070600005000F7
:102890007008788878050808060000205020700825
:1028A000788878050606060000D02878A0A850058C
:1028B00006060600FF708088702060050808060084
:1028C000004020007088F88070050808060000109D
:1028D00020007088F880700508080600002050006D
:1028E0007088F8807005070706000050007088F8AF
:1028F000807003080806010080400040C04040E0AE
:1029000003080806010020400040C04040E00308E2
:102910000806010040A00040C04040E00307070651
:102920000100A00040C04040E0050707060000A0ED
:1029300040A010788870050808060000689000B074
:10294000C88888880508080600004020007088882C
:1029500088700508080600001020007088888870BC
:102960000508080600002050007088888870050857
:1029700008060000689000708888887005070706C0
:102980000000500070888888700505050600012049
:1029900000F800200507070600FF1070A8A8A8701F
:1029A00040050808060000402000888888986805CF
:1029B0000808060000102000888888986805080824
:1029C00006000020500088888898680507070600E0
:1029D00000500088888898680509090600FF1020C3
:1029E00000888888F808700407070601FFC0406067
:1029F000506040E00508080600FF5000888888788D
:102A0000087000060900FE0000000000010900082F
:102A1000FE000005080806000040F0C88888987885
:102A200010050808060000C0F88888888888F8051E
:102A300005050600012030F83020050808060000D2
:102A40002070F820202020E00509090600FF2070F2
:102A5000A8A8B8888870200509090600FFE080C092
:102A6000B0A8283028280509090600FFF8A888889A
:102A7000888888A8F8050A0A0600FE2050505050A1
:102A800088A8A8887003030306000340A040000044
:102A90002100240027002A00000022002500280031
:102AA0002B00000020002300260029000202020261
:102AB00002020202040404040404040403030303E2
:102AC00003030303010101010101010101020408E3
:102AD00010204080010204081020408001020408F8
:102AE00010204080804020100804020100000001F6
:102AF00002000000000000000403070600000000C0
:102B0000000000000000000000000000494E46499F
:102B10004E4954594E414ECDCCCC3D0AD7233C179B
:102B2000B7D13877CC2B329595E6241FB14F0A00E8
:102B30000020410000C84200401C4620BCBE4CCAD8
:102B40001B0E5AAEC59D7400172FF833AC97ACC757
:102B5000F13311241FBECFEFD0E4DEBFCDBF13E0B1
:102B6000A0E0B1E0E4E2F0EB01E00BBF02C00790AF
:102B70000D92AE39B107D9F71BBE14E1AEE9B3E04F
:102B800001C01D92A235B107E1F71BE2C0E5DBE20F
:102B900004C02297FE010E94B7D7C834D107C9F7F5
:102BA0000E9465D20C9405D80C940000A0E0B0E01F
:102BB000ECEDF5E10C94D4D7EC015B0161157105E6
:102BC00019F0FB0191838083F9908F2D90E00E9492
:102BD000BBD7892BC9F7FDE2FF1621F4F990EE244B
:102BE000E39405C02BE2F21609F4F990EE248E016D
:102BF00001501040C8016CE07BE243E050E00E94CD
:102C00006518892B01F58E010E5F1F4FC8016FE01B
:102C10007BE245E050E00E946518892B19F48E0193
:102C2000095F1F4FA114B10419F0F501118300834E
:102C3000E0FC04C070E090E080E814C070E090E038
:102C400080E86FEF08C1C80164E17BE243E050E037
:102C50000E946518892B69F4A114B10429F470E06D
:102C600090E080EC6FE7F7C02296F501D183C08336
:102C7000F6CF8824992440E050E060E070E0EF2D2A
:102C8000E053EA30A0F5F2E0EF2A8E2D90E09C01AF
:102C900028703070E2FE06C0232B79F50894811C61
:102CA000911C2BC0232B19F0089481089108DB019B
:102CB000CA0112E0880F991FAA1FBB1F1A95D1F7EE
:102CC000480F591F6A1F7B1F440F551F661F771F30
:102CD0004E0F511D611D711D483929E9520729E91F
:102CE000620729E1720748F084E0E82A06C0EE3F57
:102CF00031F4E3FC39C098E0E92AF990C0CFE5331C
:102D000011F0E53189F529912D3219F4E0E1EE2A2F
:102D100005C02B3219F081E090E003C0299182E0D8
:102D200090E0E22FE053EA3018F0C81BD90B1CC02A
:102D300020E030E0FCE020383F075CF4C901880F58
:102D4000991F880F991F280F391F220F331F2E0F2D
:102D5000311DE991E053EA3068F3E4FE03C0309599
:102D600021953F4F820E931ECE2CDD24E1FE07C03D
:102D7000A114B10421F02197F501D183C083CB01C7
:102D8000BA010E9420D47B018C01F3E0CF22DD2424
:102D900023E0C216D10421F417FB109517F9109502
:102DA00057016801C801B70120E030E040E050E081
:102DB0000E9480D3882309F44AC097FE0DC02BE2FD
:102DC000E22E2BE2F22E9094819491089394C0E22B
:102DD000D0E000E010E012C093E4E92E9BE2F92E6F
:102DE000F6CFF7012591359145915491C601B50172
:102DF0000E9460D65B016C018C1A9D0A8C169D06A0
:102E000084F7D595C7950F5F1F4F0630110529F040
:102E10008CEF9FEFE80EF91EF1CFC501D6017C01C2
:102E20008D018C2D880F8D2D881F8F3F51F0C6018D
:102E3000B50120E030E040E050E00E9480D38823DC
:102E400031F482E290E090935114809350147E2DDF
:102E50009F2D802F612F272F392F482F562FB901F3
:102E6000CA01CDB7DEB7ECE00C94F0D72F923F92B9
:102E70005F926F927F928F929F92AF92BF92CF920A
:102E8000DF92EF92FF920F931F93CF93DF938C010A
:102E90001B01EA016115710519F0FB019183808323
:102EA000209749F0CE010297839728F020E030E088
:102EB00040E050E0F6C0F801A1908F018A2D90E02B
:102EC0000E94BBD7892BB9F7FDE2AF1631F4F801A8
:102ED000A1908F015524539407C0FBE2AF1619F45B
:102EE000F801A1908F015524209719F0C031D10528
:102EF000C1F4F0E3AF1679F4F8018081883711F05E
:102F0000883549F4F801A1800E5F1F4FF2E05F2A77
:102F1000C0E1D0E006C0209721F480E3A816E9F4D0
:102F200027C0C830D10531F1C930D10524F4C230F1
:102F3000D10531F50CC0CA30D10589F0C031D105B9
:102F4000F9F4C12CD12CE12CB8E0FB2E28C0C12C07
:102F5000D12CE12CA0E4FA2E22C0CAE0D0E0FCEC97
:102F6000CF2EFCECDF2EFCECEF2EFCE0FF2E17C08A
:102F7000C8E0D0E0C12CD12CE12CE0E1FE2E0FC046
:102F80009E01442737FD4095542F60E070E080E0BB
:102F900090E80E9478D7C901DA016C017D0120E038
:102FA00030E040E050E060E03E01882477FC80940F
:102FB000982C70EDB72EBA0CE9E0EB1570F48A2D61
:102FC00081548A3118F499ECB92E06C08A2D8156A5
:102FD0008A3150F589EAB82EBA0C8B2D90E08C1707
:102FE0009D0714F56F3FE1F0C216D306E406F5061F
:102FF000B0F0CA01B901A40193010E9432D79B012C
:10300000AC012B0D311D411D511D2130F0E03F075A
:10301000F0E04F07F0E85F0710F461E001C06FEFE8
:10302000F801A1908F01C5CF2114310481F06623EE
:1030300031F001501040F1011183008308C051FEAE
:103040001AC002501040F1011183008314C067FFC1
:1030500012C050FC05C02FEF3FEF4FEF5FE704C0F9
:1030600020E030E040E050E882E290E0909351149C
:103070008093501416C050FE08C05095409530956E
:1030800021953F4F4F4F5F4F0CC057FF0AC082E260
:1030900090E090935114809350142FEF3FEF4FEF37
:1030A0005FE7B901CA01DF91CF911F910F91FF90A6
:1030B000EF90DF90CF90BF90AF909F908F907F90D8
:1030C0006F905F903F902F900895FB01DC0141507D
:1030D000504088F08D9181341CF08B350CF4805E6B
:1030E000659161341CF06B350CF4605E861B6111D8
:1030F00071F3990B0895881BFCCFFB01DC01415053
:10310000504048F005900D920020C9F701C01D9273
:1031100041505040E0F70895FB0155915523A9F027
:10312000BF01DC014D9145174111E1F759F4CD0183
:103130000590002049F04D9140154111C9F3FB0164
:103140004111EFCF81E090E001970895FB01DC0190
:1031500004C08D910190801921F441505040C8F76E
:10316000881B990B0895FB01DC0102C001900D92B0
:1031700041505040D8F70895FB01DC018D91813416
:103180001CF08B350CF4805E619161341CF06B3562
:103190000CF4605E861B611189F3990B0895FB01A5
:1031A000DC010D900020E9F7119701900D920020AD
:1031B000E1F70895FC018191861721F08823D9F762
:1031C000992708953197CF010895FB01DC018D9176
:1031D000019080190110D9F3990B0895FB01DC01CE
:1031E00001900D920020E1F70895FB01DC014150B0
:1031F000504030F08D910190801919F40020B9F7FA
:10320000881B990B0895FB01DC014150504048F0A8
:1032100001900D920020C9F701C01D92415050400D
:10322000E0F70895AEE0B0E0E8E1F9E10C94DCD716
:103230000D891E898EE08C831A8309838FEF9FE7A7
:103240009E838D839E01275E3F4FCE0101966F893D
:10325000788DA9010E9436192F813885020F131F1E
:10326000F80110822E96E4E00C94F8D7ABE0B0E0C1
:10327000ECE3F9E10C94CED73C012B015A01FC019F
:1032800017821682838181FD03C06FEF7FEFC6C175
:103290009AE0892E1E010894211C311CF301238120
:1032A000F20123FD859123FF81912F01882309F4E9
:1032B000B2C1853239F423FD859123FF81912F011D
:1032C000853229F490E0B3010E94291BE7CF982FA3
:1032D000FF24EE249924FFE1FF15D0F09B3269F022
:1032E0009C3228F4903259F0933291F40EC09D3202
:1032F00049F0903369F441E024C052E0F52A84E0BB
:10330000F82A28C098E0F92A25C0E0E1FE2A22C068
:10331000F7FC29C0892F80538A3070F4F6FE05C06F
:10332000989C902C1124980E15C0E89CE02C112438
:10333000E80EF0E2FF2A0EC09E3229F4F6FC6BC1C3
:1033400040E4F42A07C09C3619F450E8F52A02C07C
:10335000983649F4F20123FD959123FF91912F01B5
:10336000992309F0B8CF892F8554833018F0805203
:10337000833038F444E050E0A40EB51E5FE3598377
:103380000FC0933631F0933779F0933509F056C07A
:1033900020C0F5018081898342E050E0A40EB51E73
:1033A000610101E010E012C0F501C080D180F6FC9F
:1033B00003C06FEF7FEF02C0692D70E042E050E084
:1033C000A40EB51EC6010E941E1B8C015FE7F522EC
:1033D00014C0F501C080D180F6FC03C06FEF7FEF11
:1033E00002C0692D70E042E050E0A40EB51EC60197
:1033F0000E94131B8C0150E8F52AF3FE07C01AC087
:1034000080E290E0B3010E94291BEA948E2D90E0A7
:1034100008171907A8F30EC0F601F7FC8591F7FE0F
:1034200081916F0190E0B3010E94291BE110EA94A1
:10343000015010400115110579F7EAC0943611F0DA
:10344000993669F5F7FE08C0F50120813181428186
:10345000538184E090E00AC0F501808191819C0154
:10346000442737FD4095542F82E090E0A80EB91E06
:103470009FE6F92257FF09C0509540953095219558
:103480003F4F4F4F5F4FE0E8FE2ACA01B901A1014B
:103490002AE030E00E94551BD82ED21840C0953744
:1034A00029F41F2D1F7E2AE030E01DC01F2D197F3B
:1034B0009F3661F0903720F4983509F0ACC00FC00A
:1034C000903739F0983709F0A6C004C028E030E002
:1034D0000AC0106114FD146020E130E004C014FD46
:1034E000166020E132E017FF08C0F50160817181AC
:1034F0008281938144E050E008C0F5018081918190
:10350000BC0180E090E042E050E0A40EB51EA101B5
:103510000E94551BD82ED2188FE7F82EF122F6FE06
:103520000BC05EEFF522D91438F4F4FE07C0F2FCAC
:1035300005C08FEEF82202C01D2D01C0192DF4FE2A
:103540000DC0FE01ED0DF11D8081803319F499EE5F
:10355000F92208C01F5FF2FE05C003C08F2D8678D8
:1035600009F01F5F0F2DF3FC14C0F0FE0FC01E15F5
:1035700010F09D2C0BC09D2C9E0C911A1E2D06C088
:1035800080E290E0B3010E94291B1F5F1E15C0F36B
:1035900004C01E1510F4E11A01C0EE2404FF0FC090
:1035A00080E390E0B3010E94291B02FF1DC001FDD2
:1035B00003C088E790E00EC088E590E00BC0802F44
:1035C000867891F001FF02C08BE201C080E2F7FC37
:1035D0008DE290E0B3010E94291B06C080E390E0D9
:1035E000B3010E94291B9A94D914C0F3DA94F10113
:1035F000ED0DF11D808190E0B3010E94291BDD20BB
:10360000A9F706C080E290E0B3010E94291BEA946A
:10361000EE20C1F743CEF30166817781CB012B9673
:10362000E2E10C94EAD7FC01059061507040011072
:10363000D8F7809590958E0F9F1F0895FC016150DB
:10364000704001900110D8F7809590958E0F9F1FC4
:1036500008950F931F93CF93DF938C01EB018B8120
:1036600081FF1BC082FF0DC02E813F818C819D8117
:103670002817390764F4E881F9810193F983E88315
:1036800006C0E885F985802F0995892B31F48E8154
:103690009F8101969F838E8302C00FEF1FEFC801A9
:1036A000DF91CF911F910F910895FA01AA27283039
:1036B00051F1203181F1E8946F936E7F6E5F7F4FFF
:1036C0008F4F9F4FAF4FB1E03ED0B4E03CD0670F7B
:1036D000781F891F9A1FA11D680F791F8A1F911DCE
:1036E000A11D6A0F711D811D911DA11D20D009F41E
:1036F00068943F912AE0269F11243019305D319360
:10370000DEF6CF010895462F4770405D4193B3E048
:103710000FD0C9F7F6CF462F4F70405D4A3318F0EF
:10372000495D31FD4052419302D0A9F7EACFB4E0A0
:10373000A6959795879577956795BA95C9F7009758
:103740006105710508959B01AC010A2E06945795F9
:10375000479537952795BA95C9F7620F731F841F50
:10376000951FA01D0895FC01128213820895FC018B
:103770008381882311F081E082830895FC01828196
:10378000811112820895CF93DF93DC01FC01EB5588
:10379000FE4F808191810097C9F1019791838083C9
:1037A000ED01CC5ADF4FFD01ED58FF4F8BE1019049
:1037B00009928150E1F7FD01EE5AFF4FAF58BF4F1C
:1037C0008D919C911197A157B04091838083FD0109
:1037D000ED58FF4F20E030E0AD014B555E4F10C07B
:1037E0002F5F3F4FEF01DF015F968BE10D90099254
:1037F0008150E1F7858D968D329791838083B196C4
:10380000DA018D919C912817390750F3DF91CF9100
:103810000895FC0189E693E0918380838781882362
:1038200021F0CF0104960E94A16C0895CF92DF92FF
:10383000EF92FF920F931F93DF93CF93CDB7DEB735
:103840006F970FB6F894DEBF0FBECDBF8C017B0122
:10385000095A1F4FD8018C9107551040882321F435
:103860002FE2C22ED12C03C090E5C92ED12CC00E60
:10387000D11E89E693E09A8389831C821B82188675
:103880001D82B6016C5F7F4FCE010596A70121E036
:103890000E94A573882381F5EEE4F5E007C08091CE
:1038A000C00085FFFCCF9093C60031969491992378
:1038B000B1F7E3EEF0E007C08091C00085FFFCCFD8
:1038C0009093C600319694919923B1F709C08091E5
:1038D000C00085FFFCCF0894E11CF11C9093C6004A
:1038E000F7019081992399F78091C00085FFFCCF63
:1038F0008AE08093C6005AC0F801EB55FE4F208144
:1039000031812A30310508F040C02F5F3F4F3183AD
:10391000208321503040F90185E0EE0FFF1F8A958A
:10392000E1F7E21BF30BED58FF4FE00FF11F13C05F
:10393000AF01415E5F4FBF018BE1DB010D90BD0127
:10394000DA010D92AD018150C1F7929182913296C8
:10395000968F858F7F9721503040BFEF2E3F3B07DA
:1039600039F7D801AD58BF4FF60134968BE101907D
:103970000D928150E1F70F581F4FF601828193811C
:10398000D8018D939C9301571040D801AC5ABF4F7A
:10399000FE0135968BE101900D928150E1F70E5AB0
:1039A0001F4F8B819C81F80191838083CE0101960A
:1039B0000E94091C6F960FB6F894DEBF0FBECDBFF4
:1039C000CF91DF911F910F91FF90EF90DF90CF90FB
:1039D0000895EF92FF920F931F938C013EECE32E1C
:1039E00031E0F32EE80EF91EC7010E94536CC701A7
:1039F0000E94A16CF801118210821F910F91FF901B
:103A0000EF900895CF92DF92EF92FF920F931F9362
:103A1000CF93DF937C016B01DB010D900020E9F770
:103A20008D0101501040061B170BEEECF1E0EE0E7D
:103A3000FF1ED7011C92E2E3FEEFEE0EFF1ECB014C
:103A40006EE470E00E94DA18EC01009731F4F8019E
:103A50003197EC0DFD1D86010EC060E270E00E9402
:103A6000DA188C010F5F1F4FCE016AE270E00E94EE
:103A7000DA18FC0131978DE081838AE0828313821A
:103A8000C70186539E4FB8010E94BF748EEC91E02F
:103A9000E80EF91ED7018C91882309F1E7E4F5E0DF
:103AA00007C08091C00085FFFCCF9093C60031967F
:103AB00094919923B1F7EDE0F1E007C08091C00047
:103AC00085FFFCCF9093C600319694919923B1F76E
:103AD0008091C00085FFFCCF8AE08093C600DF9113
:103AE000CF911F910F91FF90EF90DF90CF900895AD
:103AF000CF93DF93EC018B81882319F4E3E2F1E0AB
:103B00003AC0E3E3F1E007C08091C00085FFFCCF3D
:103B10009093C600319694919923B1F7CD57DD4F1C
:103B2000488159816A817B81C358D24082E294E006
:103B30002AE030E00E94B22F8091C00085FFFCCFC8
:103B40008FE28093C600C558DD4F488159816A8154
:103B50007B8182E294E02AE030E00E94B22F8091E3
:103B6000C00085FFFCCF0EC08091C00085FFFCCF58
:103B70009093C600319694919923B1F78091C0003B
:103B800085FFFCCF8AE08093C600DF91CF91089536
:103B90002F923F924F925F926F927F928F929F925D
:103BA000AF92BF92CF92DF92EF92FF920F931F934B
:103BB000DF93CF93CDB7DEB7AC970FB6F894DEBFE7
:103BC0000FBECDBF5C014B01FC018381882309F44A
:103BD00020C1C50182539E4F0E94A16CF501128243
:103BE0001A8A1D8A198A188A89E693E09F878E8728
:103BF0005EE4C52ED12CCA0CDB1C2FE230E0A20EF5
:103C0000B31EF601B182A08221ED3FEFA20EB31EDA
:103C1000F40180818F3209F081C0C4016FE270E04D
:103C20000E94DA187C010894E11CF11C3E01089402
:103C3000611C711C260142E1242E312C2C0E3D1EEC
:103C400068C0C7016FE270E00E94DA186C0100974B
:103C500009F472C0E816F90608F06EC08C010E195E
:103C60001F09C301B701A8010E940319060D171D02
:103C7000F8011082F30107C08091C00085FFFCCFDE
:103C800031969093C60090819923B1F78091C0003E
:103C900085FFFCCFFAE0F093C600F20160817181EC
:103CA0006115710519F460E070E002C06C5F7F4F30
:103CB000C101A30121E00E94A5738823F9F4EBE67A
:103CC000F1E007C08091C00085FFFCCF9093C60053
:103CD000319694919923B1F7FE01319607C08091F6
:103CE000C00085FFFCCF31969093C6009081992348
:103CF000B1F78091C00085FFFCCF84C02EE030E09A
:103D00002C0F3D1FF2013183208376010894E11CC2
:103D1000F11CE114F10409F094CF0BC080E590E0B0
:103D2000A80EB91EF601B182A08220EB3FEFA20ED1
:103D3000B31ED82C092D02C0DE2C0F2D8EE490E08E
:103D4000A80EB91EF5018081918122EB3FEFA20EF2
:103D5000B31E009719F480E090E001C004966D2D29
:103D6000702F0E947774882319F4E5E4F1E034C0E1
:103D7000EDE5F1E007C08091C00085FFFCCF909396
:103D8000C600319694919923B1F78D2D902F9C0107
:103D9000F90107C08091C00085FFFCCF3196909358
:103DA000C60090819923B1F78091C00085FFFCCFB8
:103DB0008AE08093C60083E892E0A80EB91EF50160
:103DC000108211821282138220C08091C00085FF70
:103DD000FCCF9093C600319694919923B1F78D2D25
:103DE000902F9C01F90107C08091C00085FFFCCF96
:103DF00031969093C60090819923B1F78091C000CD
:103E000085FFFCCF8EE28093C600CE010E960E9405
:103E1000091CAC960FB6F894DEBF0FBECDBFCF9194
:103E2000DF911F910F91FF90EF90DF90CF90BF90A7
:103E3000AF909F908F907F906F905F904F903F904A
:103E40002F900895BF92CF92DF92EF92FF920F933F
:103E50001F93CF93DF938C01EB018FE28993EE24C4
:103E6000E394FF2475EAC72E71E0D72EC00ED11E51
:103E70006FE1B62E14C0FB9CC00111248D589F4FDA
:103E8000800F911FBE010E94B36C02C02196E39483
:103E90008881882319F08CE88E15C0F7F3942F2DB4
:103EA00030E0F601808191812817390720F3E7FC83
:103EB00007C0C80182539E4FBE010E94B36C01C06F
:103EC0001882DF91CF911F910F91FF90EF90DF90BB
:103ED000CF90BF900895EF92FF920F931F93CF93CF
:103EE000DF93EC011B828EA9882321F0CE01C396BB
:103EF0000E94A16CE7EAEE2EE1E0FE2EEC0EFD1E24
:103F0000C70160E04FE10E94476A8823F9F4EEE4BC
:103F1000F5E007C08091C00085FFFCCF9093C600FC
:103F2000319694919923B1F7EDEBF2E007C08091BF
:103F3000C00085FFFCCF9093C600319694919923E1
:103F4000B1F78091C00085FFFCCF76C08E0104558B
:103F50001E4FC801B70141E00E945475882331F516
:103F6000C801B70140E00E9454758823F9F4E7E4E2
:103F7000F5E007C08091C00085FFFCCF9093C6009C
:103F8000319694919923B1F7EAEAF2E007C0809163
:103F9000C00085FFFCCF9093C60031969491992381
:103FA000B1F78091C00085FFFCCF46C0CE01C3961B
:103FB000B8010E94986F8823F9F4E7E4F5E007C0A0
:103FC0008091C00085FFFCCF9093C60031969491FC
:103FD0009923B1F7EAE9F2E007C08091C00085FFBC
:103FE000FCCF9093C600319694919923B1F78091BC
:103FF000C00085FFFCCF20C081E08B83EEE4F5E0BC
:1040000007C08091C00085FFFCCF9093C600319619
:1040100094919923B1F7EFE8F2E007C08091C000D6
:1040200085FFFCCF9093C600319694919923B1F708
:104030008091C00085FFFCCF8AE08093C600DE013E
:10404000AC5ABF4FFE01F3968BE101900D92815067
:10405000E1F789A99AA9CE5ADF4F99838883C2557F
:10406000D040CE018F96C25BDF4F99838883DF916A
:10407000CF911F910F91FF90EF9008952F923F9253
:104080004F925F926F927F929F92AF92BF92CF9228
:10409000DF92EF92FF920F931F93DF93CF93CDB7F1
:1040A000DEB7CC5BD0400FB6F894DEBF0FBECDBFFD
:1040B0006C01662309F0E5C027E832E0C20ED31E8A
:1040C000D6018C91E9E7FDEFCE0EDF1E882309F4BF
:1040D000E9C02FE732E0C20ED31ED601ED90FD906D
:1040E0000D911C91E1E8FDEFCE0EDF1E0E9458D02D
:1040F000E616F7060807190708F4D4C0C2C0C601BF
:104100000E946B1FD60113968C91882309F4CAC0B4
:1041100000D000D000D0EDB7FEB731967E010894F4
:10412000E11CF11CADB7BEB71296FC92EE9211974E
:1041300084E091E093838283D6019D968D919C913A
:104140009E97958384830E9412198701EDB7FEB76D
:1041500036960FB6F894FEBF0FBEEDBF57010AC0EA
:10416000D8018C91992787FD90950E94C3D7F801BB
:1041700081938F01F50101900020E9F73197EA1949
:10418000FB09802F8E198E175CF313E3A12EB12C3F
:10419000AC0CBD1CC50140E050E060E070E00E9446
:1041A000896B9924BBE0EB2EF12CEC0EFD1E2E0149
:1041B0000894411C511CABE26A2E712C6C0E7D1EC2
:1041C000FDEF2F2EF0E03F2E41C0D8018C9190E002
:1041D0000E94C3D7F80181938F01D7010D90002071
:1041E000E9F71197AE19BF09802F8E198A176CF362
:1041F0008C898E3759F1C701B20145E050E00E9429
:10420000F518009719F500D000D000D0EDB7FEB733
:104210003196ADB7BEB712967C926E9211973382EB
:104220002282558244820E941219EDB7FEB736965B
:104230000FB6F894FEBF0FBEEDBFC3010E946142EE
:1042400089EF90E00E94AE5399249394C501B70181
:1042500040E050E00E94BE6E181614F48701BDCFF6
:10426000992041F48FEF9FEFD6019E969C938E93F9
:104270009D9718C0F60185A596A5019696A785A7D6
:1042800011C027E832E0C20ED31ED6011C92E9E726
:10429000FDEFCE0EDF1ED60113968C91882309F414
:1042A0002ECF36CFC454DF4F0FB6F894DEBF0FBE0B
:1042B000CDBFCF91DF911F910F91FF90EF90DF90D5
:1042C000CF90BF90AF909F907F906F905F904F90F6
:1042D0003F902F9008952F923F924F925F926F924E
:1042E0007F928F929F92AF92BF92CF92DF92EF9286
:1042F000FF920F931F93DF93CF93CDB7DEB7C857CD
:10430000D0400FB6F894DEBF0FBECDBF7C015B017D
:104310003A01E1963FAF2EAFE1978DB79EB7E39696
:104320009FAF8EAFE397E4E0F0E06E0E7F1EC70113
:104330004296AF969FAF8EAFAF9725E0822E912C1D
:104340008E0C9F1CAD961FAEAD979CE4C92ED12C50
:10435000CC0EDD1EF701E857FD4FE996FFAFEEAF3B
:10436000E9978AE8282E82E0382E2E0C3F1C0BE0BD
:10437000402E512C4C0C5D1C80C1F6018385282FEA
:1043800030E0A901487150704031510509F081C1F8
:10439000E996EEADFFADE99780819181813091057D
:1043A00009F477C1029709F474C1FDB7E696FFAF2F
:1043B000E6978EB7E7968FAFE797F501019000205B
:1043C000E9F7EA19FB093D968DB79EB78E1B9F0B47
:1043D0000FB6F8949EBF0FBE8DBF0DB71EB70F5F0F
:1043E0001F4FF601DE0111969081903239F08E2F29
:1043F0008C19883011F48EE28D939D933196E415DB
:10440000F50591F71C92F8011082F501808188234F
:1044100029F4C80160E071E00E94CF18E4960FAF64
:10442000E497E5961FAFE597C801B5010E94CF1844
:10443000C801BE016F5F7F4F0E94CF18C80160E0C6
:1044400071E00E94CF181A8A1D8A198A188A89E693
:1044500093E09F878E87CE014296B301AE014F5FF6
:104460005F4F21E00E94A573882309F03DC0E996C3
:10447000EEADFFADE99780819181892BA9F5EEE43E
:10448000F5E007C08091C00085FFFCCF9093C60087
:10449000319694919923B1F7E2E0F1E007C0809161
:1044A000C00085FFFCCF31969093C6009081992380
:1044B000B1F78091C00085FFFCCFFAE0F093C60011
:1044C000FE01319607C08091C00085FFFCCF319678
:1044D0009093C60090819923B1F78091C00085FF29
:1044E000FCCF8AE08093C600DE01D196FE01729671
:1044F0008BE101900D928150E1F78889998998AB01
:104500008FA7E9E6F3E0FEA7EDA7C701E4966FAD3C
:10451000E497E5967FADE597AE01435D5F4F20E000
:1045200030E00E946B21CE018D960E94091CCE01C5
:104530000E960E94091CE6962FADE697E7963FADD2
:10454000E797C9010FB6F8949EBF0FBE8DBF95C007
:104550008E3209F492C0F70182898E3209F48DC03F
:1045600023FD8BC080E04031510509F481E0F70163
:104570008483882349F4F6018085873409F07DC05F
:1045800081858E3709F479C0E996EEADFFADE997E4
:10459000808191818130910531F082309105E1F186
:1045A000892B41F06AC0F10180819181019691834C
:1045B000808363C0D401F6018081803241F08E2F68
:1045C0008C19883011F48EE28D9380818D93319611
:1045D000E415F50589F71C92F50107C08091C0002C
:1045E00085FFFCCF31969093C60090819923B1F757
:1045F000F40107C08091C00085FFFCCF31969093F5
:10460000C60090819923B1F78091C00085FFFCCF4F
:104610009AE09093C60031C0D401F60180818032C7
:1046200041F08E2F8C19883011F48EE28D938081A9
:104630008D933196E415F50589F71C92E196EEAD60
:10464000FFADE197309739F0CF01B4010E94BC185B
:10465000892B61F423C0AD96FFADAD972F2F30E0CD
:10466000F1018081918128173907C1F0AD96FFAD26
:10467000AD97FF5FAD96FFAFAD97C301B601AF96A3
:104680004EAD5FADAF970E94BE6E18160CF475CE9E
:1046900005C0F6018081882309F05ACFE3968EADDC
:1046A0009FADE3970FB6F8949EBF0FBE8DBFC8585D
:1046B000DF4F0FB6F894DEBF0FBECDBFCF91DF91B5
:1046C0001F910F91FF90EF90DF90CF90BF90AF9030
:1046D0009F908F907F906F905F904F903F902F9022
:1046E0000895EF92FF920F931F93DF93CF93CDB76F
:1046F000DEB76F970FB6F894DEBF0FBECDBF7C015B
:104700008C01025B1F4F805B9F4FF8019183808378
:1047100028E832E0E20EF31E21E030E0F7012193B9
:1047200031937F011182108226E73DEFE20EF31EE6
:10473000049640E050E060E070E00E94896BF80170
:1047400020813181DE011596F90134968BE10190CB
:104750000D928150E1F7F901828193819C838B83D3
:1047600089E693E09A838983C70165E171E08E0150
:104770000F5F1F4FA80120E030E00E946B21C801AD
:104780000E94091CF701E657FD4F808191816F96C9
:104790000FB6F894DEBF0FBECDBFCF91DF911F9152
:1047A0000F91FF90EF900895CF92DF92EF92FF92DA
:1047B0000F931F93DF93CF93CDB7DEB76F970FB6ED
:1047C000F894DEBF0FBECDBF7C016A018C01025B95
:1047D0001F4F805B9F4FF8019183808328E832E070
:1047E000E20EF31E22E030E0F701219331937F01C6
:1047F0007183608326E73DEFE20EF31E049640E0EE
:1048000050E060E070E00E94896BF8012081318106
:10481000DE011596F90134968BE101900D928150DD
:10482000E1F7F901828193819C838B8389E693E090
:104830009A838983C70165E171E08E010F5F1F4F85
:10484000A80196010E946B21C8010E94091C6F9665
:104850000FB6F894DEBF0FBECDBFCF91DF911F9191
:104860000F91FF90EF90DF90CF9008952F923F929D
:104870004F925F926F927F928F929F92AF92BF9270
:10488000CF92DF92EF92FF920F931F93DF93CF931C
:10489000CDB7DEB7AD970FB6F894DEBF0FBECDBF74
:1048A0007C014B014DA7DC0113968C91882309F400
:1048B00021C3E1EDF1E0EE0EFF1ED7018C91EFE296
:1048C000FEEFEE0EFF1E882309F412C1222319F019
:1048D000EEE4F5E0E4C029EE31E0E20EF31ED7018C
:1048E0008C91E7E1FEEFEE0EFF1E882319F4EEE453
:1048F000F5E035C0E7E4F5E007C08091C00085FF32
:10490000FCCF9093C600319694919923B1F7ECE4D3
:10491000F2E007C08091C00085FFFCCF9093C600F5
:10492000319694919923B1F782E294E061E070E0CE
:104930004AE050E00E9406308091C00085FFFCCF25
:104940008AE08093C60083E492E00E940934D2C2D8
:104950008091C00085FFFCCF9093C6003196949162
:104960009923B1F7EAE2F2E007C08091C00085FF29
:10497000FCCF9093C600319694919923B1F7F4013E
:1049800007C08091C00085FFFCCF31969093C60090
:1049900090819923B1F7EFE1F2E007C08091C00068
:1049A00085FFFCCF9093C600319694919923B1F77F
:1049B000C7012EEE31E0E20EF31EB7010E94221F66
:1049C0004BEF5FEFE40EF51ED7019C91E7E1FEEFA0
:1049D000EE0EFF1E8DE8989FF0011124E251FE4F6C
:1049E000EE0DFF1D07C08091C00085FFFCCF319602
:1049F0009093C60090819923B1F7E9E1F2E007C0F6
:104A00008091C00085FFFCCF9093C60031969491B1
:104A10009923B1F723E832E0E20EF31ED7014D915E
:104A20005D916D917C91EDE7FDEFEE0EFF1E82E250
:104A300094E02AE030E00E94B22F8091C00085FF10
:104A4000FCCF8AE08093C600A70147515E4FDA0190
:104A50002C91E22FF0E0EE0FFF1FEE0FFF1FEE0D87
:104A6000FF1DE651FE4F83E892E0E80EF91ED701E4
:104A7000AD90BD90CD90DC908DE79DEFE80EF91ED6
:104A8000A082B182C282D3822F5FDA012C932AC026
:104A90008091C00085FFFCCF9093C6003196949121
:104AA0009923B1F7E8E0F2E007C08091C00085FFEC
:104AB000FCCF9093C600319694919923B1F7F401FD
:104AC00007C08091C00085FFFCCF31969093C6004F
:104AD00090819923B1F78091C00085FFFCCF8AE0D7
:104AE0008093C600C70182539E4F0E94A16C37C0BD
:104AF000E9EEF1E0EE0EFF1ED7011C92E7E1FEEFBA
:104B0000EE0EFF1EEEE4F5E007C08091C00085FFC9
:104B1000FCCF9093C600319694919923B1F7E7EFBB
:104B2000F1E007C08091C00085FFFCCF9093C600E4
:104B3000319694919923B1F7F40107C08091C00098
:104B400085FFFCCF31969093C60090819923B1F7F1
:104B50008091C00085FFFCCF8AE08093C600D7011A
:104B600012961C921A8A1D8A198A188A89E693E07D
:104B70009F878E87F701E25BFF4F2FE230E0E20E66
:104B8000F31EF182E08241ED5FEFE40EF51ED401E9
:104B90008C918F3209F07FC064010894C11CD11C34
:104BA0003E010894611C711C2F0132E1232E312C2F
:104BB0002C0E3D1E6BC0C6016FE270E00E94DA1839
:104BC0005C01009709F473C0C816D90608F06FC0DD
:104BD0008C010C191D09C301B601A8010E9403191B
:104BE000060D171DF8011082F30107C08091C00067
:104BF00085FFFCCF31969093C60090819923B1F741
:104C00008091C00085FFFCCFFAE0F093C600D2018E
:104C10006D917C916115710519F460E070E002C03E
:104C20006C5F7F4FC101A30121E00E94A57388231F
:104C300011F5E3EEF1E007C08091C00085FFFCCFE5
:104C40009093C600319694919923B1F7FE01319665
:104C500007C08091C00085FFFCCF31969093C600BD
:104C600090819923B1F78091C00085FFFCCF8EE23F
:104C70008093C6003BC12EE030E02C0F3D1FF201B7
:104C80003183208365010894C11CD11CC114D10457
:104C900009F091CF0AC040E550E0E40EF51EF18224
:104CA000E08280EB9FEFE80EF91E840101C08601CF
:104CB000F701E25BFF4F9DA5992309F4B6C060811F
:104CC00071816115710519F460E070E002C06C5FDC
:104CD0007F4FC70182539E4FA80121E00E94A57318
:104CE000882319F4EBEAF1E083C0AFEDB1E0EA0EFE
:104CF000FB1EF70140815181628173812CE930E014
:104D0000E20EF31ED7014D935D936D937C93139741
:104D1000E5E8FDEFEE0EFF1EE5EDF1E007C0809146
:104D2000C00085FFFCCF9093C600319694919923E3
:104D3000B1F7F80107C08091C00085FFFCCF319624
:104D40009093C60090819923B1F7EDECF1E007C094
:104D50008091C00085FFFCCF9093C600319694915E
:104D60009923B1F782E294E02AE030E00E94B22F6A
:104D70008091C00085FFFCCF8AE08093C60023E8C5
:104D800032E0E20EF31ED7011D921D921D921C927D
:104D90001397EDE7FDEFEE0EFF1EEFEBF1E007C01E
:104DA0008091C00085FFFCCF9093C600319694910E
:104DB0009923B1F78091C00085FFFCCF8AE08093F2
:104DC000C600C70160E070E0A8010E94D423D701AB
:104DD00052968C91882309F485C087010E5E1F4F7F
:104DE00081C08091C00085FFFCCF9093C6003196B2
:104DF00094919923B1F7F80107C08091C00085FF15
:104E0000FCCF31969093C60090819923B1F7E8EAE0
:104E1000F1E007C08091C00085FFFCCF9093C600F1
:104E2000319694919923B1F761C0608171816115C8
:104E3000710519F460E070E002C06C5F7F4FC7013C
:104E400082539E4FA80126E50E94A573882339F559
:104E5000E4E9F1E007C08091C00085FFFCCF9093AA
:104E6000C600319694919923B1F7F80107C080915B
:104E7000C00085FFFCCF31969093C60090819923A6
:104E8000B1F7E1E9F1E007C08091C00085FFFCCFF8
:104E90009093C600319694919923B1F727C081E091
:104EA000F7018083EFE7F1E007C08091C00085FF44
:104EB000FCCF9093C600319694919923B1F7F401F9
:104EC00007C08091C00085FFFCCF31969093C6004B
:104ED00090819923B1F78091C00085FFFCCF8AE0D3
:104EE0008093C600C80160E00E94689BCE010E96C8
:104EF0000E94091CAD960FB6F894DEBF0FBECDBF61
:104F0000CF91DF911F910F91FF90EF90DF90CF90A5
:104F1000BF90AF909F908F907F906F905F904F90D9
:104F20003F902F900895EF92FF920F931F93CF938E
:104F3000DF93EC010E949E7A8E0107511E4FD8012B
:104F40008C91BEECEB2EB1E0FB2EEC0EFD1E882307
:104F5000A1F1C7010E94A16CF801608161506083DA
:104F60008DE8689FB001112462517E4F6C0F7D1F48
:104F7000CE0141E021E00E943624D801EC91F0E01E
:104F8000EE0FFF1FEE0FFF1FEC0FFD1FE651FE4F50
:104F90004081518162817381CD57DD4F48835983B0
:104FA0006A837B83C358D240C7010E94896B8B817F
:104FB000882399F181E08A8330C0C7010E94A16CE7
:104FC0001A8287ED90E00E94AE53809109098823F0
:104FD00021F1109209098091D706082F10E0E8010D
:104FE000CC0FDD1FC55ADF4E68817981882777FD98
:104FF0008095982F0E9422D420917A0230917B02D2
:1050000040917C0250917D020E948ED518162CF49E
:1050100019821882C8010E94D785DF91CF911F9114
:105020000F91FF90EF900895FC0181E08183CF0103
:1050300040E021E00E9436240895EF92FF920F9302
:105040001F93DF93CF93CDB7DEB76F970FB6F8946A
:10505000DEBF0FBECDBF7C0188E892E0E80EF91EEE
:10506000F7011182108288E79DEFE80EF91E870193
:105070000D5C1F4FC80140E050E060E070E00E940E
:10508000896BDE011596F8018BE101900D9281503C
:10509000E1F7F70181A992A99C838B8389E693E0CC
:1050A0009A838983C70165E171E08E010F5F1F4F0D
:1050B000A80120E030E00E946B21C8010E94091C79
:1050C0006F960FB6F894DEBF0FBECDBFCF91DF91C4
:1050D0001F910F91FF90EF900895CF93DF93EC0114
:1050E0001BAA1EAA1AAA19AA89E693E098AB8FA751
:1050F000CC5ADF4F188223961882C755D040FE0144
:10510000E05BFF4FCE5ADF4F19821882C255D04064
:1051100091838083DE01A159BF4FFD0120E030E083
:10512000482F148217821382128240839183215E5A
:105130003F4F7F9681E02633380799F7C855DE4FF9
:1051400089E1888323961882689618822B961882A4
:1051500023961882C15DD140FE01E653FE4FC45331
:10516000DE4F1982188240839183C155DF4F188228
:1051700019821A821B822896188219821A821B822F
:10518000C358D2401A821B8218821982CB55DE4F37
:1051900019821882CC5BDF4F1882FD01C901119280
:1051A0000197E9F7C256DF4F81E08883C758D240A4
:1051B0001EA61DA60E9458D0C158DD4F68577C4ED0
:1051C0008F4F9F4F688379838A839B83DF91CF9131
:1051D00008951F93182F882371F5EEE4F5E007C0BA
:1051E0008091C00085FFFCCF9093C60031969491CA
:1051F0009923B1F7ECEFF4E007C08091C00085FF80
:10520000FCCF9093C600319694919923B1F7809189
:10521000C00085FFFCCF8AE08093C600EEE4F5E095
:1052200007C08091C00085FFFCCF9093C6003196E7
:1052300094919923B1F74091B9085091BA086091BF
:10524000BB087091BC0884EF94E00E9486384091BE
:10525000BD085091BE086091BF087091C00881EFF1
:1052600094E00E9486384091C1085091C208609134
:10527000C3087091C4088EEE94E00E948638409175
:10528000C5085091C6086091C7087091C8088BEE98
:1052900094E00E9486388091C00085FFFCCF8AE0B0
:1052A0008093C600112371F5EEE4F5E007C080910C
:1052B000C00085FFFCCF9093C6003196949199234E
:1052C000B1F7E1EDF4E007C08091C00085FFFCCFAD
:1052D0009093C600319694919923B1F78091C000C4
:1052E00085FFFCCF8AE08093C600EEE4F5E007C0BE
:1052F0008091C00085FFFCCF9093C60031969491B9
:105300009923B1F74091A9085091AA086091AB0880
:105310007091AC0888EC94E00E9486384091AD080A
:105320005091AE086091AF087091B00885EC94E0A0
:105330000E9486384091B1085091B2086091B3083C
:105340007091B40882EC94E00E9486384091B508D0
:105350005091B6086091B7087091B8088FEB94E04F
:105360000E9486388091C00085FFFCCF8AE0809340
:10537000C600112371F5EEE4F5E007C08091C0008E
:1053800085FFFCCF9093C600319694919923B1F795
:10539000E1EAF4E007C08091C00085FFFCCF909364
:1053A000C600319694919923B1F78091C00085FF92
:1053B000FCCF8AE08093C600EEE4F5E007C0809160
:1053C000C00085FFFCCF9093C6003196949199233D
:1053D000B1F74091C9085091CA086091CB0870910B
:1053E000CC0888E994E00E9499384091CD0850910A
:1053F000CE086091CF087091D00885E994E00E94B2
:1054000099384091D1085091D2086091D308709199
:10541000D40882E994E00E9499384091D5085091CF
:10542000D6086091D7087091D8088FE894E00E9460
:1054300099388091C00085FFFCCF8AE08093C60038
:10544000112371F5EEE4F5E007C08091C00085FFFF
:10545000FCCF9093C600319694919923B1F7EDE576
:10546000F4E007C08091C00085FFFCCF9093C60098
:10547000319694919923B1F78091C00085FFFCCFBC
:105480008AE08093C600EEE4F5E007C08091C0009A
:1054900085FFFCCF9093C600319694919923B1F784
:1054A0004091DD085091DE086091DF087091E008BE
:1054B00084E594E00E9486384091E1085091E2082A
:1054C0006091E3087091E40881E594E00E948638D9
:1054D0004091E5085091E6086091E7087091E8086E
:1054E0008EE494E00E9486388091C00085FFFCCF56
:1054F0008AE08093C600112371F5EEE4F5E007C061
:105500008091C00085FFFCCF9093C60031969491A6
:105510009923B1F7EBE9F3E007C08091C00085FF64
:10552000FCCF9093C600319694919923B1F7809166
:10553000C00085FFFCCF8AE08093C600EEE4F5E072
:1055400007C08091C00085FFFCCF9093C6003196C4
:1055500094919923B1F74091D9085091DA0860915C
:10556000DB087091DC0882E993E00E948638409164
:10557000F5085091F6086091F7087091F8088FE8E7
:1055800093E00E9486384091A5085091A60860914A
:10559000A7087091A8088CE893E00E949938409180
:1055A000E9085091EA086091EB087091EC0889E8ED
:1055B00093E00E9486384091ED085091EE0860918A
:1055C000EF087091F00886E893E00E9486384091D9
:1055D000F1085091F2086091F3087091F40883E8A3
:1055E00093E00E9486388091C00085FFFCCF8AE05E
:1055F0008093C600112371F5EEE4F5E007C08091B9
:10560000C00085FFFCCF9093C600319694919923FA
:10561000B1F7E1E7F3E007C08091C00085FFFCCF60
:105620009093C600319694919923B1F78091C00070
:1056300085FFFCCF8AE08093C600EEE4F5E007C06A
:105640008091C00085FFFCCF9093C6003196949165
:105650009923B1F74091CB065091CC066091CD06CD
:105660007091CE0688E693E00E9486384091CF067E
:105670005091D0066091D1067091D20685E693E0F4
:105680000E9486384091D3065091D4066091D50689
:105690007091D60682E693E00E9486388091C00021
:1056A00085FFFCCF8AE08093C600112371F5EEE4FC
:1056B000F5E007C08091C00085FFFCCF9093C60045
:1056C000319694919923B1F7E6E4F3E007C0809115
:1056D000C00085FFFCCF9093C6003196949199232A
:1056E000B1F78091C00085FFFCCF8AE08093C600AF
:1056F000EEE4F5E007C08091C00085FFFCCF9093F9
:10570000C600319694919923B1F74091FB105091C6
:10571000FC10662757FD6095762F8AE393E00E9480
:1057200099384091FD105091FE10662757FD609505
:10573000762F87E393E00E9499384091FF105091B3
:105740000011662757FD6095762F84E393E00E9451
:1057500099388091C00085FFFCCF8AE08093C60015
:10576000112369F4EEE4F5E007C08091C00085FFE5
:10577000FCCF9093C600319694919923B1F7409154
:10578000011150910211662757FD6095762F88E22E
:1057900093E00E94993840910311509104116627BB
:1057A00057FD6095762F85E293E00E9499384091ED
:1057B000051150910611662757FD6095762F82E2FC
:1057C00093E00E9499388091C00085FFFCCF8AE069
:1057D0008093C600112371F5EEE4F5E007C08091D7
:1057E000C00085FFFCCF9093C60031969491992319
:1057F000B1F7E4E1F3E007C08091C00085FFFCCF82
:105800009093C600319694919923B1F78091C0008E
:1058100085FFFCCF8AE08093C600EEE4F5E007C088
:105820008091C00085FFFCCF9093C6003196949183
:105830009923B1F7409187025091880260918902C3
:1058400070918A028BE093E00E94863860918B020F
:1058500070918C0280918D0290918E020E94B28490
:10586000AB01BC0188E093E00E94863860918F0212
:105870007091900280919102909192020E94C08456
:10588000AB01BC0185E093E00E9486384091930211
:1058900050919402609195027091960282E093E09B
:1058A0000E9486388091C00085FFFCCF8AE08093FB
:1058B000C6008091CA06882309F441C0112371F5FE
:1058C000EEE4F5E007C08091C00085FFFCCF909327
:1058D000C600319694919923B1F7EFEEF2E007C03C
:1058E0008091C00085FFFCCF9093C60031969491C3
:1058F0009923B1F78091C00085FFFCCF8AE08093A7
:10590000C600EEE4F5E007C08091C00085FFFCCF43
:105910009093C600319694919923B1F74091480233
:105920005091490260914A0270914B0286EE92E0DA
:105930000E9486388091C00085FFFCCF20C01123D3
:1059400009F5EEE4F5E007C08091C00085FFFCCFCB
:105950009093C600319694919923B1F7EAECF2E066
:1059600007C08091C00085FFFCCF9093C6003196A0
:1059700094919923B1F78091C00085FFFCCF8AE014
:105980008093C6001F910895DF93CF93CDB7DEB704
:10599000E0970FB6F894DEBF0FBECDBFDE011196C3
:1059A000E5E1F3E080E101900D928150E1F7DE0145
:1059B0005196E5E0F3E080E101900D928150E1F72E
:1059C000DE019196E5EFF2E080E101900D928150C9
:1059D000E1F789819A81AB81BC818093B90890936A
:1059E000BA08A093BB08B093BC0889899A89AB898F
:1059F000BC898093A9089093AA08A093AB08B093A0
:105A0000AC0889A19AA1ABA1BCA18093C9089093CD
:105A1000CA08A093CB08B093CC088D819E81AF813A
:105A2000B8858093BD089093BE08A093BF08B0933B
:105A3000C0088D899E89AF89B88D8093AD089093F9
:105A4000AE08A093AF08B093B0088DA19EA1AFA1FE
:105A5000B8A58093CD089093CE08A093CF08B093BB
:105A6000D00889859A85AB85BC858093C1089093C1
:105A7000C208A093C308B093C408898D9A8DAB8DDA
:105A8000BC8D8093B1089093B208A093B308B093F3
:105A9000B40889A59AA5ABA5BCA58093D10890931D
:105AA000D208A093D308B093D4088D859E85AF8586
:105AB000B8898093C5089093C608A093C708B0938F
:105AC000C8088D8D9E8DAF8DB8A18093B508909339
:105AD000B608A093B708B093B8088DA59EA5AFA54A
:105AE000B8A98093D5089093D608A093D708B0930F
:105AF000D8080E94375580E090E0AAE7B4E480938C
:105B0000DD089093DE08A093DF08B093E00880934F
:105B1000E1089093E208A093E308B093E40880932F
:105B2000E5089093E608A093E708B093E80820E022
:105B300030E040E050E02093D9083093DA084093F9
:105B4000DB085093DC0880E29EE4A0E0B0E08093A4
:105B5000A5089093A608A093A708B093A80820933F
:105B6000F5083093F6084093F7085093F80880E062
:105B700090E0A0EAB1E48093E9089093EA08A0934A
:105B8000EB08B093EC088DEC9CECACECBEE380939E
:105B9000ED089093EE08A093EF08B093F00880E032
:105BA00090E0A0EAB0E48093F1089093F208A0930B
:105BB000F308B093F4082093D3063093D4064093AF
:105BC000D5065093D6062093CF063093D006409347
:105BD000D1065093D2062093CB063093CC06409347
:105BE000CD065093CE0684EB90E09093FC1080930A
:105BF000FB1088E290E09093FE108093FD101092CD
:105C000000111092FF1080EF90E0909302118093AA
:105C1000011186E490E09093041180930311109297
:105C20000611109205118AE999E9A1EBB1E480937C
:105C3000870290938802A0938902B0938A0261E759
:105C40007DE38AE89FE30E94AB8460938B027093AC
:105C50008C0280938D0290938E0260E070E084EE5F
:105C600092E40E94B98460938F02709390028093B3
:105C700091029093920280E090E0A0E8BFE38093CD
:105C8000930290939402A0939502B09396020E947F
:105C90000F821092CA0680E090E0A0E4B0E4809306
:105CA000480290934902A0934A02B0934B020E948B
:105CB0008833EEE4F5E007C08091C00085FFFCCF9B
:105CC0009093C600319694919923B1F7ECE0F5E0FA
:105CD00007C08091C00085FFFCCF9093C60031962D
:105CE00094919923B1F78091C00085FFFCCF8AE0A1
:105CF0008093C600E0960FB6F894DEBF0FBECDBF0E
:105D0000CF91DF9108951F920F920FB60F920BB6AD
:105D10000F9211242F933F934F938F939F93EF9361
:105D2000FF934091C600E0911E04F0911F0431964C
:105D30009F012F773070319780912004909121043A
:105D40002817390739F0E256FC4F408330931F047F
:105D500020931E04FF91EF919F918F914F913F915E
:105D60002F910F900BBE0F900FBE0F901F901895A4
:105D70009A01AB01203081EE380780E0480780E0CF
:105D8000580749F182E08093C00060E079E08DE33C
:105D900090E00E949AD72150304040405040CA01C4
:105DA000B90122E030E040E050E00E949AD7309301
:105DB000C5002093C4008091C10080618093C10020
:105DC0008091C10088608093C1008091C10080688B
:105DD0008093C10008951092C00020E130E0E7CF29
:105DE000209120043091210480911E0490911F0481
:105DF0008217930719F42FEF3FEF0EC0F901E25617
:105E0000FC4F80812F5F3F4F2F77307030932104FC
:105E100020932004282F30E0C901089580912004A8
:105E20009091210490931F0480931E040895089577
:105E30002F923F924F925F926F927F928F929F929A
:105E4000AF92BF92CF92DF92EF92FF920F931F9388
:105E5000DF93CF93CDB7DEB7A0970FB6F894DEBF30
:105E60000FBECDBF1C016A017B01411551056105C3
:105E7000710549F440E350E060E070E020E030E07C
:105E80000E94D12F56C0882499245401422E5524B3
:105E90006624772401E010E00C0F1D1F080D191D6A
:105EA000C701B601A30192010E9478D7F80160836F
:105EB0000894811C911CA11CB11CC701B601A3014F
:105EC00092010E9478D7C901DA016C017D01C114E9
:105ED000D104E104F104F1F681E0E82EF12CEC0E9E
:105EE000FD1EE80CF91C3E010894611C711CD501D3
:105EF000C4010197A109B1096C01C818D90816C0DD
:105F0000F601EE0DFF1D40814A3010F4405D01C0E6
:105F1000495C552747FD5095652F752FC10120E03D
:105F200030E00E94D12F0894E108F1086E147F043C
:105F300039F7A0960FB6F894DEBF0FBECDBFCF9154
:105F4000DF911F910F91FF90EF90DF90CF90BF9066
:105F5000AF909F908F907F906F905F904F903F9009
:105F60002F9008952115310539F48091C00085FFE7
:105F7000FCCF4093C60008950E94182F0895EF9219
:105F8000FF920F931F939A01E62EFF2400E010E08A
:105F9000B801A7010E94B22F1F910F91FF90EF90BF
:105FA0000895EF92FF920F931F93CF93DF93EC012D
:105FB0007A018B012115310539F48091C00085FFEC
:105FC000FCCFE092C6001BC02A303105B1F477FF48
:105FD00010C04DE250E060E070E020E030E00E9450
:105FE000D12F10950095F094E094E11CF11C011D57
:105FF000111DCE01B801A7012AE00E94182FDF91E0
:10600000CF911F910F91FF90EF900895EF92FF9223
:106010000F931F937B019A010027F7FC0095102F27
:10602000B801A7010E94D12F1F910F91FF90EF900F
:1060300008950F931F938C014DE050E060E070E0F5
:1060400020E030E00E94D12FC8014AE050E060E03B
:1060500070E020E030E00E94D12F1F910F91089551
:10606000CF92DF92EF92FF920F931F938C019A01D0
:106070006B01EE24FF24B701A6010E94B22FC801D4
:106080000E9419301F910F91FF90EF90DF90CF90F9
:1060900008959F92AF92BF92CF92DF92EF92FF92BC
:1060A0000F931F93CF93DF93EC017A018B01922E14
:1060B000CB01BA0120E030E040E050E00E9480D304
:1060C00088236CF4CE014DE250E060E070E020E007
:1060D00030E00E94D12F17FB109517F9109520E0A2
:1060E00030E040E05FE3AA240BC0CA01B90120E020
:1060F00030E040E251E40E9487D39B01AC01A394BD
:10610000A91498F3C801B7010E94A7D25B016C01E2
:106110000E94F4D37B018C01CE01B801A7012AE0D3
:1061200030E00E94B22F992049F0CE014EE250E0BB
:1061300060E070E020E030E00E94D12FC801B7019C
:106140000E9420D49B01AC01C601B5010E94A6D2D9
:1061500022C020E030E040E251E40E9460D67B01A2
:106160008C010E94EFD35B016C01CC24B7FCC0947E
:10617000DC2CCE01B601A5012AE030E00E94D12F2F
:10618000C601B5010E9422D49B01AC01C801B70130
:106190000E94A6D29A949920E1F6DF91CF911F91A7
:1061A0000F91FF90EF90DF90CF90BF90AF909F90B6
:1061B00008950E94493008950F931F939C01220F68
:1061C000331FF901E75DFC4F0190F081E02DD9010B
:1061D000AA0FBB1F1E161F06E4F48D010C5C1D4F99
:1061E000BF01882777FD8095982F0E9422D49B01BC
:1061F000AC01F80160817181828193810E9487D313
:106200006093710270937202809373029093740290
:1062100028C0AC5CBD4F6D917D918D919C9120E02B
:1062200030E040E251E40E9487D3609371027093A2
:1062300072028093730290937402E6E1F1E007C06A
:106240008091C00085FFFCCF31969093C60090816D
:106250009923B1F78091C00085FFFCCF8AE080933D
:10626000C6001F910F910895EEE4F5E007C08091FC
:10627000C00085FFFCCF9093C6003196949199237E
:10628000B1F7E5E7F9E007C08091C00085FFFCCFDA
:106290009093C600319694919923B1F780918F081D
:1062A000909190089C01F90107C08091C00085FF82
:1062B000FCCF31969093C60090819923B1F7E2E725
:1062C000F9E007C08091C00085FFFCCF9093C60025
:1062D000319694919923B1F70895E6E5F1E007C06E
:1062E0008091C00085FFFCCF31969093C6009081CD
:1062F0009923B1F78091C00085FFFCCF8AE080939D
:10630000C600ECE8F8E007C08091C00085FFFCCF34
:106310009093C600319694919923B1F7329B03C0B4
:10632000EFE6F1E00AC0E4E7F1E007C08091C000C9
:1063300085FFFCCF31969093C60090819923B1F7E9
:106340008091C00085FFFCCF8AE08093C600E4E81E
:10635000F8E007C08091C00085FFFCCF9093C60095
:10636000319694919923B1F7339B03C0EFE6F1E0A6
:106370000AC0E4E7F1E007C08091C00085FFFCCFD0
:1063800031969093C60090819923B1F78091C00017
:1063900085FFFCCF8AE08093C600ECE7F8E007C0F9
:1063A0008091C00085FFFCCF9093C60031969491F8
:1063B0009923B1F7349B03C0EFE6F1E00AC0E4E7AC
:1063C000F1E007C08091C00085FFFCCF319690932B
:1063D000C60090819923B1F78091C00085FFFCCF62
:1063E0008AE08093C6000895EF92FF920F931F9367
:1063F000CF93DF93EC01E0905002F09051020091B6
:10640000520210915302688179818A819B81A8018F
:1064100097010E9480D3882324F4E882F9820A83BA
:106420001B83E0905402F0905502009156021091A7
:1064300057026C817D818E819F81A80197010E9406
:1064400080D3882324F4EC82FD820E831F83609125
:1064500058027091590280915A0290915B0220E09B
:1064600030E040E050E00E94A7D27B018C016885BB
:1064700079858A859B85A80197010E9480D388230E
:1064800024F4E886F9860A871B87E0905C02F09086
:106490005D0200915E0210915F02688179818A81BC
:1064A0009B81A80197010E948ED5181624F4E882DA
:1064B000F9820A831B83E0906002F09061020091F0
:1064C0006202109163026C817D818E819F81A8019F
:1064D00097010E948ED5181624F4EC82FD820E835B
:1064E0001F83E0906402F0906502009166021091B3
:1064F0006702688579858A859B85A80197010E9436
:106500008ED5181624F4E886F9860A871B87DF9152
:10651000CF911F910F91FF90EF9008958F929F92CE
:10652000AF92BF92CF92DF92EF92FF920F931F93A1
:10653000CF93DF93EC014B01FB01E080F1800281FE
:106540001381C801B701288139814A815B810E948A
:10655000A6D25B016C0120E030E040E050E00E94F8
:1065600080D3882309F47AC0E091D706F0E0EE0FDB
:10657000FF1FEE0FFF1FE359FF4E60817181828183
:1065800093812091690230916A0240916B0250918F
:106590006C020E9480D388232CF5E882F9820A835A
:1065A0001B83EEE4F5E007C08091C00085FFFCCFBF
:1065B0009093C600319694919923B1F7EDE2F6E0FD
:1065C00007C08091C00085FFFCCF9093C600319634
:1065D00094919923B1F78091C00085FFFCCF8AE0A8
:1065E0008093C600C601B5010E94EFD397FF07C094
:1065F00090958095709561957F4F8F4F9F4F685B09
:1066000072408040904054F1F40180819181A281D8
:10661000B38188839983AA83BB83EEE4F5E007C046
:106620008091C00085FFFCCF9093C6003196949175
:106630009923B1F7EFE0F6E007C08091C00085FF35
:10664000FCCF9093C600319694919923B1F7809135
:10665000C00085FFFCCF8AE08093C600DF91CF9118
:106660001F910F91FF90EF90DF90CF90BF90AF9070
:106670009F908F9008955E9A1092C1065E9A109234
:10668000C2065E9A1092C3065E9A0895EF92FF9238
:106690000F931F937B018C018091CA06882349F1D7
:1066A000C801B70120E030E040E050E00E9480D314
:1066B0008823F9F0C801B70120E030E040E05FE353
:1066C0000E9460D67B018C012BED3FE049E450E451
:1066D0000E9460D6A80197010E9460D69B01AC0180
:1066E00060E070E080E89FE30E9487D3E62F692F87
:1066F00004C0E0E070E080E86FE32E2F372F482FD2
:10670000562FB901CA011F910F91FF90EF90089584
:10671000609148027091490280914A0290914B0227
:106720000E94463360934C0270934D0280934E0258
:1067300090934F0208950F931F93CF93DF9381306F
:10674000910549F46F5F7F4F09F046C083E294E002
:106750000E946D2841C0892B09F03EC06F5F7F4FBA
:10676000D9F589E693E09093EE058093ED0580914D
:10677000F405882321F081EF95E00E94A16CC9EA1D
:10678000D5E009E613E005C06F9784E0C337D8076A
:1067900051F0198308838F818823B1F3CE010496C9
:1067A0000E94A16CF1CF89E693E0998388838F8161
:1067B000882321F0CE0104960E94A16C89E693E023
:1067C000909353048093520480915904882321F0BC
:1067D00086E594E00E94A16CDF91CF911F910F910B
:1067E000089580E090E06FEF7FEF0E949B33089563
:1067F00081E090E06FEF7FEF0E949B3308958DEC76
:1068000096E060E00E94489B5E985E985E985E9875
:106810000895CF93DF930E94629BF8940E943A867A
:106820005E9A1092C1065E9A1092C2065E9A10920B
:10683000C3065E9AE7E4F5E007C08091C00085FFDB
:10684000FCCF9093C600319694919923B1F7E7EE6F
:10685000F5E007C08091C00085FFFCCF9093C60093
:10686000319694919923B1F78091C00085FFFCCFB8
:106870008AE08093C6007894C5E0D0E008C068EC58
:1068800070E080E090E00E9466D00E9468982197B6
:106890008FEFCF3FD80799F7F894FFCF83E097E0C9
:1068A0000E94093408950E9458D06093DD067093C9
:1068B000DE068093DF069093E006E0910907F091F1
:1068C0000A07E55FF84F80818823A1F4E7E4F6E04A
:1068D00007C08091C00085FFFCCF9093C600319621
:1068E00094919923B1F78091C00085FFFCCF8AE095
:1068F0008093C60008958F929F92AF92BF92CF92DD
:10690000DF92EF92FF920F931F93B9EFCB2EB6E079
:10691000DB2EA8E0AA2EB12CAC0CBD1CFCE08F2E07
:10692000912C8C0C9D1C20E030E040E752E40E944A
:1069300087D37B018C01C60124E030E0C20ED31E58
:10694000B601A5019401E7EDCE2EE6E0DE2E0E9411
:10695000095C1F910F91FF90EF90DF90CF90BF9057
:10696000AF909F908F90089589EF96E00E94F43148
:106970000E9458D06093DD067093DE068093DF0698
:106980009093E0068DEB96E065E077E00E948E3212
:106990006091B1067091B2068091B3069091B406F1
:1069A0002091F9063091FA064091FB065091FC06C1
:1069B0000E9480D38823E9F46091B5067091B606F1
:1069C0008091B7069091B8062091FD063091FE06A1
:1069D0004091FF06509100070E9480D3882349F41C
:1069E00060917102709172028091730290917402B1
:1069F0001AC06091440270914502882777FD809506
:106A0000982F0E9422D420917102309172024091FD
:106A10007302509174020E9460D620E030E048EC8E
:106A200052E40E9487D30E947B34A1EBB6E0E9EFE9
:106A3000F6E080E101900D928150E1F7089582E245
:106A400094E00E940E2FEAE4F6E007C08091C000B7
:106A500085FFFCCF9093C600319694919923B1F7AE
:106A60004091EB065091EC066091ED067091EE06B8
:106A70004F5F5F4F6F4F7F4F82E294E02AE030E03C
:106A80000E94D12F8091C00085FFFCCF8AE08093C7
:106A9000C6000E94533408951F939C01162FE7E40B
:106AA000F5E007C08091C00085FFFCCF9093C60041
:106AB000319694919923B1F708C08091C00085FF69
:106AC000FCCF9093C6002F5F3F4FF901949199231B
:106AD000A1F74091EB065091EC066091ED067091A4
:106AE000EE0682E294E02AE030E00E94D12F80910D
:106AF000C00085FFFCCF8AE08093C600112311F00F
:106B00000E941F3510929C0810929B081F910895B7
:106B1000682F772767FD7095809191089091920872
:106B20000E94DA189C01909394088093930880E067
:106B3000232B09F081E0089561EB76E0AB01485F1B
:106B40005F4F9B01245F3F4FCB016C5F7F4F0E94E3
:106B5000805508952F923F924F925F926F927F924D
:106B60008F929F92AF92BF92CF92DF92EF92FF925D
:106B70000F931F93DF93CF9300D000D0CDB7DEB734
:106B80009C838B838330910508F008C1FC01E45A93
:106B9000F94FA4906C01CC0CDD1CCC0CDD1C9601D3
:106BA0002F54394F3A8329830F2EF0E04F2EF0E017
:106BB0005F2EF0E06F2EF0E07F2EF02DF901408285
:106BC0005182628273820E949C35F601E15AF94F2C
:106BD000E590F590059114916A2D772767FD7095E2
:106BE000882777FD8095982F0E9422D44B015C0165
:106BF00039EF232E36E0332E2C0C3D1CC801B70193
:106C000020E030E040EC5FE30E9460D6A5019401F3
:106C10000E9460D6F1016083718382839383F601C1
:106C2000EC5CFD4F60817181828193816093710280
:106C30007093720280937302909374020E947B346B
:106C40000E949E7AE981FA81408251826282738237
:106C50000E949C3580E00E949479F601E559F94F35
:106C6000E590F59005911491C801B7019058A501E0
:106C700094010E9460D6F1016083718382839383C3
:106C8000609171027091720280917302909174020E
:106C90000E947B340E949E7A81E00E9494798B81CD
:106CA0009C810E94DC30C801B701A80197010E94B5
:106CB000A7D2A50194010E9460D6F101608371837F
:106CC000828393836091710270917202809173024A
:106CD000909174020E947B340E949E7AF601E958DA
:106CE000F94F6591759185919491F601E553F94FAE
:106CF000E080F18002811381A80197010E94A7D250
:106D0000E981FA816083718382839383F601ED5771
:106D1000F94F659175918591949120E5A22E22E01D
:106D2000B22EAC0CBD1CA80197010E94A7D2F501A0
:106D30006083718382839383F601E157F94F6591F4
:106D40007591859194912CE532E0C20ED31EA80175
:106D500097010E94A7D2F601608371838283938397
:106D60000E949C35E981FA8180819181A281B38161
:106D7000F10180839183A283B38340927102509288
:106D8000720260927302709274020E9491792B8158
:106D90003C812F53394F81E0F90180830F900F9090
:106DA0000F900F90CF91DF911F910F91FF90EF9077
:106DB000DF90CF90BF90AF909F908F907F906F901B
:106DC0005F904F903F902F900895FF920F931F93E5
:106DD0000E949E7A8091710290917202A09173023A
:106DE000B09174028093960890939708A0939808A6
:106DF000B093990880914402909145029093C906FE
:106E00008093C80684E690E0909345028093440204
:106E10000E9458D06093DD067093DE068093DF06F3
:106E20009093E00681E00E949479A9EFB6E0E1EB4F
:106E3000F6E080E101900D928150E1F780E090E072
:106E4000A0E0B0E08093710290937202A09373026D
:106E5000B093740288E50E948835F82E89E50E9477
:106E60008835182F8AE50E948835082FFF2039F4CD
:106E7000112339F480E0002329F481E003C01123B9
:106E800009F480E080937502882311F4FF2021F03B
:106E900080E090E00E94AA3580917502882311F469
:106EA000112321F081E090E00E94AA3580917502C3
:106EB000882311F4002321F082E090E00E94AA359B
:106EC0000E949C3580E00E94947980919608909170
:106ED0009708A0919808B0919908809371029093B7
:106EE0007202A0937302B09374028091C8069091CD
:106EF000C90690934502809344020E9458D0609343
:106F0000DD067093DE068093DF069093E0060E9414
:106F100091791F910F91FF900895E4EEF6E007C07C
:106F20008091C00085FFFCCF9093C600319694916C
:106F30009923B1F78091C00085FFFCCF8AE0809350
:106F4000C60083E294E00E941D28E6EDF6E007C04B
:106F50008091C00085FFFCCF9093C600319694913C
:106F60009923B1F78091C00085FFFCCF8AE0809320
:106F7000C6000895CF92DF92EF92FF920F931F9376
:106F8000DF93CF93CDB7DEB76E970FB6F894DEBF21
:106F90000FBECDBF0E9458D06093E5067093E60601
:106FA0008093E7069093E8062091E1063091E2068F
:106FB0004091E3065091E406621B730B840B950B22
:106FC00028EE33E040E050E00E9478D7F22EE32E26
:106FD000D42EC52E8DB79EB708970FB6F8949EBFD6
:106FE0000FBE8DBF0DB71EB70F5F1F4FCE010196AD
:106FF000EDB7FEB79283818384EF96E0F801938327
:107000008283622F732F842F952F2CE330E040E092
:1070100050E00E9478D7F801358324836F2D7E2DB0
:107020008D2D9C2D2CE330E040E050E00E9478D77D
:10703000F801778366830E941219EEE4F5E08DB7BC
:107040009EB708960FB6F8949EBF0FBE8DBF07C0BF
:107050008091C00085FFFCCF9093C600319694913B
:107060009923B1F7FE01319607C08091C00085FFDA
:10707000FCCF31969093C60090819923B1F780910F
:10708000C00085FFFCCF8AE08093C600CE01019648
:1070900060E00E94689B80910909882341F1109269
:1070A00009098091D706C82EDD247601EE0CFF1C5D
:1070B000EBE5F0E1EE0EFF1EF7016081718188279C
:1070C00077FD8095982F0E9422D420917A023091EA
:1070D0007B0240917C0250917D020E948ED5181651
:1070E00034F4F70111821082C6010E94D7856E9692
:1070F0000FB6F894DEBF0FBECDBFCF91DF911F91C9
:107100000F91FF90EF90DF90CF900895FC0107C0A2
:107110008091C00085FFFCCF9093C600319694917A
:107120009923B1F782E294E022E030E00E94D93066
:107130000895FC0107C08091C00085FFFCCF9093AB
:10714000C600319694919923B1F782E294E02AE047
:1071500030E00E94B22F08950E943A860E949E7AE3
:107160005E9A0E94A87A1092D9061092D80668EE0C
:1071700073E080E090E00E9466D084E797E060E0F2
:107180000E94489B0E9468980895E9E7F8E007C0CC
:107190008091C00085FFFCCF9093C60031969491FA
:1071A0009923B1F74091B1065091B2066091B306B0
:1071B0007091B40682E294E022E030E00E94D9307F
:1071C000E5E7F8E007C08091C00085FFFCCF909311
:1071D000C600319694919923B1F74091B50650912C
:1071E000B6066091B7067091B80682E294E022E09C
:1071F00030E00E94D930E1E7F8E007C08091C0009C
:1072000085FFFCCF9093C600319694919923B1F7F6
:107210004091B9065091BA066091BB067091BC06C8
:1072200082E294E022E030E00E94D930EDE6F8E01E
:1072300007C08091C00085FFFCCF9093C6003196B7
:1072400094919923B1F74091BD065091BE0660918B
:10725000BF067091C00682E294E022E030E00E9416
:10726000D930E2E6F8E007C08091C00085FFFCCF8E
:107270009093C600319694919923B1F780E00E94D3
:10728000647A0E9422D42091B9083091BA084091C2
:10729000BB085091BC080E9487D3AB01BC0182E2BD
:1072A00094E022E030E00E94D930EEE5F8E007C03B
:1072B0008091C00085FFFCCF9093C60031969491D9
:1072C0009923B1F781E00E94647A0E9422D4209130
:1072D000BD083091BE084091BF085091C0080E947F
:1072E00087D3AB01BC0182E294E022E030E00E944F
:1072F000D930EAE5F8E007C08091C00085FFFCCFF7
:107300009093C600319694919923B1F782E00E9440
:10731000647A0E9422D42091C1083091C208409121
:10732000C3085091C4080E9487D3AB01BC0182E21C
:1073300094E022E030E00E94D9308091C00085FFC7
:10734000FCCF8AE08093C60008952F923F924F921F
:107350005F926F927F928F929F92AF92BF92CF92E5
:10736000DF92EF92FF920F931F93DF93CF93CDB7EE
:10737000DEB768970FB6F894DEBF0FBECDBFDE0153
:107380001D96E1EBF6E08CE001900D928150E1F763
:10739000DE011196EBECF6E08CE001900D9281504D
:1073A000E1F71E010894211C311C7DE0472E512C71
:1073B0004C0E5D1E8824992466247724F401EF5333
:1073C000F94F8081882309F48BC0F201E080F180BD
:1073D00002811381F301E05BFD4FD301A45ABD4F3D
:1073E00060817181828193812D913D914D915C915C
:1073F0000E94A7D220E030E040E05FE30E9460D628
:107400009B01AC01C801B7010E948ED518165CF033
:107410000F2EF0E0AF2EF0E0BF2EF0E0CF2EF0E028
:10742000DF2EF02D0BC0F401EE0FFF1FEE0FFF1F3C
:10743000E958F94FA590B590C590D490C801B7010F
:10744000A60195010E94A6D27B018C0120E030E0CC
:1074500040EA51EC0E948ED5181634F5C801B701E8
:1074600020E030E040EA51E40E9480D38823E4F435
:10747000F1016081718182819381A80197010E944D
:10748000A6D2F1016083718382839383F201A0828B
:10749000B182C282D38224C08091C00085FFFCCF1C
:1074A0009093C600319602C0E7E4F5E094919923E9
:1074B00099F7E5E5F9E007C08091C00085FFFCCFB2
:1074C0009093C600319694919923B1F78091C000B2
:1074D00085FFFCCF8AE08093C60087E499E026C050
:1074E0000894811C911C84E090E0280E391E680EDF
:1074F000791E480E591E93E08916910409F05ECF5B
:10750000A1EBB6E0FE013D968CE001900D9281501A
:10751000E1F7ABECB6E0FE0131968CE001900D9204
:107520008150E1F70E949C3587E399E00E94629BBD
:1075300068960FB6F894DEBF0FBECDBFCF91DF9136
:107540001F910F91FF90EF90DF90CF90BF90AF9081
:107550009F908F907F906F905F904F903F902F9073
:1075600008952F923F924F925F926F927F928F92E7
:107570009F92AF92BF92CF92DF92EF92FF920F93C2
:107580001F93DF93CF93CDB7DEB7CB56D0400FB666
:10759000F894DEBF0FBECDBFA5969FAF8EAFA59767
:1075A000A7967FAF6EAFA797A8964FAFA897DB01BE
:1075B0006D917D918D919D916F96BFAFAEAF6F979D
:1075C000A3966CAF7DAF8EAF9FAFA397A796AEADDE
:1075D000BFADA79714966D917D918D919C91179752
:1075E0006D966CAF7DAF8EAF9FAF6D976091B1061A
:1075F0007091B2068091B3069091B40669966CAF13
:107600007DAF8EAF9FAF6997A3962CAD3DAD4EADCC
:107610005FADA3970E94A7D269AF7AAF8BAF9CAF43
:107620008091B5069091B606A091B706B091B806C4
:1076300065968CAF9DAFAEAFBFAF6597BC01CD0176
:107640006D962CAD3DAD4EAD5FAD6D970E94A7D24E
:107650006DAB7EAB8FAB98AF6091B9067091BA06F7
:107660008091BB069091BC0661966CAF7DAF8EAFEA
:107670009FAF6197A596AEADBFADA59718966D91DA
:107680007D918D919C911B9761962CAD3DAD4EAD3A
:107690005FAD61970E94A6D269AB7AAB8BAB9CAB16
:1076A000A596AEADBFADA5971C966D917D918D91C0
:1076B0009C911F972D966CAF7DAF8EAF9FAF2D978E
:1076C0006091BD067091BE068091BF069091C00684
:1076D00029966CAF7DAF8EAF9FAF2997A3968CADE7
:1076E0009DADAEADBFADA397B0588DA79EA7AFA778
:1076F000B8AB6D966CAD7DAD8EAD9FAD6D9790586E
:1077000069A77AA78BA79CA7A596AEADBFADA59795
:107710008D919D910D90BC91A02D25968CAF9DAF24
:10772000AEAFBFAF2597BC01CD0129AD3AAD4BAD92
:107730005CAD0E94A6D23B014C01A596AEADBFAD9B
:10774000A59714966D917D918D919C911797219697
:107750006CAF7DAF8EAF9FAF21972DA93EA94FA9EA
:1077600058AD0E94A6D25B016C016DA57EA58FA5C8
:1077700098A9A60195010E9460D67B018C0169A59C
:107780007AA58BA59CA5A40193010E9460D69B01BC
:10779000AC01C801B7010E94A6D21B012C016DA546
:1077A0007EA58FA598A9A40193010E9460D67B01B4
:1077B0008C0169A57AA58BA59CA5A60195010E94BF
:1077C00060D69B01AC01C801B7010E94A7D29B0102
:1077D000AC01C201B1010E941AD35B016C0120E02F
:1077E00030E040E050E00E9480D3882354F4C6018A
:1077F000B5012BED3FE049EC50E40E94A7D25B01BC
:107800006C01A896BFADA897BB2351F0C601B50186
:107810002BED3FE049EC50E40E94A6D25B016C01E5
:1078200069966CAD7DAD8EAD9FAD699725962CADFB
:107830003DAD4EAD5FAD25970E9480D3882321F5E5
:1078400065966CAD7DAD8EAD9FAD659721962CADE7
:107850003DAD4EAD5FAD21970E9480D38823A1F44A
:10786000C601B50120E030E040E050E00E9480D346
:10787000882351F4C601B5012BED3FE049EC50E4FB
:107880000E94A7D25B016C01A3966CAD7DAD8EAD5D
:107890009FADA3976D962CAD3DAD4EAD5FAD6D9791
:1078A0000E949BD59B01AC01C601B5010E9460D628
:1078B00029A93AA94BA95CA95F770E949BD57B01B6
:1078C0008C012FE632E143E85AE30E9480D387FD22
:1078D000EBC1C801B7010E945DD40E94F4D378A720
:1078E0006FA3672B21F4E1E0F0E0F8A7EFA32FA14D
:1078F00038A5B90180E090E00E9420D47B018C0182
:10790000C601B501A80197010E9487D36BA37CA390
:107910008DA39EA369A97AA98BA99CA9A801970107
:107920000E9487D36F8F78A389A39AA32D966CADFD
:107930007DAD8EAD9FAD2D9729962CAD3DAD4EAD55
:107940005FAD29970E94A6D2A80197010E9487D314
:107950006B8F7C8F8D8F9E8F6BA17CA18DA19EA143
:1079600020E030E040E05FEB0E9460D62BA13CA11C
:107970004DA15EA10E9460D620E030E040E85FE3C8
:107980000E94A7D26F8B788F898F9A8F61966CAD8A
:107990007DAD8EAD9FAD619769877A878B879C8718
:1079A00029968CAD9DADAEADBFAD29978D879E87D5
:1079B000AF87B88B6091440270914502882777FDAC
:1079C0008095982F0E9422D42091710230917202EA
:1079D00040917302509174020E9460D620E030E022
:1079E00040E752E40E9487D320E030E048EC52E4C4
:1079F0000E9487D3A9966FAFA997AA967FAFAA973F
:107A0000AB968FAFAB97AC969FAFAC97A1E0B0E0D1
:107A1000BA8BA98B662410C1B8E1B6150CF446C028
:107A20006DA57EA58FA598A92BA13CA14DA15EA116
:107A30000E9460D67B018C0169A57AA58BA59CA5C7
:107A40002F89388D498D5A8D0E9460D69B01AC01DB
:107A5000C801B7010E94A7D27B018C016DA57EA54C
:107A60008FA598A92F89388D498D5A8D0E9460D68F
:107A70005B016C0169A57AA58BA59CA52BA13CA1F6
:107A80004DA15EA10E9460D69B01AC01C601B5016B
:107A90000E94A6D26DA77EA78FA798AB6394C7015B
:107AA000D80189A79AA7ABA7BCA765C0E989FA89BD
:107AB000BF0180E090E00E9420D42BA13CA14DA109
:107AC0005EA10E9460D67B018C01C8010E9484D314
:107AD0006B8B7C8B8D8B9E8BB701C8010E94C3D6AC
:107AE0003B014C01A796AEADBFADA797ED90FD90C1
:107AF0000D911C9117FB109517F910956F96EEAD2F
:107B0000FFAD6F972080318042805380C801B7015C
:107B10002B893C894D895E890E9460D65B016C018E
:107B2000C201B101A40193010E9460D69B01AC0186
:107B3000C601B5010E94A7D26DA77EA78FA798ABFB
:107B4000C801B701A40193010E9460D67B018C019A
:107B5000C201B1012B893C894D895E890E9460D6A2
:107B60009B01AC01C801B7010E94A6D269A77AA700
:107B70008BA79CA7662469AD7AAD8BAD9CAD2DA576
:107B80003EA54FA558A90E94A7D269837A838B830B
:107B90009C836DA97EA98FA998AD29A53AA54BA56F
:107BA0005CA50E94A7D26D837E838F8398876985A9
:107BB0007A858B859C852F8D38A149A15AA10E9479
:107BC000A7D269877A878B879C876D857E858F850D
:107BD00098892B8D3C8D4D8D5E8D0E94A7D26D872F
:107BE0007E878F87988BCE0101960E94F431CE015B
:107BF0000196BE016B5F7F4FAE01475F5F4F9E01F5
:107C0000235F3F4FA996EFADA997AA96FFADAA971C
:107C1000AB96AFADAB97AC96BFADAC977F018D0186
:107C2000F7EDCF2EF6E0DF2E0E94095C29893A8914
:107C30002F5F3F4F3A8B298B69897A898FA198A54D
:107C40006817790708F4E8CEA5964EAD5FADA59705
:107C5000485F5F4FA5962EAD3FADA597245F3F4F80
:107C6000A5968EAD9FADA597DC011496BD01A99692
:107C7000EFADA997AA96FFADAA97AB96AFADAB971C
:107C8000AC96BFADAC977F018D01E7EDCE2EE6E05F
:107C9000DE2E0E94095CA1EBB6E0E9EFF6E080E1A0
:107CA00001900D928150E1F7C559DF4F0FB6F8945E
:107CB000DEBF0FBECDBFCF91DF911F910F91FF901F
:107CC000EF90DF90CF90BF90AF909F908F907F907C
:107CD0006F905F904F903F902F9008958091930800
:107CE00090919408019660E070E04AE050E00E94B4
:107CF0003617CB010895CF93DF93EC018091D7061F
:107D00008093EA0684E50E948835882309F440C000
:107D10000E946E3E8093EA06882309F439C0EEE49F
:107D2000F5E007C08091C00085FFFCCF9093C600AE
:107D3000319694919923B1F78091C00085FFFCCFD3
:107D40008DE48093C60082E294E0BE014AE050E0F8
:107D50000E940630E4E5F5E007C08091C00085FF91
:107D6000FCCF9093C600319694919923B1F782E2AB
:107D700094E06091EA0640E050E00E94BF2F8091BD
:107D8000C00085FFFCCF8AE08093C60081E001C07F
:107D900080E0DF91CF91089589E690E00E947B3EDC
:107DA000882309F00BC1E9E2F7E007C08091C00029
:107DB00085FFFCCF9093C600319694919923B1F73B
:107DC000E5E2F7E007C08091C00085FFFCCF90930B
:107DD000C600319694919923B1F7E091EA06F0E05C
:107DE000EE0FFF1FEE0FFF1FE359FF4E4081518141
:107DF0006281738182E294E021E030E00E94D93018
:107E0000E2E2F7E007C08091C00085FFFCCF9093CD
:107E1000C600319694919923B1F7E091EA06F0E01B
:107E2000EE0FFF1FE55AFF4E60817181882777FDB5
:107E30008095982F0E9422D4AB01BC0182E294E08D
:107E400021E030E00E94D930EEE1F7E007C08091F8
:107E5000C00085FFFCCF9093C60031969491992382
:107E6000B1F740917F105091801060918110709116
:107E7000821082E294E021E030E00E94D930EBE110
:107E8000F7E007C08091C00085FFFCCF9093C6004B
:107E9000319694919923B1F76091631070916410B9
:107EA000882777FD8095982F0E9422D4AB01BC01D2
:107EB00082E294E021E030E00E94D930E8E1F7E08E
:107EC00007C08091C00085FFFCCF9093C60031961B
:107ED00094919923B1F782E294E060E070E04AE087
:107EE00050E00E9406308091C00085FFFCCF8AE3FD
:107EF0008093C60040916D1050916E1060916F108C
:107F00007091701082E294E021E030E00E94D9305C
:107F1000E5E1F7E007C08091C00085FFFCCF9093BA
:107F2000C600319694919923B1F760915B107091DE
:107F30005C10882777FD8095982F0E9422D4AB0192
:107F4000BC0182E294E021E030E00E94D930E1E11E
:107F5000F7E007C08091C00085FFFCCF9093C6007A
:107F6000319694919923B1F78091EA060E94268276
:107F7000BC0182E294E04AE050E00E940630ECE06E
:107F8000F7E007C08091C00085FFFCCF9093C6004A
:107F9000319694919923B1F78FEF9FEF0E9426823B
:107FA000BC0182E294E04AE050E00E9406308091F9
:107FB000C00085FFFCCF8AE08093C600089583E56A
:107FC0000E948835882361F10E946E3E823010F154
:107FD000E7E4F5E007C08091C00085FFFCCF9093F7
:107FE000C600319694919923B1F7E4E9F8E007C00F
:107FF0008091C00085FFFCCF9093C600319694918C
:108000009923B1F78091C00085FFFCCF8AE080936F
:10801000C6000895882321F0813009F087C044C04C
:1080200088E40E948835882391F00E946E3E8A3A47
:1080300091051CF48AEA90E006C021E085309207A1
:1080400014F084E091E09093FC108093FB1086E4A0
:108050000E948835882381F00E946E3E8F3F9105F3
:1080600019F014F08FEF90E097FF02C080E090E0ED
:10807000909300118093FF1082E40E94883588233A
:1080800009F454C00E946E3E853091051CF485E0D1
:1080900090E005C08838910514F087E890E090934F
:1080A000FE108093FD10089588E40E94883588238F
:1080B00091F00E946E3E8A3A91051CF48AEA90E0A3
:1080C00006C021E08530920714F084E091E090939F
:1080D00002118093011186E40E948835882381F083
:1080E0000E946E3E8F3F910519F014F08FEF90E0E3
:1080F00097FF02C080E090E09093061180930511F5
:1081000082E40E948835882389F00E946E3E853083
:1081100091051CF485E090E005C08838910514F0C5
:1081200087E890E090930411809303110895809163
:10813000930890919408019660E070E04AE050E066
:108140000E94361708950F931F93CF93DF930091EA
:10815000930810919408C80165E470E00E94DA1851
:10816000EC01C8010196209749F0188260E070E0A8
:108170000E94D615E82F85E4888305C060E070E092
:108180000E94D615E82F4E2F592FCA01DF91CF91AB
:108190001F910F910895AF92BF92DF92EF92FF92DD
:1081A0000F931F93DF93CF9300D000D0CDB7DEB7EE
:1081B00085E40E948835882311F40E949E7A11EB91
:1081C000E12E16E0F12EDD2400E010E05E010894BF
:1081D000A11CB11CF801EB5DFC4F80810E94883529
:1081E0008823A1F00E94A340F701608371838283FA
:1081F000938369837A838B839C830330110519F001
:10820000DD24D39403C0C5010E9462550F5F1F4F48
:1082100084E090E0E80EF91E04301105D9F6DD2067
:1082200011F00E949C350F900F900F900F90CF91FE
:10823000DF911F910F91FF90EF90DF90BF90AF9073
:10824000089583E50E9488358823F9F00E94A340B1
:10825000AB01BC014093DD085093DE086093DF085A
:108260007093E0084093E5085093E6086093E708B0
:108270007093E8088FE099E00E9486388091C000F2
:1082800085FFFCCF8AE08093C60080E50E94883598
:108290008823B9F00E94A340AB01BC014093DD08E4
:1082A0005093DE086093DF087093E00882EF98E057
:1082B0000E9486388091C00085FFFCCF8AE08093C1
:1082C000C60082E50E9488358823B9F00E94A34049
:1082D000AB01BC014093E1085093E2086093E308CE
:1082E0007093E40883ED98E00E9486388091C00086
:1082F00085FFFCCF8AE08093C60084E50E94883524
:108300008823B9F00E94A340AB01BC014093E5086B
:108310005093E6086093E7087093E80885EB98E0CF
:108320000E9486388091C00085FFFCCF8AE0809350
:10833000C6000895AF92BF92CF92DF92EF92FF9264
:108340000F931F93CF93DF9309EFA02E06E0B02E7B
:10835000C1EBD6E000E010E0F801EB5DFC4F80815E
:108360000E948835882309F10E94A3406B017C019B
:10837000F801EC53F94F8081882349F480919508E6
:10838000882329F420E030E040E050E004C0288158
:1083900039814A815B81C701B6010E94A7D2F501EC
:1083A000608371838283938309C088819981AA81C4
:1083B000BB81F50180839183A283B3830F5F1F4F3D
:1083C00084E090E0A80EB91E24960430110521F631
:1083D00086E40E9488358823A1F00E94A3407B0197
:1083E0008C0120E030E040E050E00E948ED518166D
:1083F00044F4E0927102F0927202009373021093BF
:108400007402DF91CF911F910F91FF90EF90DF9059
:10841000CF90BF90AF9008951F93DF93CF93CDB7C8
:10842000DEB728970FB6F894DEBF0FBECDBF182F6A
:10843000809132028823D9F10E949A41FE0131963F
:1084400088E0DF011D928A95E9F789E40E9488356A
:10845000882329F460E070E080E090E002C00E9490
:10846000A34069837A838B839C838AE40E94883546
:10847000882329F460E070E080E090E002C00E9470
:10848000A3406D837E838F83988789EF96E0BE013A
:108490006F5F7F4F412F0E94B13A0E9458D0609386
:1084A000DD067093DE068093DF069093E006289643
:1084B0000FB6F894DEBF0FBECDBFCF91DF911F91F5
:1084C0000895CF93DF93FC0180818B3309F46CC056
:1084D0008091F3069091F40604970CF065C020910A
:1084E0009E0830919F0880E690E0289FE001299F38
:1084F000D00D389FD00D1124C15FD84FCE01BF01E0
:108500000E94EE18EEE4F5E007C08091C00085FF00
:10851000FCCF9093C600319694919923B1F7E4EE85
:10852000FBE007C08091C00085FFFCCF9093C600A0
:10853000319694919923B1F7FE0107C08091C00054
:1085400085FFFCCF31969093C60090819923B1F7B7
:10855000E2EEFBE007C08091C00085FFFCCF909366
:10856000C600319694919923B1F78091C00085FFA0
:10857000FCCF8AE08093C60080919E0890919F086E
:10858000019664E070E00E9465D790939F08809305
:108590009E088091F3069091F40601969093F4065C
:1085A0008093F30681E001C080E0DF91CF910895D0
:1085B000EF92FF920F931F93DF93CF93CDB7DEB768
:1085C0006E970FB6F894DEBF0FBECDBF6091DB068D
:1085D0007091DC066115710511F480E037C08E01E1
:1085E0000F5F1F4FC8014DE150E00E947D181E8EA5
:1085F000EE24FF24C801FC01EE0DFF1D10811123A4
:1086000031F01A3021F00894E11CF11CF4CFCE01B6
:108610000196FC01EE0DFF1D10820E94614288232D
:10862000A1F0112371F00894E11CF11C8091DB068C
:108630009091DC068E0D9F1D9093DC068093DB06E7
:1086400004C01092DC061092DB0681E06E960FB635
:10865000F894DEBF0FBECDBFCF91DF911F910F9178
:10866000FF90EF9008954F925F926F927F928F925A
:108670009F92AF92BF92CF92DF92EF92FF920F93B1
:108680001F93DF93CF93CDB7DEB76E970FB6F894F5
:10869000DEBF0FBECDBF0E94D842882309F457C168
:1086A00010C32D3041F080919B0890919C088F352C
:1086B00091050CF4EEC010929D0880919B0890915A
:1086C0009C08009709F4FDC2A0909E08B0909F08F6
:1086D000A69CF001A79CF00DB69CF00D11244FE074
:1086E000842E47E0942E8E0E9F1EE80FF91FE15F47
:1086F000F84F1082F501E55FF84F1082C4016EE477
:1087000070E00E94DA187C01C4016AE270E00E9405
:10871000DA186C01E114F10409F462C0C701019692
:1087200060E070E04AE050E00E9436176093A008D5
:108730007093A1088093A2089093A3082091EB0660
:108740003091EC064091ED065091EE062F5F3F4FC1
:108750004F4F5F4F621773078407950709F4A3C251
:10876000C4016EED7AE00E948C18892B09F09BC23F
:108770008BEA9AE01DC00E278F5FF901E80FF11D0B
:10878000E15FF84FE081EA32B1F7C601019660E09F
:1087900070E04AE050E00E943617202F30E040E0C1
:1087A00050E0621773078407950749F08CE89AE058
:1087B00061E00E944C3585C282E69AE0F9CF809153
:1087C000A0089091A108A091A208B091A30880935D
:1087D000EB069093EC06A093ED06B093EE0606C070
:1087E000009721F088E39AE060E0E3CF80913202C5
:1087F000882349F5C40167E470E00E94DA18009705
:1088000011F1019660E070E04AE050E00E943617F6
:1088100064307105C0F4E2ECF9E007C08091C0005B
:1088200085FFFCCF9093C600319694919923B1F7C0
:108830008091C00085FFFCCF1093C60088EB99E0C3
:1088400060E00E94489BC4016EE771E00E94E51859
:10885000009721F48FEA99E00E94093480919E08E4
:1088600090919F08019664E070E00E9465D7909314
:108870009F0880939E088091F3069091F4060196DC
:108880009093F4068093F30610929C0810929B0834
:1088900064C02C35B9F580911E0490911F0420917D
:1088A000200430912104821B930B8F779070892BC9
:1088B00009F453C08091F3069091F40604970CF0EC
:1088C0004CC082E294E00E94F02E80939A0840917E
:1088D0009B0850919C0820919E0830919F08269DEE
:1088E000F001279DF00D369DF00D1124E40FF51FCA
:1088F000E15FF84F80834F5F5F4F50939C08409338
:108900009B082BC02B3311F450929D0880919D0839
:10891000882319F520919B0830919C0880919E082E
:1089200090919F08869DF001879DF00D969DF00D1A
:108930001124E20FF31FE15FF84F80919A088083C2
:108940002F5F3F4F30939C0820939B0806C030E672
:10895000632E712C1AE0552453944091F3065091E4
:10896000F40644305105CCF480911E0490911F040C
:108970002091200430912104821B930B8F779070FB
:10898000892B59F082E294E00E94F02E282F8093E8
:108990009A088A3009F085CE8ECE809125048823EE
:1089A00009F48FC180919B0890919C08892B09F054
:1089B00088C1452B09F02DC11092A4082AC14D3061
:1089C00099F0433211F04A3321F480919D088823B5
:1089D00059F080919B0890919C088F35910524F463
:1089E0002F5F3F4F09F0F0C02091A6063091A706F7
:1089F0004091A8065091A90680919E0690919F06ED
:108A0000A091A006B091A106281739074A075B0775
:108A100008F49CC0ECE9F9E007C08091C00085FF34
:108A2000FCCF9093C600319694919923B1F7809131
:108A3000C00085FFFCCF8092C6000E9458D0609392
:108A4000E5067093E6068093E7069093E80620918A
:108A5000E1063091E2064091E3065091E406621B84
:108A6000730B840B950B28EE33E040E050E00E943E
:108A700078D7F22EE32ED42EC52EEDB7FEB7389759
:108A80000FB6F894FEBF0FBEEDBF0DB71EB70F5F58
:108A90001F4FB282A182F80153824282622F732F4C
:108AA000842F952F20E13EE040E050E00E9478D7EF
:108AB000F801358324836F2D7E2D8D2D9C2D2CE385
:108AC00030E040E050E00E9478D7CA01B9012CE3C1
:108AD00030E040E050E00E9478D7F8017783668369
:108AE0000E941219EEE4F5E08DB79EB708960FB616
:108AF000F8949EBF0FBE8DBF07C08091C00085FF58
:108B0000FCCF9093C600319694919923B1F7F5016B
:108B100007C08091C00085FFFCCF31969093C600BE
:108B200090819923B1F78091C00085FFFCCF80929E
:108B3000C600C50161E00E94689B83E294E00E9448
:108B4000932783E294E061E00E943E2080919A089E
:108B5000833211F49092A40820919B0830919C08D4
:108B60002115310519F410929D08ABC080919E0823
:108B700090919F08869DF001879DF00D969DF00DC8
:108B80001124E20FF31FE15FF84F1082FC01E55F53
:108B9000F84F90822091F3063091F4062F5F3F4FFB
:108BA0003093F4062093F306019664E070E00E948F
:108BB00065D790939F0880939E0810929D0810920D
:108BC0009C0810929B0834C04B3311F490929D087E
:108BD00080919D08882361F520919B0830919C0825
:108BE00080919E0890919F08869DF001879DF00DD1
:108BF000969DF00D1124E20FF31FE15FF84F809175
:108C00009A0880832F5F3F4F30939C0820939B08E6
:108C10000FC020E6622E712C992493949AE0892E3D
:108C20005E010894A11CB11C88E8482E89E0582EEA
:108C30002091A6063091A7064091A8065091A9065A
:108C400080919E0690919F06A091A006B091A106EA
:108C5000281739074A075B07A0F58091F306909122
:108C6000F406049774F58091A408882351F5809147
:108C7000F9059091FA05A091FB05B091FC05809350
:108C8000A6069093A706A093A806B093A90681EF25
:108C900095E00E94446F9C01482F80939A088A3087
:108CA00009F08DCEA1CEC114D10409F485CD00E028
:108CB00080E0A69C9001A79C300DB69C300D11243D
:108CC0005CCD6E960FB6F894DEBF0FBECDBFCF91D0
:108CD000DF911F910F91FF90EF90DF90CF90BF90A9
:108CE000AF909F908F907F906F905F904F9008957E
:108CF000DF92EF92FF920F931F93D82E8091F3068D
:108D00009091F406039714F40E9433430E9458D0C4
:108D10007B018C012091F5063091F6064091F70613
:108D20005091F8062115310541055105A9F08091B2
:108D3000DD069091DE06A091DF06B091E006280FD7
:108D4000391F4A1F5B1F2E153F054007510720F4AE
:108D500086E096E00E94093420916D0230916E0207
:108D600040916F0250917002211531054105510566
:108D700019F18091DD069091DE06A091DF06B09199
:108D8000E006280F391F4A1F5B1F2E153F054007BD
:108D9000510790F4DD2081F49091DA0D8091DB0D84
:108DA000981751F45E9A1092C1065E9A1092C2060C
:108DB0005E9A1092C3065E9A0E941D591F910F91F0
:108DC000FF90EF90DF9008950E94498980E00E9413
:108DD00078460E9468980895EF92FF920F931F9330
:108DE00080E50E948835882321F4EE24FF24870142
:108DF00007C00E949740AC01CB01DA017C018D01D4
:108E000083E50E948835882361F00E94A34020E01A
:108E100030E04AE754E40E9460D60E94F4D37B011C
:108E20008C010E949E7A0E9458D06093DD06709358
:108E3000DE068093DF069093E006E60EF71E081F1D
:108E4000191F0E94CA90882341F483E596E060E0F0
:108E50000E94489B02C00E94E4460E9458D06E15B2
:108E60007F0580079107B8F31F910F91FF90EF9056
:108E70000895DF92EF92FF920F931F93CF93DF93AA
:108E8000C0919108D091920880E50E94883588238E
:108E900029F4EE24FF248701DD240FC00E946E3EDA
:108EA0007C010027F7FC0095102FDD24E114F1046C
:108EB0000105110511F0DD24D39483E50E94883566
:108EC000882399F00E94A34020E030E04AE754E470
:108ED0000E9460D60E94F4D37B018C0180E0E114F3
:108EE000F1040105110509F081E0DD2051F488232A
:108EF00041F48881882329F0CE0161E00E94689BBB
:108F000005C08CEB96E060E00E94489B81E00E94E7
:108F1000A5900E949E7A0E9458D06093DD067093BF
:108F2000DE068093DF069093E006E114F10401056C
:108F3000110591F0E60EF71E081F191F0E9458D068
:108F40006E157F0580079107F8F40E94D49088235E
:108F5000D9F40E94E446F2CF0E94D290882319F4FB
:108F600017C00E94E4460E94D4908823D1F38091D8
:108F70002504882319F08DEA96E002C08BE996E07B
:108F800060E00E94489B04C080E00E94A590EFCF63
:108F9000DF91CF911F910F91FF90EF90DF90089597
:108FA0007F928F929F92AF92BF92CF92DF92EF9279
:108FB000FF920F931F93CF93DF938DE690E00E9473
:108FC0007B3E882309F0CFC187E497E060E00E94F0
:108FD000489B83E50E94883580936802882329F4A2
:108FE00082E50E948835882391F00E94A340E0909A
:108FF000EA06FF248701000F111F055A1F4E0E9429
:10900000EFD3F80171836083C7010E94D78586E49E
:109010000E94883580930909882351F00E94A3405B
:1090200060937E0270937F0280938002909381020E
:1090300083E50E948835882351F00E94A340609305
:109040007A0270937B0280937C0290937D0282E48B
:109050000E948835882351F00E94A34060937602D5
:109060007093770280937802909379020E9458D08F
:109070004B015C012091EA06C22FD0E01092E90674
:10908000CC0FDD1FFE01E55AFF4E608171818827FC
:1090900077FD8095982F0E9422D4CC0FDD1FC359F5
:1090A000DF4E288139814A815B810E948ED5181656
:1090B0001CF481E08093E9061092DA06CC24CA946D
:1090C000DC2C76012AE0722E10C18091C00085FF51
:1090D000FCCF9093C600319694919923B1F7E0911B
:1090E000EA06F0E0EE0FFF1FEE0FFF1FE359FF4E01
:1090F000408151816281738182E294E021E030E01D
:109100000E94D930E0E4F7E007C08091C00085FFFD
:10911000FCCF9093C600319694919923B1F760915A
:10912000EA0682E294E070E04AE050E00E940630F5
:10913000ECE3F7E007C08091C00085FFFCCF90937F
:10914000C600319694919923B1F7F7FE03C0EAE384
:10915000F7E028C00E9458D0A7019601205F384D43
:109160004F4F5F4F261B370B480B590BCA01B901F4
:1091700028EE33E040E050E00E9478D782E294E0AD
:10918000BA01A9012AE030E00E94B22F8091C0000C
:1091900085FFFCCF0EC08091C00085FFFCCF90936F
:1091A000C600319694919923B1F78091C00085FF54
:1091B000FCCF7092C6000E9458D04B015C010E9407
:1091C000E446FFEFCF16FFEFDF06FFEFEF06FFEFFE
:1091D000FF0609F052C08091E906E091EA06882373
:1091E00031F1F0E08F01000F111F000F111F035923
:1091F0001F4EEE0FFF1FE55AFF4E608171818827D9
:1092000077FD8095982F0E9422D420E030E040E83E
:109210005FE30E94A6D29B01AC01F80160817181DD
:10922000828193810E948ED587FF58C05EC0F0E096
:109230008F01000F111F000F111F03591F4EEE0F5A
:10924000FF1FE55AFF4E60817181882777FD809569
:10925000982F0E9422D420E030E040E85FE30E9493
:10926000A7D29B01AC01F801608171818281938159
:109270000E9480D3181694F538C0F7FC36C0E091F0
:10928000EA06F0E08F01000F111F000F111F0359B4
:109290001F4EEE0FFF1FE55AFF4E60817181882738
:1092A00077FD8095982F0E9422D49B01AC01F80194
:1092B00060817181828193810E94A6D20E94EFD346
:1092C00097FF07C090958095709561957F4F8F4F60
:1092D0009F4F64307105810591053CF00E9458D084
:1092E000AC01CB01DA016C017D018091DA068823A3
:1092F00019F5FFEFCF16FFEFDF06FFEFEF06FFEFE9
:10930000FF0649F0F7FC18C00E9458D06C197D097F
:109310006051774288F40E9458D0A50194012851E9
:109320003C4F4F4F5F4F261737074807590708F044
:1093300046CFE4E4F7E0D0CE8CE297E060E00E9414
:10934000489B0E9458D06093DD067093DE068093A0
:10935000DF069093E0066093E1067093E206809347
:10936000E3069093E406DF91CF911F910F91FF9058
:10937000EF90DF90CF90BF90AF909F908F907F90B5
:1093800008959F92AF92BF92CF92DF92EF92FF9299
:109390000F931F9387E697E060E00E94489B83E568
:1093A0000E94883580936802882329F482E50E9410
:1093B0008835882341F00E94A3400E94EFD3709328
:1093C0006410609363100E9458D07B018C0110924E
:1093D000DA061092E9066091631070916410882794
:1093E00077FD8095982F0E9422D420917F10309194
:1093F000801040918110509182100E948ED51816D5
:109400000CF070C081E08093E9066CC00E9458D0D7
:109410005B016C01D801C70188519C4FAF4FBF4F12
:109420008A159B05AC05BD0508F059C0E091D7062B
:10943000F0E0EE0FFF1FEE0FFF1FE359FF4E4081DC
:10944000518162817381E4E6F7E007C08091C0003A
:1094500085FFFCCF9093C600319694919923B1F784
:1094600082E294E022E030E00E94D930E0E6F7E0CA
:1094700007C08091C00085FFFCCF9093C600319655
:1094800094919923B1F76091D70682E294E070E05D
:109490004AE050E00E940630ECE5F7E007C080911A
:1094A000C00085FFFCCF9093C6003196949199231C
:1094B000B1F740917F1050918010609181107091B0
:1094C000821082E294E021E030E00E94D930809165
:1094D000C00085FFFCCF9092C600860175010E94F6
:1094E000E44602C06AE0962E8091E9068823E1F006
:1094F0008091DA068823C1F4609163107091641042
:10950000882777FD8095982F0E9422D420917F1084
:109510003091801040918110509182100E948ED520
:1095200018160CF473CF1BC0609163107091641017
:10953000882777FD8095982F0E9422D420917F1054
:109540003091801040918110509182100E9480D300
:1095500088232CF480916802882309F457CF82E590
:1095600097E060E00E94489B0E9458D06093DD061F
:109570007093DE068093DF069093E0061F910F91B3
:10958000FF90EF90DF90CF90BF90AF909F900895A5
:109590004F925F926F927F928F929F92AF92BF9203
:1095A000CF92DF92EF92FF920F931F93CF93DF93AF
:1095B0008091090790910A0720E630E0829FA00180
:1095C000839F500D929F500D1124415F584F50932F
:1095D000900840938F088091330280FF26C0EEE40C
:1095E000F5E007C08091C00085FFFCCF9093C600D6
:1095F000319694919923B1F7FA0107C08091C00088
:1096000085FFFCCF31969093C60090819923B1F7E6
:109610008091C00085FFFCCF8AE08093C60005C022
:109620003196F0939008E0938F08E0918F08F091C5
:10963000900880818032A1F38E34F9F481818033E7
:10964000E4F08A3334F019C03196F0939008E09337
:109650008F08E0918F08F091900880818032A1F707
:1096600005C03196F0939008E0938F08E0918F0841
:10967000F091900880818032A1F380918F089091C1
:1096800090086AE270E00E94DA18FC01009709F085
:109690001082E0918F08F0919008108181818053B1
:1096A0008A3008F0C2C701C03196F0939208E09367
:1096B0009108E0919108F091920880818032A1F7A1
:1096C00005C03196F0939208E0939108E0919108DB
:1096D000F091920880818032A1F380918F0890915F
:1096E000900890939408809393080E946E3E1D34D6
:1096F00009F446C0143509F415C7173409F095C7A5
:109700008430910569F18530910534F497FD81C766
:10971000823091059CF01CC08A35910539F18B355A
:10972000910524F44C9709F074C71DC08B35910541
:1097300001F18C35910509F06CC71FC08091320290
:10974000882309F466C70E949A410E94B43461C715
:1097500020E0029709F421E0822F0E940C4259C7B1
:109760000E94EC4656C70E94E53653C710929508F2
:1097700050C781E0809395084CC70E94CB4049C7F1
:109780008037910509F46EC2813791050CF080C0D5
:109790008F31910509F4F9C180329105CCF58631FC
:1097A000910509F422C187319105BCF481319105FD
:1097B00009F410C18231910524F4029708F029C7F9
:1097C00006C18431910509F408C1853191050CF079
:1097D00007C1429709F01DC78BC28A31910509F470
:1097E00028C18B31910544F48831910509F40DC1EC
:1097F00049970CF019C1FEC08C31910509F43DC1A7
:109800008C3191050CF434C14E9709F002C740C168
:109810008535910509F4B7C286359105C4F48135C3
:10982000910509F45BC28235910544F480329105BB
:1098300009F441C18A9709F0ECC6AAC183359105A4
:1098400009F452C2843591050CF052C24AC28A36DC
:10985000910509F422C28B3691056CF48836910586
:1098600009F4D4C1893691050CF00EC28C359105EE
:1098700009F0CFC6A1C28D36910509F408C28F3612
:10988000910509F4E3C18B36910509F0C2C621C2E6
:109890008E3C910509F414C48F3C91050CF045C031
:1098A0008C38910509F4E1C18D389105ECF48537C8
:1098B000910509F40DC3863791054CF48237910563
:1098C00009F40EC38337910509F0A3C67DC088371C
:1098D000910509F408C38937910509F408C387374E
:1098E000910509F096C607C3893C910509F453C355
:1098F0008A3C91056CF48E3B910509F4CBC1883C00
:10990000910509F4FEC28139910509F082C6F6C2BB
:109910008C3C910509F473C38D3C91050CF072C326
:109920008B3C910509F075C652C321E0803992073E
:1099300009F4B9C5E1E081399E07FCF4823E910546
:1099400009F411C4833E91054CF48C3D910509F452
:10995000CFC38D3D910509F05CC6D9C3F1E08E32CD
:109960009F0709F448C521E08F32920709F458C5D2
:109970008D52914009F04DC645C4F1E0863F9F07E6
:1099800009F4A0C521E0873F92077CF4E1E08C3A1E
:109990009E0709F48EC5F1E0853F9F0709F48CC549
:1099A0008A59914009F035C681C5E3E0803A9E07A7
:1099B00009F4E2C0F3E0873E9F0709F49BC5875F87
:1099C000914009F026C681C5E4E8F7E07DC20E9417
:1099D00039471FC60E94FF331CC60E948D3719C627
:1099E00083E294E00E946B1F14C683E294E00E941D
:1099F000B31B0FC6609191087091920883E294E0C6
:109A000041E021E00E94362404C683E294E00E94F3
:109A1000B71B0E9458D06093E1067093E2068093D2
:109A2000E3069093E406F5C583E294E00E94BE1B32
:109A3000F0C580912604882309F4EBC583E50E94D4
:109A40008835882309F4E5C50E946E3EAC0166277F
:109A500057FD6095762F4093A6065093A706609316
:109A6000A8067093A90681EF95E00E94896BD1C585
:109A700083E294E00E94781DCCC5609191087091BA
:109A8000920883E294E040E021E00E943624C1C5C0
:109A900080912604882309F4BCC583E294E060E049
:109AA0000E94E91C609191087091920883E294E011
:109AB0000E94C81DAEC580912504882311F00E9424
:109AC0009E7AC0919108D0919208CE0161E270E037
:109AD0000E94DA18009711F0EC01219680E50E94AF
:109AE0008835882311F410E009C010E080919308B4
:109AF000909194088C179D0708F411E0809126043A
:109B0000882309F486C521E0212783E294E0BE0181
:109B100041E00E94362483E50E9488358823D1F0F5
:109B200080919308909194088C179D0798F40E9457
:109B30006E3EAC01662757FD6095762F4093A606D2
:109B40005093A7066093A8067093A90681EF95E04D
:109B50000E94896B83E294E00E94B71B112309F0F5
:109B600058C50E9458D06093E1067093E206809336
:109B7000E3069093E4064DC56091910870919208B8
:109B800083E294E00E94142844C50E94BA3741C57C
:109B900083E50E948835882309F43BC50E946E3E08
:109BA0008C0180E50E948835882351F017FD08C09C
:109BB0000F3F110509F024F40E946E3EEC0102C033
:109BC000CBE1D0E0EFE2F3E0808191818C179D073B
:109BD00009F41FC5329683E0E536F807A9F7C430CB
:109BE000D10529F41093D9060093D80602C0D7FDF9
:109BF00010C58C2F61E00E9485D18C2F602F0E94B0
:109C000002D28C2FB8010E9407D103C588E690E0EC
:109C10000E947B3E882309F0FCC483E50E948835BE
:109C2000882309F4F6C40E94A340E090EA06FF24CA
:109C30008701000F111F055A1F4E0E94EFD3F80134
:109C400071836083C7010E94D785E3C483E50E94C6
:109C50008835882311F486E002C00E946E3E80930E
:109C60003302D7C40E944E34D4C483E50E948835A1
:109C7000882309F4CEC40E94A3400E94EFD37093BE
:109C8000641060936310C5C40E94CC3ED1C40E948E
:109C9000D047BFC40E94C149BCC483E50E94883537
:109CA000882381F00E946E3E97FF03C080E090E021
:109CB0000BC00E946E3E8F3F910509F01CF40E947C
:109CC0006E3E02C08FEF90E09093D9068093D80645
:109CD000A0C41092D9061092D8069BC40E94AC383A
:109CE00098C41092C70695C481E08093C70691C4BA
:109CF00083E50E948835882399F00E94A34020E0E4
:109D000030E04AE754E40E9460D60E94F4D36093A6
:109D10006D0270936E0280936F029093700279C40B
:109D200088E50E948835882309F076C489E50E9479
:109D30008835882309F070C48AE50E948835882315
:109D400009F06AC485E40E948835882309F064C458
:109D50000E949E7A5E9A0E94A87A5BC45E9A1092D4
:109D6000C10689E50E948835882319F05E9A109211
:109D7000C2068AE50E948835882309F44AC45E9A9F
:109D80001092C30646C483E50E948835882309F4EF
:109D900040C40E94A34020E030E04AE754E40E941F
:109DA00060D60E94F4D36093F5067093F606809314
:109DB000F7069093F8062DC499EB892E98E0992E1A
:109DC00089EA482E88E0582E09EF602E08E0702EB0
:109DD000C0E0D0E0FE01EB5DFC4F80810E94883541
:109DE000882309F45CC0C33009F052C00E94A3402C
:109DF0005B016C0120E030E040EA51E40E9480D336
:109E000088230CF03FC0F4016081718182819381CD
:109E1000A60195010E9487D37B018C016091F10816
:109E20007091F2088091F3089091F408A8019701CD
:109E30000E9460D66093F1087093F2088093F30853
:109E40009093F408F2016081718182819381A8016D
:109E500097010E9460D6F2016083718382839383AD
:109E6000F30160817181828193810E9420D4A801D5
:109E700097010E9460D60E94F4D3F301608371833E
:109E800082839383F401A082B182C282D38207C00D
:109E90000E94A340F401608371838283938321969F
:109EA00084E090E0880E991E480E591E680E791EB7
:109EB000C430D10509F08ECFACC38091C00085FFBE
:109EC000FCCF9093C600319694919923B1F7A1C32A
:109ED000809191089091920860E00E94689B99C3DC
:109EE0000E94C53896C381E00E94947992C380E0B5
:109EF0000E9494798EC30E946D318BC30E94DF3F14
:109F000088C388EC90E00E947B3E882309F081C3DF
:109F100084E40E948835882309F47BC30E94A3400F
:109F20006B017C0110E020E030E040E050E00E9456
:109F300080D3811111E01093CA06112349F1E091F9
:109F4000EA06F0E0EE0FFF1FEE0FFF1FE85BFD4F8C
:109F5000C082D182E282F38260914802709149020C
:109F600080914A0290914B0220E030E040E050E0C6
:109F70000E9480D3882361F480E090E0A0E4B0E404
:109F80008093480290934902A0934A02B0934B02F7
:109F90000E9488333EC3C5E2D3E009EC18E0888113
:109FA0000E948835882349F00E94A3400E94F4D380
:109FB000F801608371838283938321960C5F1F4F26
:109FC000F3E0C932DF0759F70E94375522C3C5E2D3
:109FD000D3E009EA18E088810E948835882339F0A7
:109FE0000E94A340F801608371838283938321964A
:109FF0000C5F1F4FF3E0C932DF0769F70AC30E9405
:10A00000214107C383E50E948835882351F00E94CF
:10A01000A3406093D9087093DA088093DB0890938B
:10A02000DC0884E50E948835882351F00E94A34013
:10A030006093F5087093F6088093F7089093F808FA
:10A0400082E40E948835882361F00E94A3400E9428
:10A05000F4D36093A5087093A6088093A708909303
:10A06000A80888E50E948835882351F00E94A34003
:10A070006093E9087093EA088093EB089093EC08EA
:10A080008AE50E948835882351F00E94A34060939E
:10A09000ED087093EE088093EF089093F00885E444
:10A0A0000E948835882309F4B4C20E94A3406093BB
:10A0B000F1087093F2088093F3089093F408A9C212
:10A0C000C5E2D3E00BEC16E088810E948835882336
:10A0D00039F00E94A340F8016083718382839383E7
:10A0E00021960C5F1F4FF3E0C832DF0769F791C27A
:10A0F00083E50E948835882309F48BC20E94A3401F
:10A100000E94EFD3709345026093440282C283E5BC
:10A110000E948835882309F47CC20E94A3400E94D3
:10A12000EFD37B018C0184E50E948835882389F078
:10A130008DED90E00E947B3E882309F06AC2E09199
:10A14000EA06F0E0EE0FFF1FEA5BFD4FF182E082CE
:10A1500060C2E091D706F0E0EE0FFF1FEA5BFD4F13
:10A16000F182E08256C280E50E948835882309F496
:10A1700050C20E94A3400E94EFD38B0183E50E944E
:10A180008835882319F4CFEFDFEF05C00E94A34084
:10A190000E94EFD3EB01CE010196039708F039C27C
:10A1A000EFE2F3E0808191818017910709F431C2D9
:10A1B000329623E0E536F207A9F717FD2AC20E947E
:10A1C0009E7AF02E802F60E00E9485D18FEFCF3FE6
:10A1D000D80729F0219751F0C0E0D0E00CC0802FC3
:10A1E0000E9435D2C0E0D0E0892B29F4C1E0D0E054
:10A1F00002C00E94E4468F2D0E9435D28C179D0725
:10A20000C1F707C285E40E948835882351F00E9477
:10A21000A3400E94EFD3161617061CF4EEE4F5E0F7
:10A22000D2C080E50E948835882351F00E94A34067
:10A2300060938702709388028093890290938A02C8
:10A2400089E40E948835882361F00E94A3400E941F
:10A25000AB8460938B0270938C0280938D029093F9
:10A260008E0284E40E948835882361F00E94A34016
:10A270000E94B98460938F02709390028093910240
:10A280009093920283E40E948835882351F00E94C3
:10A29000A3406093930270939402809395029093ED
:10A2A00096020E940F82E3E8F1E007C08091C000AF
:10A2B00085FFFCCF31969093C60090819923B1F72A
:10A2C000E6E8F1E007C08091C00085FFFCCF319641
:10A2D0009093C60090819923B1F7409187025091E5
:10A2E00088026091890270918A0282E294E022E001
:10A2F00030E00E94D930EAE8F1E007C08091C00068
:10A3000085FFFCCF31969093C60090819923B1F7D9
:10A3100060918B0270918C0280918D0290918E02DF
:10A320000E94B284AB01BC0182E294E022E030E002
:10A330000E94D930EEE8F1E007C08091C00085FFAF
:10A34000FCCF31969093C60090819923B1F760912C
:10A350008F027091900280919102909192020E94DE
:10A36000C084AB01BC0182E294E022E030E00E94B4
:10A37000D930E2E9F1E007C08091C00085FFFCCF51
:10A3800031969093C60090819923B1F74091930242
:10A3900050919402609195027091960282E294E04D
:10A3A00022E030E00E94D9308091C00085FFFCCFD0
:10A3B0008AE08093C6002DC18091C00085FFFCCF4C
:10A3C0009093C600319694919923B1F7E6E9F1E0B4
:10A3D00007C08091C00085FFFCCF31969093C600E6
:10A3E00090819923B1F78091C00085FFFCCF8AE06E
:10A3F0008093C6000EC183E50E948835882329F426
:10A4000060E070E080E090E002C00E94A3406093B2
:10A41000690270936A0280936B0290936C02F9C098
:10A4200085E40E948835882319F4C0E0D0E003C099
:10A430000E946E3EEC0183E40E948835882319F463
:10A4400005E010E003C00E946E3E8C0183E50E948F
:10A450008835882319F00E94A3400BC0D7FD05C0A2
:10A4600060E070E086E193E404C060E070E08CE8B6
:10A4700092E4AE0198010E942F8B8091EB0690919F
:10A48000EC06A091ED06B091EE060196A11DB11D5E
:10A490008093EB069093EC06A093ED06B093EE0646
:10A4A0000E941F35B6C00E949E7AB3C00E94767A81
:10A4B000B0C00E94A539ADC00E94C42C80E00E94AB
:10A4C000E928A7C00E94C42CA4C083E50E94883557
:10A4D000882361F00E94A34020E030E040E050E09B
:10A4E0000E9480D3882311F481E001C080E00E94A3
:10A4F000E9288FC081E0809332020E94CF90809142
:10A50000EF069091F006A091F106B091F2068093CB
:10A51000EB069093EC06A093ED06B093EE060E9436
:10A520001F3577C0682F882379F1EEE4F5E007C086
:10A530008091C00085FFFCCF9093C6003196949126
:10A540009923B1F78091C00085FFFCCF84E580930B
:10A55000C60082E294E040E050E00E94BF2FE6E9AE
:10A56000F1E007C08091C00085FFFCCF3196909349
:10A57000C60090819923B1F78091C00085FFFCCF80
:10A580008AE08093C60045C01092EA0686E40E94E5
:10A5900088358823A1F00E94A3407B018C0120E034
:10A5A00030E040E050E00E948ED5181644F4E0926E
:10A5B0007102F09272020093730210937402EEE43F
:10A5C000F5E007C08091C00085FFFCCF9093C600E6
:10A5D000319694919923B1F7E7EAF1E007C08091B1
:10A5E000C00085FFFCCF31969093C60090819923DF
:10A5F000B1F76091D70682E294E070E04AE050E063
:10A600000E9406308091C00085FFFCCF8AE08093D5
:10A61000C6000E9453340CC00E949E7A88E50E94B6
:10A620008835882309F09ACB9CCB0E943431F1CF36
:10A63000DF91CF911F910F91FF90EF90DF90CF901E
:10A64000BF90AF909F908F907F906F905F904F9052
:10A650000895CF93DF938091F3069091F4060397CA
:10A6600014F40E94334383E294E060E00E943E20B1
:10A670008091F3069091F406892B09F468C08091CB
:10A680002304882309F44BC02091090730910A075D
:10A6900080E690E0289FE001299FD00D389FD00DE3
:10A6A0001124C15FD84FCE0168EF7AE00E948C1868
:10A6B000892BB9F083E294E060E00E94E91CE6EEA9
:10A6C000FAE007C08091C00085FFFCCF9093C600E0
:10A6D000319694919923B1F78091C00085FFFCCF0A
:10A6E0001AC083E294E0BE010E94021D80912404FE
:10A6F0008823A9F4E3EEFAE007C08091C00085FF4B
:10A70000FCCF9093C600319694919923B1F7809134
:10A71000C00085FFFCCF8AE08093C60002C00E9483
:10A72000C84A8091F3069091F40601979093F4063D
:10A730008093F3068091090790910A07019664E0DF
:10A7400070E00E9465D790930A07809309070E94E2
:10A750007D810E94E446DF91CF9108959093DC06BD
:10A760008093DB060E94D842089582E294E040E0A4
:10A7700052EC61E070E00E94B82EECEDFBE007C007
:10A780008091C00085FFFCCF9093C60031969491D4
:10A790009923B1F78091C00085FFFCCF8AE08093B8
:10A7A000C600EEE4F5E007C08091C00085FFFCCF55
:10A7B0009093C600319694919923B1F784B7282FCE
:10A7C00080FF14C0E4EDFBE007C08091C00085FF6E
:10A7D000FCCF9093C600319694919923B1F7809164
:10A7E000C00085FFFCCF8AE08093C60021FF14C023
:10A7F000E4ECFBE007C08091C00085FFFCCF9093A4
:10A80000C600319694919923B1F78091C00085FFDD
:10A81000FCCF8AE08093C60022FF14C0E3EBFBE08C
:10A8200007C08091C00085FFFCCF9093C600319691
:10A8300094919923B1F78091C00085FFFCCF8AE005
:10A840008093C60023FF14C0E3EAFBE007C08091B9
:10A85000C00085FFFCCF9093C60031969491992358
:10A86000B1F78091C00085FFFCCF8AE08093C600DD
:10A8700025FF14C0E3E9FBE007C08091C00085FF1D
:10A88000FCCF9093C600319694919923B1F78091B3
:10A89000C00085FFFCCF8AE08093C60014BEECE8C0
:10A8A000FBE007C08091C00085FFFCCF9093C600FD
:10A8B000319694919923B1F7E1E8FBE007C08091CC
:10A8C000C00085FFFCCF9093C600319694919923E8
:10A8D000B1F78091C00085FFFCCF8AE08093C6006D
:10A8E000EEE4F5E007C08091C00085FFFCCF9093B7
:10A8F000C600319694919923B1F7E1E7FBE007C0D8
:10A900008091C00085FFFCCF9093C6003196949152
:10A910009923B1F7ECE5FBE007C08091C00085FF0B
:10A92000FCCF9093C600319694919923B1F7E0E55E
:10A93000FBE007C08091C00085FFFCCF9093C6006C
:10A94000319694919923B1F7E9E3FBE007C0809138
:10A95000C00085FFFCCF9093C60031969491992357
:10A96000B1F78091C00085FFFCCF8AE08093C600DC
:10A97000EEE2FBE007C08091C00085FFFCCF909322
:10A98000C600319694919923B1F7E2E2FBE007C04B
:10A990008091C00085FFFCCF9093C60031969491C2
:10A9A0009923B1F78091C00085FFFCCF8AE08093A6
:10A9B000C600EEE4F5E007C08091C00085FFFCCF43
:10A9C0009093C600319694919923B1F7E3E1FBE0AF
:10A9D00007C08091C00085FFFCCF9093C6003196E0
:10A9E00094919923B1F70E94A774BC0182E294E08C
:10A9F0004AE050E00E940630ECEFFAE007C0809198
:10AA0000C00085FFFCCF9093C600319694919923A6
:10AA1000B1F782E294E060ED74E04AE050E00E9419
:10AA200006308091C00085FFFCCF8AE08093C6008D
:10AA300010920B0710920C0710920D0710920E0740
:10AA40000E94C42C80E00E94E9280E942E9780E199
:10AA500097E220E931E0F9013197F1F70197D9F751
:10AA60000E947B8A0E9443590E94C57908950F93E2
:10AA70001F93CF93DF93C0E0D0E08E010750174FB4
:10AA8000FE01E753F74F60817181828193810E94BB
:10AA900020D4FE01E754F74F208131814281538158
:10AAA0000E9460D60E94F4D3F80160837183828390
:10AAB00093832496C031D10501F7DF91CF911F9187
:10AAC0000F910895FC0160817181828193812091B1
:10AAD000C5083091C6084091C7085091C8080E9427
:10AAE00060D60E9430D66093E80D7093E90D809394
:10AAF000EA0D9093EB0D88EE9DE00E94537A089545
:10AB00002F923F924F925F926F927F928F929F927D
:10AB1000AF92BF92CF92DF92EF92FF920F931F936B
:10AB2000DF93CF93CDB7DEB762970FB6F894DEBF51
:10AB30000FBECDBFFC018B017A013A8B298B60815E
:10AB40007181828193812091B9083091BA08409136
:10AB5000BB085091BC080E9460D60E9430D61B01F1
:10AB60002C012092DC0D3092DD0D4092DE0D5092D2
:10AB7000DF0DF80160817181828193812091BD0890
:10AB80003091BE084091BF085091C0080E9460D625
:10AB90000E9430D63B014C016092E00D7092E10DB5
:10ABA0008092E20D9092E30DF701608171818281C4
:10ABB00093812091C1083091C2084091C3085091FF
:10ABC000C4080E9460D60E9430D65B016C01A0923E
:10ABD000E40DB092E50DC092E60DD092E70DE98943
:10ABE000FA8960817181828193812091C5083091B9
:10ABF000C6084091C7085091C8080E9460D60E94BC
:10AC000030D67B018C01E092E80DF092E90D0093C3
:10AC1000EA0D1093EB0DC201B1010E9422D40E94F3
:10AC2000EFD369837A838B839C83C401B3010E9431
:10AC300022D40E94EFD36D837E838F839887C601D1
:10AC4000B5010E9422D40E94EFD369877A878B874F
:10AC50009C87C801B7010E9422D40E94EFD36D8760
:10AC60007E878F87988BCE010196BE016B5F7F4FE9
:10AC7000AE01475F5F4F9E01235F3F4F0E94197AED
:10AC800080E090E0A0E0B0E08093F00D9093F10DB3
:10AC9000A093F20DB093F30D8093F40D9093F50D06
:10ACA000A093F60DB093F70D8093F80D9093F90DE6
:10ACB000A093FA0DB093FB0D8093FC0D9093FD0DC6
:10ACC000A093FE0DB093FF0D8093000E9093010EA4
:10ACD000A093020EB093030E62960FB6F894DEBFF7
:10ACE0000FBECDBFCF91DF911F910F91FF90EF90DD
:10ACF000DF90CF90BF90AF909F908F907F906F909C
:10AD00005F904F903F902F9008958F929F92AF92B7
:10AD1000BF92CF92DF92EF92FF920F931F93CF9348
:10AD2000DF93EC016B01009709F45CC08FA98823C5
:10AD300009F058C0EEA0FFA008A519A5FB01B6A018
:10AD4000A7A090A481A4C801B7012B2D3A2D492DAD
:10AD5000582D0E9480D388230CF044C0C801B7014D
:10AD6000A80197010E9460D67B018C016AA97BA98A
:10AD70008CA99DA9905820E030E040E050EC0E9462
:10AD800060D62EA53FA548A959A90E9460D69B016F
:10AD9000AC01C801B7010E94A7D20E94CDD67B01A9
:10ADA0008C016B2D7A2D892D982D9701A8010E9479
:10ADB00080D3882324F4EB2CFA2C092D182D6B2D2D
:10ADC0007A2D892D982D9701A8010E9480D3882380
:10ADD00049F0C701D801F60186A397A3A0A7B1A7A0
:10ADE00081E086ABDF91CF911F910F91FF90EF90A3
:10ADF000DF90CF90BF90AF909F908F900895CF92AB
:10AE0000DF92FF920F93DF93CF9300D0CDB7DEB7E1
:10AE10000091DB0DCC24DD2420E030E08DE4F82E21
:10AE200012C00F9DC0011124865F964F9A838983BB
:10AE3000C901B60149815A810E9485560F5F0F7082
:10AE40009601C980DA808091DA0D081751F7C9019F
:10AE5000B60140E050E00E9485560F900F90CF91D0
:10AE6000DF910F91FF90DF90CF900895AF92BF9246
:10AE7000CF92DF92EF92FF920F931F93CF93DF93C6
:10AE8000EB018A016115710509F466C04115510590
:10AE900009F462C0DAA4CBA4BCA4ADA46EA17FA1C6
:10AEA00088A599A52D2D3C2D4B2D5A2D0E9480D380
:10AEB000882309F451C08FA9882309F043C0F80101
:10AEC000E6A0F7A000A511A56D2D7C2D8B2D9A2D48
:10AED000A80197010E948ED51816A4F5C801B701E4
:10AEE000A80197010E9460D67B018C016AA97BA909
:10AEF0008CA99DA9905820E030E040E050EC0E94E1
:10AF000060D62EA53FA548A959A90E9460D69B01ED
:10AF1000AC01C801B7010E94A7D20E94CDD67B0127
:10AF20008C016D2D7C2D8B2D9A2D9701A8010E94EF
:10AF300080D3882324F4ED2CFC2C0B2D1A2DC70173
:10AF4000D80104C08D2D9C2DAB2DBA2D8EA39FA3AF
:10AF5000A8A7B9A781E08EABDF91CF911F910F9188
:10AF6000FF90EF90DF90CF90BF90AF900895CF9279
:10AF7000DF92EF92FF920F93DF93CF9300D0CDB784
:10AF8000DEB78091DA0D8FB7F894F090DB0D8FBFAC
:10AF90008091DA0D90E040968F1991098F70907032
:10AFA0000497E4F00091DA0D03500F70CC24DD24F7
:10AFB00040E050E09DE4E92E0FC001500F700E9D5F
:10AFC000C0011124865F964F9A838983B6010E943F
:10AFD0003657A601C980DA800F1579F70F900F90C8
:10AFE000CF91DF910F91FF90EF90DF90CF90089578
:10AFF0003F924F925F926F927F928F929F92AF9209
:10B00000BF92CF92DF92EF92FF920F931F93CF9355
:10B01000DF9380910909882309F4FDC040907A02EA
:10B0200050907B0260907C0270907D0260915B107A
:10B0300070915C10882777FD8095982F0E9422D40C
:10B0400020E030E040E050E40E94A7D2A30192014A
:10B050000E9480D387FDDFC03090DB0D0F2EF0E023
:10B060008F2EF0E09F2EF0E0AF2EF0E0BF2EF02DFF
:10B07000CDE4D0E058C0232D30E02C9FF0012D9F6F
:10B08000F00D3C9FF00D1124E65FF64F8081918119
:10B09000A281B3810097A105B10581F484819581D6
:10B0A000A681B7810097A105B10541F480859185FE
:10B0B000A285B3850097A105B10591F12C9F600190
:10B0C0002D9FD00C3C9FD00C11248AE099E0C80E33
:10B0D000D91EF60164857585868597850E9422D4E0
:10B0E0007B018C01F60160897189828993890E94B4
:10B0F00020D49B01AC01C801B7010E9487D3F6019F
:10B1000022A133A144A155A10E9460D67B018C01EC
:10B11000A50194010E948ED5181614F44701580118
:10B120003394FFE03F228091DA0D381609F0A3CF67
:10B13000C501B40120917E0230917F0240918002CE
:10B14000509181020E9460D69B01AC01C301B20103
:10B150000E94A7D27B018C01A30192010E9480D39F
:10B1600088231CF48301720118C0D0907602C0902D
:10B170007702B0907802A0907902C801B7012D2D16
:10B180003C2D4B2D5A2D0E948ED5181634F48D2D42
:10B190009C2DAB2DBA2D7C018D01A090040EB0909A
:10B1A000050EC090060ED090070EC601B501A8018D
:10B1B00097010E948ED51816D4F4C801B70120E07B
:10B1C00037ED43EA5CE30E9460D67B018C01C60147
:10B1D000B50128E431EE4AE75FE30E9460D69B01A7
:10B1E000AC01C801B7010E94A7D27B018C01E0929B
:10B1F000040EF092050E0093060E1093070EC80180
:10B20000B7010E94EFD370935C1060935B1080E0F5
:10B2100090E00E94D785DF91CF911F910F91FF9011
:10B22000EF90DF90CF90BF90AF909F908F907F90E6
:10B230006F905F904F903F9008956091D8069091E5
:10B24000DA0D8091DB0D9817B9F04091DB0D242FBA
:10B2500030E08DE490E0289FF001299FF00D389FA9
:10B26000F00D1124EE5AF64F608102C04F5F4F700F
:10B270008091DA0D4817D1F784E070E00E9407D181
:10B280000E94F85708951092DB0D8091DB0D80939A
:10B29000DA0D80E1ECEDFDE0DF011D928A95E9F722
:10B2A00080E090E0A0E0B0E08093F40D9093F50D85
:10B2B000A093F60DB093F70D8093F80D9093F90DD0
:10B2C000A093FA0DB093FB0D8093FC0D9093FD0DB0
:10B2D000A093FE0DB093FF0D8093000E9093010E8E
:10B2E000A093020EB093030E8093F00D9093F10D96
:10B2F000A093F20DB093F30D08952F923F924F92C9
:10B300005F926F927F928F929F92AF92BF92CF92F5
:10B31000DF92EF92FF920F931F93DF93CF93CDB7FE
:10B32000DEB766970FB6F894DEBF0FBECDBF9E8B1B
:10B330008D8B6A017B0148015901DC01D8966D9122
:10B340007D918D919C91DB970E9420D4698B7A8BA3
:10B350008B8B9C8BA70196010E9460D60E946DD3B7
:10B360000E94F4D36D837E838F83988769897A895D
:10B370008B899C89A50194010E9460D60E946DD39F
:10B380000E94F4D369837A838B839C832D813E81D1
:10B390004F815885283731054105510540F448E76C
:10B3A00050E060E070E04D835E836F837887698151
:10B3B0007A818B819C81683771058105910540F404
:10B3C00088E790E0A0E0B0E089839A83AB83BC83F8
:10B3D000AD89BE89AC5BBF4FAD90BD90CD90DC9088
:10B3E0001397A454B040BE8BAD8B6D817E818F814D
:10B3F00098850E9420D46D877E878F87988BC601A1
:10B40000B5010E9422D41B012C0120E030E040E075
:10B4100050E00E9480D3882329F4E0E070E080E0CF
:10B4200060E028C069897A898B899C899B01AC017D
:10B430000E9460D67B018C016D857E858F85988901
:10B440009B01AC010E9460D69B01AC01C801B70111
:10B450000E94A6D27B018C01C201B101A20191011F
:10B460000E94A7D29B01AC01C801B7010E9487D3FB
:10B47000E62F692F2E2F372F482F562FB901CA01DB
:10B480000E946DD30E94EFD33B014C0169817A8108
:10B490008B819C810E9420D469877A878B879C87C7
:10B4A00066277727CB016A197B098C099D090E94C1
:10B4B00022D45B016C0120E030E040E050E00E94CB
:10B4C00080D3882329F4E0E070E080E060E028C0C9
:10B4D00069857A858B859C859B01AC010E9460D62D
:10B4E0007B018C0169897A898B899C899B01AC01DC
:10B4F0000E9460D69B01AC01C801B7010E94A6D290
:10B500007B018C01C601B501A60195010E94A7D25D
:10B510009B01AC01C801B7010E9487D3E62F692FB8
:10B520002E2F372F482F562FB901CA010E945DD404
:10B53000ED89FE89A088B188C288D388860175010B
:10B54000E618F708080919090E94EFD3A801970126
:10B55000261B370B480B590B57FF72C0C201B101B4
:10B5600020E030E040E050E00E9480D3882329F4BE
:10B57000E0E070E080E060E044C0C201B101A201FF
:10B5800091010E94A7D27B018C01C601B5010E94E6
:10B5900020D49B01AC01C801B7010E9460D67B0199
:10B5A0008C016D857E858F8598899B01AC010E94F9
:10B5B00060D69B01AC01C801B7010E94A6D27B01F5
:10B5C0008C0169857A858B859C859B01AC010E94E5
:10B5D00060D69B01AC01C801B7010E94A7D27B01D4
:10B5E0008C01C201B10120E030E040E850E40E944B
:10B5F00060D69B01AC01C801B7010E9487D3E62F3A
:10B60000692F2E2F372F482F562FB901CA010E94BC
:10B610006DD30E94EFD3AC01CB01DA013C014D01A7
:10B6200097FE03C06624772443016A147B048C04CC
:10B630009D0410F03501460120E030E040E050E08C
:10B640009FB7F8946D897E89645B7F4FDB018C9195
:10B65000AC54B040BE8BAD8B882321F5FD01648ACC
:10B66000758A868A978A260D371D481D591D58965A
:10B670002D933D934D935C935B972D813E814F813C
:10B680005885DC962D933D934D935C93DF97A05C9A
:10B69000BF4F29813A814B815C812D933D934D931E
:10B6A0005C9313979FBF66960FB6F894DEBF0FBEEC
:10B6B000CDBFCF91DF911F910F91FF90EF90DF9061
:10B6C000CF90BF90AF909F908F907F906F905F9042
:10B6D0004F903F902F9008954F925F927F928F925C
:10B6E0009F92AF92BF92CF92DF92EF92FF920F9311
:10B6F0001F93CF93DF937090DB0DC0E0D0E02DE47B
:10B70000422E512C44C02097B1F18EA9882361F4B8
:10B71000849CF001859CF00D949CF00D1124E65F53
:10B72000F64F86A9882339F1EAA0FBA00CA11DA140
:10B730006EA17FA188A599A5A80197010E9487D332
:10B740005B016C01849CF001859CF00D949CF00DD4
:10B750001124E65FF64F66A177A180A591A5A80107
:10B7600097010E9487D38B019C01CE01B601A501F0
:10B770000E947D591EAA849CE001859CD00D949C5A
:10B78000D00D1124C65FD64F73948FE07822872C9A
:10B79000992487FC90948091DA0D90E088169906A0
:10B7A00009F0B1CF2097F1F0EAA0FBA00CA11DA1F8
:10B7B0006EA17FA188A599A5A80197010E9487D3B2
:10B7C0005B016C016DEC7CEC8CE49DE3A8019701BE
:10B7D0000E9487D38B019C01CE01B601A5010E9476
:10B7E0007D591EAADF91CF911F910F91FF90EF908D
:10B7F000DF90CF90BF90AF909F908F907F905F90A1
:10B800004F9008950E94B7570E94FF560E946C5BAC
:10B8100008952F923F924F925F926F927F928F92F4
:10B820009F92AF92BF92CF92DF92EF92FF920F93CF
:10B830001F93DF93CF93CDB7DEB7C25AD0400FB678
:10B84000F894DEBF0FBECDBF5C014B013A01290168
:10B85000C156DF4FE882CF59D040C056DF4FF88243
:10B86000C05AD040CF55DF4F0883C15AD040CE5583
:10B87000DF4F1883C25AD040C557DF4FD982C882E4
:10B88000CB58D0408091DA0D8F5F8F70282F3327EF
:10B8900027FD3095E1963FAF2EAFE19702C00E94A1
:10B8A000E4468091DB0D90E0E1964EAD5FADE1970F
:10B8B00084179507A1F3D5016D917D918D919C9190
:10B8C0002091B9083091BA084091BB085091BC084A
:10B8D0000E9460D60E9430D6C357DF4F6883CD5890
:10B8E000D040C257DF4F7883CE58D040C157DF4F8A
:10B8F0008883CF58D040C057DF4F9883C059D0407D
:10B90000F40160817181828193812091BD08309121
:10B91000BE084091BF085091C0080E9460D60E94A6
:10B9200030D6CF56DF4F6883C159D040CE56DF4F57
:10B930007883C259D040CD56DF4F8883C359D04059
:10B94000CC56DF4F9883C459D040D3016D917D917F
:10B950008D919C912091C1083091C2084091C308FB
:10B960005091C4080E9460D60E9430D6CB56DF4F5B
:10B970006883C559D040CA56DF4F7883C659D04036
:10B98000C956DF4F8883C759D040C856DF4F9883C8
:10B99000C859D040A090C508B090C608C090C7084C
:10B9A000D090C808C601B501F201208131814281E1
:10B9B00053810E9460D60E9430D6C756DF4F6883FD
:10B9C000C959D040C656DF4F7883CA59D040C556B2
:10B9D000DF4F8883CB59D040C456DF4F9883CC5972
:10B9E000D0408091DC0D9091DD0DA091DE0DB091E5
:10B9F000DF0DC357DF4F288139814A815B81CD58E4
:10BA0000D040281B390B4A0B5B0BCA01B9010E94BD
:10BA100022D4AF966CAF7DAF8EAF9FAFAF978091C2
:10BA2000E00D9091E10DA091E20DB091E30DCF56A4
:10BA3000DF4F288139814A815B81C159D040281B61
:10BA4000390B4A0B5B0BCA01B9010E9422D4AB9699
:10BA50006CAF7DAF8EAF9FAFAB978091E40D9091AF
:10BA6000E50DA091E60DB091E70DCB56DF4F288193
:10BA700039814A815B81C559D040281B390B4A0B5B
:10BA80005B0BCA01B9010E9422D4A7966CAF7DAFAF
:10BA90008EAF9FAFA7978091E80D9091E90DA0918F
:10BAA000EA0DB091EB0DC756DF4F288139814A81ED
:10BAB0005B81C959D040281B390B4A0B5B0BCA016B
:10BAC000B9010E9422D4A3966CAF7DAF8EAF9FAF19
:10BAD000A39720E030E040E050E00E9480D388232C
:10BAE00009F4BBC0C557DF4FA881B981CB58D040FE
:10BAF000EC91F0E0EE0FFF1FEE0FFF1FE359FF4E3A
:10BB000060817181828193812091690230916A0202
:10BB100040916B0250916C020E9480D388230CF0FC
:10BB20003BC0C756DF4F288139814A815B81C959A3
:10BB3000D0402093E80D3093E90D4093EA0D5093E7
:10BB4000EB0DEEE4F5E007C08091C00085FFFCCF6F
:10BB50009093C600319694919923B1F7EFE0FCE001
:10BB600007C08091C00085FFFCCF9093C60031963E
:10BB700094919923B1F78091C00085FFFCCF8AE0B2
:10BB80008093C60040E050E060E070E0A3964CAFC8
:10BB90005DAF6EAF7FAFA397A3966CAD7DAD8EAD5D
:10BBA0009FADA3970E94EFD397FF07C09095809514
:10BBB000709561957F4F8F4F9F4F0E9422D47B01DC
:10BBC0008C01C601B50120E030EC4DE254E40E9446
:10BBD00060D69B01AC01C801B7010E948ED5181632
:10BBE0000CF03BC0C756DF4F688179818A819B8109
:10BBF000C959D0406093E80D7093E90D8093EA0D28
:10BC00009093EB0DEEE4F5E007C08091C00085FF56
:10BC1000FCCF9093C600319694919923B1F7E1EF50
:10BC2000FBE007C08091C00085FFFCCF9093C60069
:10BC3000319694919923B1F78091C00085FFFCCF94
:10BC40008AE08093C60080E090E0A0E0B0E0A39698
:10BC50008CAF9DAFAEAFBFAFA3978091DA0DA82F89
:10BC6000B0E0C757DF4FB983A883C958D0408DE4EF
:10BC700090E0A89F8001A99F100DB89F100D11247E
:10BC8000065F164F045B1F4FF80110820C541040E2
:10BC9000AF966CAD7DAD8EAD9FADAF97AB962CAD35
:10BCA0003DAD4EAD5FADAB970E94A7D2CB57DF4FF6
:10BCB000688379838A839B83C558D0400E94EFD3E1
:10BCC0009B01AC01D8016D937D938D939C93139749
:10BCD00097FF0CC088279927DC01821B930BA40BCC
:10BCE000B50BF80180839183A283B383AF966CADCB
:10BCF0007DAD8EAD9FADAF97AB962CAD3DAD4EAD4E
:10BD00005FADAB970E94A6D2CF57DF4F6883798390
:10BD10008A839B83C158D0408DE490E0C757DF4FA2
:10BD200028813981C958D040289F8001299F100D52
:10BD3000389F100D1124065F164FCF57DF4F6881D3
:10BD400079818A819B81C158D0400E94EFD39B01A9
:10BD5000AC01D80114966D937D938D939C931797A6
:10BD600097FF0CC088279927DC01821B930BA40B3B
:10BD7000B50BF80184839583A683B7838DE490E0A7
:10BD8000C757DF4F28813981C958D040289F80018B
:10BD9000299F100D389F100D1124065F164FA7968E
:10BDA0006CAD7DAD8EAD9FADA7970E94EFD39B018B
:10BDB000AC01D80118966D937D938D939C931B973E
:10BDC00097FF0CC088279927DC01821B930BA40BDB
:10BDD000B50BF80180879187A287B387A3966CADD6
:10BDE0007DAD8EAD9FADA3970E94EFD39B01AC01BB
:10BDF00097FF07C050954095309521953F4F4F4F85
:10BE00005F4F8DE490E0C757DF4F68817981C95853
:10BE1000D040689F8001699F100D789F100D1124FC
:10BE2000065F164F6CE0E62EF12CE00EF11ED801F5
:10BE30001C962D933D934D935C931F97CA01B901B6
:10BE40000E9422D4C557DF4FA881B981CB58D0407A
:10BE5000EC91F0E0EE0FFF1FEE0FFF1FE45BFD4FD4
:10BE600020813181428153810E9460D60E94EFD3AC
:10BE7000F8016487758786879787C557DF4FA88144
:10BE8000B981CB58D040EC91F0E0EE0FFF1FEA5B98
:10BE9000FD4F20813181442737FD4095542F0E946A
:10BEA00032D724E630E040E050E00E949AD7F80113
:10BEB0002487D70111963C93119712964C931297B1
:10BEC00013965C936080718082809380A480B5809B
:10BED000C680D780E084F18402851385C901DA0128
:10BEE0008E159F05A007B10714F4D801C7018A1564
:10BEF0009B05AC05BD0514F4D601C5019C01AD013F
:10BF000086159705A805B90514F4A40193018DE4DD
:10BF100090E0C757DF4F68817981C958D040689F4A
:10BF2000F001699FF00D789FF00D1124E65FF64F48
:10BF3000208B318B428B538B2630310541055105C7
:10BF400010F40C946968E85BFF4F8091D8069091DB
:10BF5000D906AA2797FDA095BA2F80839183A28343
:10BF6000B383AF966CAD7DAD8EAD9FADAF9720E046
:10BF700030E040E050E00E9480D3182F111F1127BD
:10BF8000111F1295107FAB966CAD7DAD8EAD9FAD40
:10BF9000AB9720E030E040E050E00E9480D388235F
:10BFA0000CF41062CB57DF4F688179818A819B81C5
:10BFB000C558D04020E030E040E050E00E9480D3FF
:10BFC00088230CF41160CF57DF4F688179818A8113
:10BFD0009B81C158D04020E030E040E050E00E941A
:10BFE00080D388230CF41260A7966CAD7DAD8EAD26
:10BFF0009FADA79720E030E040E050E00E9480D362
:10C0000088230CF41460A3966CAD7DAD8EAD9FAD0E
:10C01000A39720E030E040E050E00E9480D38823E6
:10C020000CF418608DE490E0C757DF4FA881B98108
:10C03000C958D040A89FF001A99FF00DB89FF00DFE
:10C040001124E65FF64F10A3C557DF4FA881B981D1
:10C05000CB58D0408C9181A3208131814281538182
:10C06000C358DF4F288339834A835B83CD57D04041
:10C07000211531054105510541F484819581A68141
:10C08000B7810097A105B10511F05E985E988DE427
:10C0900090E0C757DF4F48815981C958D040489F29
:10C0A000F001499FF00D589FF00D1124E65FF64F07
:10C0B0006084718482849384611471048104910486
:10C0C00009F05E988DE490E0C757DF4F6881798171
:10C0D000C958D040689FF001699FF00D789FF00D1E
:10C0E0001124E65FF64F84859585A685B785009770
:10C0F000A105B10509F4E4C78091EC0D882319F07E
:10C1000081508093EC0DC557DF4FA881B981CB5882
:10C11000D0408C91882321F45E9880E28093EC0DCE
:10C120002090D9083090DA084090DB085090DC0865
:10C13000C156DF4F6881CF59D040C056DF4F78815C
:10C14000C05AD040CF55DF4F8881C15AD040CE551C
:10C15000DF4F9881C25AD040A20191010E9480D342
:10C1600087FD16C0C156DF4F8881CF59D040C056D9
:10C17000DF4F9881C05AD040CF55DF4FA881C15AB8
:10C18000D040CE55DF4FB881C25AD0401C012D019E
:10C19000A090B908B090BA08C090BB08D090BC0875
:10C1A000AF966CAD7DAD8EAD9FADAF97A6019501FD
:10C1B0000E9487D369A37AA38BA39CA3E090BD08B8
:10C1C000F090BE080091BF081091C008AB966CAD0E
:10C1D0007DAD8EAD9FADAB97A80197010E9487D32F
:10C1E0006DA37EA38FA398A7CB57DF4F688179817A
:10C1F0008A819B81C558D040A60195010E9487D3B2
:10C20000698B7A8B8B8B9C8BCF57DF4F68817981C1
:10C210008A819B81C158D040A80197010E9487D391
:10C220006D8B7E8B8F8B988FA7966CAD7DAD8EAD11
:10C230009FADA7972091C1083091C2084091C308D3
:10C240005091C4080E9487D3698F7A8F8B8F9C8FFF
:10C25000C557DF4FE881F981CB58D040C080DD243D
:10C26000A3966CAD7DAD8EAD9FADA3972091C50813
:10C270003091C6084091C7085091C8080E9487D3E2
:10C28000F601EE0FFF1FEE0FFF1FE45BFD4F208155
:10C290003181428153810E9460D67B018C01CC0C9C
:10C2A000DD1C26E432E0C20ED31ED6016D917C91D6
:10C2B000882777FD8095982F0E9422D49B01AC019E
:10C2C000C801B7010E9460D620E030E048EC52E49B
:10C2D0000E9487D39B01AC016D8F7E8F8F8F98A3B7
:10C2E000C358DF4F688179818A819B81CD57D040C7
:10C2F00066307105810591053CF58DE490E0C757E6
:10C30000DF4FA881B981C958D040A89FF001A99FEB
:10C31000F00DB89FF00D1124E65FF64F84819581F2
:10C32000A681B7810697A105B10574F4B6E06B1636
:10C3300071048104910444F4DA01C901BF7786A72E
:10C3400097A7A0ABB1AB39C069A17AA18BA19CA181
:10C350000E9417D73B014C016DA17EA18FA198A52A
:10C360000E9417D77B018C01698D7A8D8B8D9C8DF6
:10C370000E9417D75B016C01C401B301A8019701AA
:10C380000E94A7D2A60195010E94A7D20E94CDD6F5
:10C390002DE430E0C757DF4F48815981C958D0405C
:10C3A000429FF001439FF00D529FF00D1124E65F74
:10C3B000F64F66A777A780AB91AB8DE490E0C757A7
:10C3C000DF4F68817981C958D040689FF001699F2B
:10C3D000F00D789FF00D1124E65FF64FA6A4B7A4E8
:10C3E000C0A8D1A860E070E080E89FE3A6019501B5
:10C3F0000E9487D39B01AC01C201B1010E9460D6AB
:10C400002B013C018091DA0D9091DB0D891B8F701F
:10C41000A82FB0E06F96BFAFAEAF6F97CD01029778
:10C42000069708F046C060E074E284E799E4A3014F
:10C4300092010E9487D30E9430D67B018C016091CB
:10C44000A5087091A6088091A7089091A808E61603
:10C45000F7060807190768F56E197F09800B910B1D
:10C46000660F771F881F991F6F96EEADFFAD6F9710
:10C470009F01442737FD4095542F0E9478D7CA0169
:10C48000B9010E9420D40E9430D69B01AC012E0D30
:10C490003F1D401F511FCA01B9010E9420D49B01BA
:10C4A000AC0160E074E284E799E40E9487D32B0139
:10C4B0003C018DE490E0C757DF4F28813981C9588E
:10C4C000D040289F8001299F100D389F100D112406
:10C4D000065F164FC601B501A30192010E9460D606
:10C4E000D80192966D937D938D939C9395975096DA
:10C4F0006D917D918D919C9153970E9420D4A301C1
:10C5000092010E9460D60E946DD30E94F4D3F8017C
:10C5100060AF71AF82AF93AFC356DF4F1882CD5972
:10C52000D040C256DF4F1882CE59D04050E8252E59
:10C530004FE3342E88249924E1E1F0E0EC0FFD1F55
:10C54000E80DF91DC301B20120813181428153817F
:10C550000E9460D6E1E0F0E0EC0FFD1FE80DF91D50
:10C5600060837183828393835B016C01E894D7F8C5
:10C57000F401E755F74FE080F18002811381C60195
:10C58000B501A80197010E948ED51816CCF4C801F8
:10C59000B701A60195010E9487D36B017C01C356A8
:10C5A000DF4F6881CD59D040C256DF4F7881CE59D8
:10C5B000D040C101A70196010E9480D388236CF46A
:10C5C000C356DF4F8881CD59D040C256DF4F988186
:10C5D000CE59D040D1016C017D0124E030E0820EC3
:10C5E000931E30E18316910471F0D701C601C35642
:10C5F000DF4FC882CD59D040C256DF4F9883CE5905
:10C60000D0401D0199CFC701B60120E030E040E8DD
:10C610005FE30E9480D388230CF04EC08E010F5F31
:10C620001F4F31E1A32EB12CAC0EBD1ED8016D9170
:10C630007D918D919C91A70196010E9460D6F80191
:10C6400061937193819391938F01EA15FB0571F7C3
:10C650008DE490E0C757DF4F28813981C958D04019
:10C66000289F8001299F100D389F100D1124065F0F
:10C67000164FD80192966D917D918D919C919597D1
:10C68000A70196010E9460D6F80162A373A384A358
:10C6900095A360AD71AD82AD93AD0E9420D4A7018A
:10C6A00096010E9460D60E94F4D3D801D8966D936B
:10C6B0007D938D939C93DB978DE490E0C757DF4F7C
:10C6C000E881F981C958D040E89F8001E99F100DA9
:10C6D000F89F100D1124065F164FD80150966D91EA
:10C6E0007D918D919C9153970E9420D4F80126A5AD
:10C6F00037A540A951A90E9487D36D966CAF7DAF35
:10C700008EAF9FAF6D97D8012D913D914D915C916A
:10C71000139769962CAF3DAF4EAF5FAF69971496F4
:10C720002D913D914D915C91179765962CAF3DAF42
:10C730004EAF5FAF659718962D913D914D915C91ED
:10C740001B9761962CAF3DAF4EAF5FAF61971C96C4
:10C750002D913D914D915C911F972D962CAF3DAF42
:10C760004EAF5FAF2D9769962CAD3DAD4EAD5FAD31
:10C770006997211531054105510559F565964CAD6F
:10C780005DAD6EAD7FAD65974115510561057105D4
:10C7900001F561966CAD7DAD8EAD9FAD6197611574
:10C7A000710581059105A9F46D966CAD7DAD8EADD9
:10C7B0009FAD6D972091E1083091E2084091E30828
:10C7C0005091E4080E9460D60E946DD30C5B1F4F0D
:10C7D00050C02D962CAD3DAD4EAD5FAD2D972115C2
:10C7E00031054105510511F56D966CAD7DAD8EADF0
:10C7F0009FAD6D972091E5083091E6084091E708DC
:10C800005091E8080E9460D60E946DD32DE430E07C
:10C81000C757DF4F48815981C958D040429F800196
:10C82000439F100D529F100D112421C06D966CADC9
:10C830007DAD8EAD9FAD6D972091DD083091DE0806
:10C840004091DF085091E0080E9460D60E946DD3AD
:10C850002DE430E0C757DF4FE881F981C958D04057
:10C86000E29F8001E39F100DF29F100D1124025BE7
:10C87000164F0E94F4D3D8016D937D938D939C93B2
:10C8800013978DE490E0C757DF4F28813981C9584D
:10C89000D040289FF001299FF00D389FF00D112402
:10C8A000E65FF64FEC5BFF4FA080B180C280D38083
:10C8B000E454F0402090F9083090FA084090FB08CA
:10C8C0005090FC084091FD085091FE086091FF08CF
:10C8D0007091000929964CAF5DAF6EAF7FAF29977D
:10C8E00060910109709102098091030990910409F6
:10C8F00025966CAF7DAF8EAF9FAF259780910509D0
:10C9000090910609A0910709B091080921968CAF72
:10C910009DAFAEAFBFAF219760897189828993893E
:10C920000E9420D43B014C01C601B5010E9420D4D5
:10C930007B018C0169966CAD7DAD8EAD9FAD699725
:10C940000E9422D49B01AC01C801B7010E9460D6AD
:10C95000A40193010E9487D37B018C01C201B10124
:10C960000E9420D49B01AC01C801B7010E948ED562
:10C97000181614F462015101C601B5010E9420D4B9
:10C980007B018C0165966CAD7DAD8EAD9FAD6597DD
:10C990000E9422D49B01AC01C801B7010E9460D65D
:10C9A000A40193010E9487D37B018C0129966CAD71
:10C9B0007DAD8EAD9FAD29970E9420D49B01AC0127
:10C9C000C801B7010E948ED5181634F42996ACAC74
:10C9D000BDACCEACDFAC2997C601B5010E9420D416
:10C9E0007B018C0161966CAD7DAD8EAD9FAD619785
:10C9F0000E9422D49B01AC01C801B7010E9460D6FD
:10CA0000A40193010E9487D37B018C0125966CAD14
:10CA10007DAD8EAD9FAD25970E9420D49B01AC01CA
:10CA2000C801B7010E948ED5181634F42596ACAC17
:10CA3000BDACCEACDFAC2597C601B5010E9420D4B9
:10CA40007B018C012D966CAD7DAD8EAD9FAD2D978C
:10CA50000E9422D49B01AC01C801B7010E9460D69C
:10CA6000A40193010E9487D37B018C0121966CADB8
:10CA70007DAD8EAD9FAD21970E9420D49B01AC016E
:10CA8000C801B7010E948ED5181634F42196ACACBB
:10CA9000BDACCEACDFAC21978DE490E0C757DF4F43
:10CAA000A881B981C958D040A89F8001A99F100DC5
:10CAB000B89F100D1124065F164F0C5B1F4FF80135
:10CAC000A082B182C282D38204541040C601B50153
:10CAD0000E9420D46B017C016D962CAD3DAD4EAD16
:10CAE0005FAD6D970E9487D3D801D2966D937D93E9
:10CAF0008D939C93D597C701B60120E030E040E8C4
:10CB00005BE40E9460D620E034E244EF59E40E94E6
:10CB100087D30E94EFD3F801648F758F868F978F2C
:10CB20002091E9083091EA084091EB085091EC0817
:10CB3000ED962CAF3DAF4EAF5FAFED97CA01B90197
:10CB400020E030E040E05FE30E9460D62B013C0132
:10CB50004091ED085091EE086091EF087091F00857
:10CB6000E9964CAF5DAF6EAF7FAFE997CB01BA01ED
:10CB700020E030E040E05FE30E9460D67B018C0162
:10CB80006091F1087091F2088091F3089091F40897
:10CB9000E5966CAF7DAF8EAF9FAFE59720E030E0BC
:10CBA00040E05FE30E9460D65B016C0189859A8555
:10CBB000AB85BC8589AF9AAFABAFBCAF2D853E8549
:10CBC0004F8558892DAB3EAB4FAB58AFBC01CD0163
:10CBD0009F77A80197010E948ED5181654F4C301BF
:10CBE000B201A80197010E9480D387FD02C02701EE
:10CBF00038016DA97EA98FA998AD9F77A6019501EF
:10CC00000E948ED5181654F4C301B201A6019501F5
:10CC10000E9480D387FD02C0250136018DE490E09B
:10CC2000C757DF4F48815981C958D040489FF0010C
:10CC3000499FF00D589FF00D1124E65FF64F62A159
:10CC400073A184A195A169A77AA78BA79CA7C3010B
:10CC5000B20129A53AA54BA55CA50E9480D387FD0A
:10CC600004C049A45AA46BA47CA46F968EAD9FAD5A
:10CC70006F9702970CF4F7C02090F00D3090F10DF3
:10CC80008090F20D9090F30DB101C40127E137EBD4
:10CC900041ED58E30E948ED518160CF0E4C069816E
:10CCA0007A818B819C812091F40D3091F50D40911A
:10CCB000F60D5091F70D0E94A6D27B018C016D817B
:10CCC0007E818F8198852091F80D3091F90D4091EA
:10CCD000FA0D5091FB0D0E94A6D25B016C0169AD6B
:10CCE0007AAD8BAD9CAD2091FC0D3091FD0D409146
:10CCF000FE0D5091FF0D0E94A6D29B01AC015F7703
:10CD000029AB3AAB4BAB5CAB6DA97EA98FA998ADB3
:10CD10002091000E3091010E4091020E5091030EB1
:10CD20000E94A6D29B01AC015F772DA73EA74FA71B
:10CD300058ABC801B701A80197010E9460D67B01DA
:10CD40008C01C601B501A60195010E9460D69B0128
:10CD5000AC01C801B7010E94A7D20E94CDD67B01C9
:10CD60008C01ED962CAD3DAD4EAD5FADED970E94C3
:10CD70008ED518165CF00F2EF0E0EF2EF0E0FF2EAF
:10CD8000F0E80F2FFFE31F2FF02D0CC0ED966CADD8
:10CD90007DAD8EAD9FADED97A80197010E9487D321
:10CDA0007B018C0169A97AA98BA99CA9E9962CAD74
:10CDB0003DAD4EAD5FADE9970E948ED51816B4F427
:10CDC000E9966CAD7DAD8EAD9FADE99729A93AA9E5
:10CDD0004BA95CA90E9487D35B016C01C801B70114
:10CDE000A60195010E9480D3882314F4570168019D
:10CDF0006DA57EA58FA598A9E5962CAD3DAD4EAD50
:10CE00005FADE5970E948ED51816B4F4E5966CAD2B
:10CE10007DAD8EAD9FADE5972DA53EA54FA558A93B
:10CE20000E9487D37B018C01C601B501A80197013F
:10CE30000E9480D3882314F48601750169A57AA520
:10CE40008BA59CA5A80197010E9460D67B018C014F
:10CE5000B101C401A80197010E9480D387FD07C0DA
:10CE6000D801C70102C0D301C2011C014D018DE4EC
:10CE700090E0C757DF4F48815981C958D040489F3B
:10CE80008001499F100D589F100D1124065F164F09
:10CE9000C101D401F80182A793A7A4A7B5A762A9ED
:10CEA00073A984A995A9905820E030E040E050ECA7
:10CEB0000E9460D6D8019E962D913D914D915C9136
:10CEC000D1970E9460D62BE037ED43E25BE30E94EE
:10CED000A7D20E94CDD6E62ED72EC82EB92EB101EC
:10CEE000C4012E2D3D2D4C2D5B2D0E9480D387FD3E
:10CEF00004C02E2C3D2C8C2C9B2C8DE490E0C7572D
:10CF0000DF4FE881F981C958D040E89F8001E99F4F
:10CF1000100DF89F100D1124065F164FC101D401AA
:10CF2000F80186A397A3A0A7B1A7FF2462A173A1CC
:10CF300084A195A12E2D3D2D4C2D5B2D0E9480D3DB
:10CF4000181614F0FF24F394D801D796FC928DE4C0
:10CF500090E0C757DF4FE881F981C958D040E89F7A
:10CF60006001E99FD00CF89FD00C11242AE039E031
:10CF7000C20ED31E81E0D601D6968C9389819A8108
:10CF8000AB81BC818093F40D9093F50DA093F60DC9
:10CF9000B093F70D8D819E81AF81B8858093F80D98
:10CFA0009093F90DA093FA0DB093FB0D29AD3AAD16
:10CFB0004BAD5CAD2093FC0D3093FD0D4093FE0D09
:10CFC0005093FF0D4DA95EA96FA978AD4093000E57
:10CFD0005093010E6093020E7093030ED601929649
:10CFE000ED90FD900D911C919597E092F00DF092CF
:10CFF000F10D0093F20D1093F30D96966D917D91C6
:10D000008D919C919997A80197010E9487D34B011C
:10D010005C01C301B201A80197010E9487D38B0173
:10D020009C01C601B501A4010E947D59E096BFADE7
:10D03000E097B093DA0DC357DF4F288139814A81D9
:10D040005B81CD58D0402093DC0D3093DD0D4093B3
:10D05000DE0D5093DF0DCF56DF4F488159816A8135
:10D060007B81C159D0404093E00D5093E10D609316
:10D07000E20D7093E30DCB56DF4F688179818A8191
:10D080009B81C559D0406093E40D7093E50D80936A
:10D09000E60D9093E70DC756DF4F88819981AA81ED
:10D0A000BB81C959D0408093E80D9093E90DA093BE
:10D0B000EA0DB093EB0D0E94025C0E94977909C0C3
:10D0C0002090F5083090F6084090F7085090F80846
:10D0D0002FC8CE55DF4F0FB6F894DEBF0FBECDBFC1
:10D0E000CF91DF911F910F91FF90EF90DF90CF9044
:10D0F000BF90AF909F908F907F906F905F904F9078
:10D100003F902F900895FF920F931F93CF93DF933B
:10D110008B010E9458D0EB01FF24FA9409C00E94B1
:10D1200058D06C1B7D0B6017710710F080E008C0B1
:10D13000FEBC0DB407FEFDCF8EB58F3F81F781E0B9
:10D14000DF91CF911F910F91FF900895FC014281D3
:10D15000242F30E0C9019595879580658CBD40FFEF
:10D1600002C080E004C080E0463009F081E08DBD5F
:10D17000808160E00E9402D20895DF92EF92FF92D8
:10D180000F931F93CF93DF93EC01D62E79018A0181
:10D190000E94A668CE016CE271E00E9483688D2D2A
:10D1A00080648EBD0DB407FEFDCF28E130E0D801CC
:10D1B000C701022E04C0B695A795979587950A9446
:10D1C000D2F78EBD0DB407FEFDCF285030408FEF53
:10D1D000283F380761F7DD2011F485E906C088E0B3
:10D1E000D81611F487E801C08FEF8EBD0DB407FE8D
:10D1F000FDCF8CE0D81631F48FEF8EBD0DB407FE55
:10D20000FDCF8EB59FEF2FEF2EBD0DB407FEFDCFE6
:10D210008EB587FF04C0992311F09150F5CF8B8311
:10D22000DF91CF911F910F91FF90EF90DF900895C4
:10D23000FC01808161E00E9402D20895DC016EBD94
:10D24000FA0120E030E00DB407FEFDCF80818EBDF5
:10D250000DB407FEFDCF81818EBD2E5F3F4F32960C
:10D2600082E02030380779F70DB407FEFDCF8FEF4D
:10D270008EBD0DB407FEFDCF8FEF8EBD0DB407FE42
:10D28000FDCF8FEF8EBD0DB407FEFDCF8EB513968B
:10D290008C9313978F71853011F481E0089583E1A9
:10D2A00011968C931197CD010E94186980E0089522
:10D2B000CF92DF92EF92FF920F931F93CF93DF9362
:10D2C000EC017A018B0169018C81833039F059E0DE
:10D2D000EE0CFF1C001F111F5A95D1F7CE0168E11B
:10D2E000A80197010E94BD68882311F086E023C041
:10D2F000CE016EEFA6010E941E698823E9F0CE01DF
:10D3000068E572E00E948368882311F487E113C006
:10D31000CE016DE020E030E040E050E00E94BD68CA
:10D32000882341F48FEF8EBD0DB407FEFDCF8EB57F
:10D33000882379F086E18983CE010E94186980E014
:10D34000DF91CF911F910F91FF90EF90DF90CF90E1
:10D350000895CE010E94186981E0F2CFBF92CF926A
:10D36000DF92EF92FF920F931F93CF93DF93EC0125
:10D370006B017A010E9458D08B01BB24BA9409C07A
:10D380000E9458D0601B710B6D52714010F081E10A
:10D390000BC0BEBC0DB407FEFDCF8EB58B838F3F97
:10D3A00079F38E3F39F08FE08983CE010E941869AE
:10D3B00080E02FC0D7011197EF28D9F08FEF8EBDF5
:10D3C00020E030E09FEF0BC00DB407FEFDCF8EB51F
:10D3D000F601E20FF31F80839EBD2F5F3F4F2A1798
:10D3E0003B0790F30DB407FEFDCF8EB5AC0DBD1D10
:10D3F0008C938FEF8EBD0DB407FEFDCF8EB58FEFF2
:10D400008EBD0DB407FEFDCF8EB5CE010E9418690A
:10D4100081E0DF91CF911F910F91FF90EF90DF900E
:10D42000CF90BF900895CF92DF92EF92FF920F932B
:10D430001F93CF93DF93EC017A018B0169018C81FB
:10D44000833039F0A9E0EE0CFF1C001F111FAA95D4
:10D45000D1F7CE0161E1A80197010E94BD68882340
:10D4600039F084E08983CE010E94186980E006C00B
:10D47000CE01B60140E052E00E94AE69DF91CF914B
:10D480001F910F91FF90EF90DF90CF900895BF9282
:10D49000CF92DF92EF92FF920F931F93CF93DF9380
:10D4A000EC01B62E1C82198248830E9458D06B0171
:10D4B000888161E00E9485D1CE010E94186986E0D2
:10D4C00060E00E9485D185E061E00E9485D187E01F
:10D4D00061E00E9485D184E061E00E9485D184E012
:10D4E00061E00E9402D285E08A8382E58CBD1DBC8A
:10D4F00080E09FEF9EBD0DB407FEFDCF8F5F8A30A9
:10D50000C9F709C00E9458D06C197D09615D774048
:10D5100010F081E05EC0CE0160E020E030E040E04D
:10D5200050E00E94BD68182F8B83813059F7CE01DF
:10D5300068E02AEA31E040E050E00E94BD6882FFE6
:10D5400002C01C8311C080E02FEF2EBD0DB407FE7A
:10D55000FDCF9EB58F5F8430C1F79B839A3A11F05F
:10D5600082E037C082E08C838C81823021F0EE240F
:10D57000FF2487010FC0E12CF12C012D00E4102FB6
:10D5800009C00E9458D06C197D09615D774010F088
:10D590008AE01FC0CE0167E320E030E040E050E0C9
:10D5A0000E94BD68CE0169E2A80197010E94BD6892
:10D5B0008B83882331F78C81823029F5CE016AE391
:10D5C00020E030E040E050E00E94BD68882331F068
:10D5D00088E08983CE010E94186921C08FEF8EBD3B
:10D5E0000DB407FEFDCF8EB5807C803C11F483E046
:10D5F0008C8380E09FEF9EBD0DB407FEFDCF2EB55E
:10D600008F5F8330C1F7CE010E94186986E08B15C9
:10D6100018F488E1898303C0BA8281E001C080E008
:10D62000DF91CF911F910F91FF90EF90DF90CF90FE
:10D63000BF900895CF93DF93EB01DC0190E020E0F1
:10D640003EE28C91803269F0283029F4FE01E90F26
:10D65000F11D30839F5FFE01E90FF11D8C918083E6
:10D660009F5F2F5F11962B3061F7C90FD11D188274
:10D67000DF91CF9108950F931F93CF93DF93DC0138
:10D68000EB018A0180E090E020E2FE01E80FF91F43
:10D69000208301968B309105C1F757E040E024C00C
:10D6A000622F2E3219F089E29CE007C05A3051F106
:10D6B0005AE048E018C0321729F1FC010196349174
:10D6C0003323C9F75417F0F02132E0F02F37D0F4AC
:10D6D000822F81568A3110F4622F6052FE01E40FCE
:10D6E000F11D60834F5F11962C91222311F02F3290
:10D6F000B9F6F801B183A08390E08881803219F0F7
:10D7000091E001C090E0892FDF91CF911F910F919F
:10D7100008956F927F928F929F92AF92BF92CF9215
:10D72000DF92EF92FF920F931F93CF93DF93EC0161
:10D730007A018B012B81222309F480C089899A897F
:10D74000AB89BC8984179507A607B70708F476C08C
:10D7500085C0E114F1040105110551F41C821D82FC
:10D760001E821F82188619861A861B8681E067C072
:10D77000288539854A855B85E98DFA8D858590E018
:10D780000996215030404040504039014A01082E4E
:10D7900004C096948794779467940A94D2F72F5F85
:10D7A0003F4F4F4F5F4F0894E108F10801091109FD
:10D7B0005701680104C0D694C794B794A7948A957A
:10D7C000D2F70894E11CF11C011D111DA614B70429
:10D7D000C804D90428F0211531054105510549F443
:10D7E0008D899E89AF89B88D8C839D83AE83BF83DD
:10D7F00016C0A618B708C808D90811C04C815D81A9
:10D800006E817F81898D9A8D94010E944277089460
:10D81000A108B108C108D108882331F40FC084E001
:10D82000882E912C8C0E9D1EA114B104C104D1042C
:10D8300029F7E886F9860A871B8798CF80E0DF9171
:10D84000CF911F910F91FF90EF90DF90CF90BF90FD
:10D85000AF909F908F907F906F900895223009F045
:10D8600078CFE7CFCF93DF93EC018C859D85AE8594
:10D87000BF8540E0611141E0BC01CD010E941875F7
:10D88000882319F420E030E00AC08889282F30E08E
:10D8900095E0220F331F9A95E1F7225F314FC901BE
:10D8A000DF91CF9108950F931F93CF93DF938C0156
:10D8B000FC0183818823E1F1818187FF36C0C801A3
:10D8C00061E00E94326CEC01009791F18881853E05
:10D8D00079F1F8018381823040F481899289A389AA
:10D8E000B4898C8F9D8FAE8FBF8FF8018589968903
:10D8F000A789B08D9B8F8A8FCD01AA27BB279D8BCF
:10D900008C8BE091080EF091090E309751F0BE011A
:10D910006A5E7F4FCE0148960995888D998D9B8BC5
:10D920008A8BF80181818F7781830E94DD7404C026
:10D9300081E0F801808380E0DF91CF911F910F910A
:10D9400008950F931F938C010E94536CF80113826A
:10D950001F910F910895FC018381882319F0CF0155
:10D960000E94A16C0895CF93DF93FC01EB018381AA
:10D97000882391F08250823020F48FE288831982CC
:10D9800009C0CF0160E00E94326C009729F0BE010F
:10D990000E941A6B81E001C080E0DF91CF91089571
:10D9A0006F927F928F929F92AF92BF92CF92DF92AF
:10D9B000EF92FF920F931F93DF93CF9300D000D08D
:10D9C000CDB7DEB77C015A016B01DC0113968C9157
:10D9D0001397813009F091C011968C9181FF8DC011
:10D9E000A0C00097A105B10511F481E087C0F7013F
:10D9F0006084718482849384C701B601A5010E946A
:10DA0000896B882309F479C0D70159968D919C912F
:10DA10005A97A114B104C104D10489F455964D91CB
:10DA20005D916D917C9158970E94B877882309F495
:10DA300064C0F701158A168A178A108E44C0D70170
:10DA400014964D915D916D917C9117979E012F5F7A
:10DA50003F4F0E944277882309F44FC0D70159965F
:10DA6000ED91FC915A9749815A816B817C8187891C
:10DA7000803149F4483FBFEF5B07B0E06B07B0E08F
:10DA80007B0748F020C0483F8FEF58078FEF6807AB
:10DA90008FE07807C0F4CF010E94B877882369F13E
:10DAA000D70114964D915D916D917C911797599680
:10DAB0008D919C915A970FEF1FEF2FEF3FE00E943F
:10DAC000BB768823D1F0F701A18AB28AC38AD48AAF
:10DAD000818180688183C7010E94536C882369F02B
:10DAE000B601A5016A147B048C049D0410F4B401F2
:10DAF000A301C7010E94896B01C080E00F900F90C5
:10DB00000F900F90CF91DF911F910F91FF90EF90A9
:10DB1000DF90CF90BF90AF909F908F907F906F904D
:10DB20000895F70181899289A389B489841795079B
:10DB3000A607B70708F055CFE0CFCF93DF93EC01EE
:10DB400040E050E060E070E00E94D06C882369F013
:10DB5000CE0161E00E94326CFC01009731F085EE4D
:10DB600080831B820E94DD7401C080E0DF91CF9131
:10DB700008952F923F924F925F926F927F928F9271
:10DB80009F92AF92BF92CF92DF92EF92FF920F934C
:10DB90001F93CF93DF93EC012A018B81882309F433
:10DBA000B6C0898180FFB3C0C8C025014E185F0888
:10DBB0003B0174E0272E312C2C0E3D1E4201A1C0EA
:10DBC000288539854A855B856FEFA62E61E0B62EE4
:10DBD000A222B3228B8179018A0199E016950795DB
:10DBE000F794E7949A95D1F7E98DFA8D823049F44C
:10DBF000428D538D648D758D4E0D5F1D601F711F9D
:10DC00003FC0D480DA94DE20A114B104D9F4DD2021
:10DC1000C9F4211531054105510549F48D899E89C5
:10DC2000AF89B88D8C839D83AE83BF830BC04C813D
:10DC30005D816E817F81CF0191010E9442778823AF
:10DC400009F465C0E98DFA8D4C815D816E817F811B
:10DC50004250504060407040058404C0440F551F3E
:10DC6000661F771F0A94D2F786859785A089B189A8
:10DC7000480F591F6A1F7B1F4D0D511D611D711DDE
:10DC800080E092E08A199B0984018815990508F4BF
:10DC90008C0182E00030180709F067C080910A0EFD
:10DCA00090910B0EA0910C0EB0910D0E48175907D4
:10DCB0006A077B0709F459C080910E1090910F10EC
:10DCC00093010E94136A882349F421C09501225FC1
:10DCD000314FC301B901A8010E94B318600E711E33
:10DCE000980140E050E088859985AA85BB85820F20
:10DCF000931FA41FB51F88879987AA87BB87801A9F
:10DD0000910A8114910409F05BCFA20102C04FEF88
:10DD10005FEFCA01DF91CF911F910F91FF90EF90BC
:10DD2000DF90CF90BF90AF909F908F907F906F903B
:10DD30005F904F903F902F900895A988BA88CB8824
:10DD4000DC88E884F9840A851B859A0140E050E06C
:10DD5000D601C5018E199F09A00BB10B28173907F1
:10DD60004A075B0708F021CF23CFCB01BA0140E07F
:10DD70000E941875882309F0A9CFC9CFCF92DF92EE
:10DD8000EF92FF920F931F93CF93DF937C01EB01F0
:10DD90008A01FC018381823008F465C08085918509
:10DDA000A285B3858F719070A070B0700097A105A7
:10DDB000B10509F058C063C0F8011082EDE0CE2E25
:10DDC000D12CC701BE0140E250E00E94B96D9C0118
:10DDD0008032910521F0009709F045C046C0488186
:10DDE000442309F442C0453E61F34E3251F301151C
:10DDF0001105A1F18B858F738F3081F58A8D9B8DF5
:10DE0000892B61F5842F90E08F719070009731F12C
:10DE1000833091051CF58C9D90018D9D300D9C9D4E
:10DE2000300D11242D503040D801A20FB31FFE0138
:10DE300090E0953010F4818105C09B3010F484810E
:10DE400001C086818D939F5F32969D3091F78881C6
:10DE500086FF04C0F801E20FF31F15868B8583FD52
:10DE6000B0CF822F03C08FEF01C080E0DF91CF9150
:10DE70001F910F91FF90EF90DF90CF900895411583
:10DE8000510509F099CF9ACFDF93CF930F92CDB779
:10DE9000DEB7BE016F5F7F4F41E050E00E94B96D79
:10DEA000019719F02FEF3FEF03C08981282F30E051
:10DEB000C9010F90CF91DF910895EF92FF920F93D8
:10DEC0001F93CF93DF93EC018B81823038F1E8848C
:10DED000F9840A851B85CE010E94446F97FD1EC000
:10DEE00088859985AA85BB854F96A11DB11D888718
:10DEF0009987AA87BB87A5E016950795F794E794BD
:10DF0000AA95D1F72E2D30E02F703070F5E0220F5A
:10DF1000331FFA95E1F7225F314F02C020E030E075
:10DF2000C901DF91CF911F910F91FF90EF9008955C
:10DF30000F931F93CF93DF93EC018B018B81882389
:10DF400009F040C0FB018789803109F041C082E0BF
:10DF50008B831D8A1E8A1F8A188E808D918DA0E06A
:10DF6000B0E045E0880F991FAA1FBB1F4A95D1F763
:10DF7000898B9A8BAB8BBC8B13C083E08B83F801AE
:10DF8000428D538D648D758D4D8B5E8B6F8B788F2D
:10DF90009E012F5E3F4FC8010E941678882391F0A2
:10DFA0001A8F098F81E089831C821D821E821F8245
:10DFB000188619861A861B861C861D861E861F8655
:10DFC000188A01C080E0DF91CF911F910F910895D1
:10DFD0008032C1F7D2CF1F93CF93DF93EC01142F80
:10DFE000262F30E0F90175E0EE0FFF1F7A95E1F77B
:10DFF000E25FF14F8385817121F0842F827109F0F6
:10E0000069C080910A0E90910B0EA0910C0EB091F8
:10E010000D0E8C879D87AE87BF87688BF90165E001
:10E02000EE0FFF1F6A95E1F7E25FF14F8489958952
:10E03000A0E0B0E0DC01992788278D8B9E8BAF8B09
:10E04000B88F228D338DA90160E070E0482B592BE9
:10E050006A2B7B2B4D8B5E8B6F8B788F838590E04B
:10E0600088719070009751F4848D958DA68DB78D31
:10E07000898B9A8BAB8BBC8B81E00CC0409751F5A0
:10E080009E012F5E3F4F898D9A8D0E9416788823BE
:10E0900009F184E08B83812F8F7089831C821D821C
:10E0A0001E821F82188619861A861B8614FF18C0C6
:10E0B000CE0140E050E060E070E00E94D06C882328
:10E0C00079F40AC049895A896B897C89CE010E94FA
:10E0D000896B02C01B8280E0DF91CF911F91089570
:10E0E00015FDF0CF81E0F8CFCF93DF93EC019C01D9
:10E0F0002C5F3F4F898D9A8D41E050E060E070E0E9
:10E100000E9482788823A1F08D899E89AF89B88D7D
:10E110000097A105B10559F48C819D81AE81BF8125
:10E120008D8B9E8BAF8BB88F89818068898381E0CE
:10E13000DF91CF9108952F923F924F925F927F92FD
:10E140008F929F92AF92BF92CF92DF92EF92FF9207
:10E150000F931F93DF93CF9300D000D000D0CDB7A3
:10E16000DEB76C01162F072F5E834D83DC011396FB
:10E170008C911397813009F06FC111968C9181FFBA
:10E180006BC188C1F6014189528963897489808590
:10E190009185A285B38584179507A607B70731F047
:10E1A000C6010E94896B882309F456C1812F902FE4
:10E1B0009C0119014D805E8013C1D6015996ED91E5
:10E1C000FC915A97DA01C90149E0B695A795979550
:10E1D00087954A95D1F774807A9478228FEF882EAC
:10E1E00081E0982E82229322772009F053C0811477
:10E1F000910409F04FC0D60114964D915D916D9137
:10E200007C911797411551056105710581F455966B
:10E210008D919D910D90BC91A02D0097A105B10508
:10E2200061F1F60184839583A683B78333C0CF0160
:10E230009E012F5F3F4F0E944277882309F40CC153
:10E2400029813A814B815C81D6015996ED91FC91EF
:10E250005A978789803149F4283FBFEF3B07B0E0E8
:10E260004B07B0E05B0778F008C0283FEFEF3E07B0
:10E27000EFEF4E07EFE05E0730F0C6010E947470CA
:10E28000882341F4E9C0D60114962D933D934D9314
:10E290005C93179780E092E08819990952018415E0
:10E2A000950508F45C01D6015996ED91FC915A97B9
:10E2B0001496ED90FD900D911C9117978EEF9FEFA6
:10E2C000AFEFBFEFE80EF91E0A1F1B1F058404C045
:10E2D000EE0CFF1C001F111F0A94D2F7868597854C
:10E2E000A089B189E80EF91E0A1F1B1FE70CF11C5B
:10E2F000011D111D90E0A91692E0B90639F5809133
:10E300000A0E90910B0EA0910C0EB0910D0E8E1571
:10E310009F05A007B10771F4109210108FEF9FEFC7
:10E32000AFEFBFEF80930A0E90930B0EA0930C0EED
:10E33000B0930D0E80910E1090910F10B801A701AF
:10E3400091010E9458698823B9F586C0811491040F
:10E3500019F5D60118962D913D914D915C911B9721
:10E3600051968D919D910D90BC91A02D2817390744
:10E370004A075B0788F00E94DD74882309F46CC0AB
:10E3800081E080931010E0920A0EF0920B0E009341
:10E390000C0E10930D0E08C0C801B70141E00E9499
:10E3A0001875882309F458C09401225F314FC901C0
:10E3B000B101A5010E94B318950140E050E0F601BB
:10E3C00080859185A285B385820F931FA41FB51FF9
:10E3D00080879187A287B3872A0C3B1C4A185B0869
:10E3E000D60118962D913D914D915C911B9741144A
:10E3F000510409F0E2CE51968D919D910D90BC9102
:10E40000A02D82179307A407B50748F4F601218BC6
:10E41000328B438B548B81818068818311C08091C2
:10E42000080E9091090E892B59F08D819E81892BC0
:10E4300039F0D60111968C911197806811968C93C2
:10E44000F601818183FF05C0C6010E94536C8823B9
:10E4500019F04D815E8105C081E0D6018C934FEFAC
:10E460005FEFCA0126960FB6F894DEBF0FBECDBF90
:10E47000CF91DF911F910F91FF90EF90DF90CF90A0
:10E48000BF90AF909F908F907F905F904F903F9004
:10E490002F90089582FD76CE89CEDF92EF92FF9283
:10E4A0000F931F93CF93DF93EC0189899A89AB89EE
:10E4B000BC89805E9F4FAF41B04008F071C0CE0173
:10E4C0000E947470882309F46BC00E94DD74882355
:10E4D00009F466C0E98DFA8DEC80FD800E811F8104
:10E4E0008EEF9FEFAFEFBFEFE80EF91E0A1F1B1F65
:10E4F000058404C0EE0CFF1C001F111F0A94D2F704
:10E5000086859785A089B189E80EF91E0A1F1B1F11
:10E5100081E080931010E0920A0EF0920B0E0093AF
:10E520000C0E10930D0E80E092E0EEE0FEE0DF01B5
:10E530009C011D9221503040E1F7DD24D39411C09D
:10E54000B801A7014D0D511D611D711D80910E1067
:10E5500090910F102EE03EE00E945869882301F14F
:10E56000D394E98DFA8D8481D81650F320E032E0FF
:10E5700040E050E0058404C0220F331F441F551FA4
:10E580000A94D2F789899A89AB89BC89820F931F33
:10E59000A41FB51F898B9A8BAB8BBC8B81E001C00C
:10E5A00080E0DF91CF911F910F91FF90EF90DF906E
:10E5B00008958F929F92AF92BF92CF92DF92EF9287
:10E5C000FF920F931F93CF93DF936C01EB01942E77
:10E5D000852EA22E898D9A8DD6015A969C938E9364
:10E5E0005997CB0140E050E060E070E00E94896BF9
:10E5F000BB2438C0CE010E945D6FFC01009709F476
:10E6000093C055E016950795F794E7945A95D1F77E
:10E610001E2D1F708081882311F0853EC9F4BB2018
:10E6200099F420910A0E30910B0E40910C0E5091EE
:10E630000D0ED6011C962D933D934D935C931F9721
:10E6400050961C93BB24B3948081882359F418C03E
:10E65000892D982DBF014BE050E00E94A61800972D
:10E6600009F470C0E884F9840A851B8589899A8930
:10E67000AB89BC89E816F9060A071B0708F4BACF6C
:10E68000A6FE52C0A1FE50C0BB2051F0F601108979
:10E69000C60161E00E94326CEC01009769F444C04D
:10E6A0008B81823009F440C0CE010E944D728823D4
:10E6B000D9F110E0CEE0DEE080E2DE011D928A9525
:10E6C000E9F7DE01292D382DC901FC018BE001900D
:10E6D0000D928150E1F7E091080EF091090E30970C
:10E6E00039F0BE01625F7F4FCE014096099508C0A8
:10E6F00081E298E2998B888B80E098E09F878E87F3
:10E70000888999899B8B8A8B998F888F8E859F8525
:10E710009F8B8E8B0E94DD74882331F0C601612FA0
:10E720004A2D0E94EB6F01C080E0DF91CF911F91D5
:10E730000F91FF90EF90DF90CF90BF90AF909F90A0
:10E740008F900895A7FEEACFEFCF2F923F924F927E
:10E750005F926F927F928F929F92AF92BF92CF9271
:10E76000DF92EF92FF920F931F93DF93CF93CDB77A
:10E77000DEB7C654D0400FB6F894DEBF0FBECDBF93
:10E780003C016B01DE01AE5BBF4F11965C934E9373
:10E7900025962FAF25971C861F861FA21AA66115E6
:10E7A000710509F480C0FC018381882309F07BC0D6
:10E7B000FA0180818F32F1F08601ECE0EE2EF12C2F
:10E7C000EC0EFD1E72E4A72EB12CAC0EBD1E4E0148
:10E7D0000894811C911C2796FFAEEEAE279767E246
:10E7E000262E312C2C0E3D1E270124C01196B183FC
:10E7F000A08301C0FD01A081B1818C918F32B1F362
:10E80000D60113968C91139782508230A8F28E0114
:10E81000095D1F4F59966D917C915A97C8010E94CE
:10E82000986F882351F63FC0342D252D8701832F03
:10E83000922F7C01F50180819181B401A5010E9494
:10E840003B6B882329F42FC03196D501ED93FC93BF
:10E85000D501ED91FC9180818F32B1F38823C9F00D
:10E86000C701B801A40121E00E94D9728823D9F020
:10E870000C151D0519F0C8010E94A16C2796EEAD7C
:10E88000FFAD2797EE16FF0679F6C101322D292F2D
:10E89000CDCFC301B801A40125962FAD25970E94C5
:10E8A000D972182F01C010E0CE0187960E94AB6C80
:10E8B000CE010C960E94AB6C812FCA5BDF4F0FB666
:10E8C000F894DEBF0FBECDBFCF91DF911F910F91A6
:10E8D000FF90EF90DF90CF90BF90AF909F908F9080
:10E8E0007F906F905F904F903F902F9008950F937F
:10E8F0001F93DF93CF93CDB7DEB76B970FB6F89426
:10E90000DEBF0FBECDBF9C01AB0119821C828E0100
:10E910000F5F1F4FC801B90122E00E94A573882331
:10E9200011F410E004C0C8010E949D6D182FCE01A3
:10E9300001960E94AB6C812F6B960FB6F894DEBFE8
:10E940000FBECDBFCF91DF911F910F910895DF933F
:10E95000CF930F92CDB7DEB780914C1490914D14A8
:10E960009E012F5F3F4F009719F0281B390B02C003
:10E9700022553441C9010F90CF91DF910895DB01F9
:10E980000D900020E9F71197A61BB70B0496AD0177
:10E990000E949B700895DF93CF930F92CDB7DEB79F
:10E9A00069830496BE016F5F7F4F41E050E00E9493
:10E9B0009B700F90CF91DF91089580911010882364
:10E9C00099F140910A0E50910B0E60910C0E7091CE
:10E9D0000D0E80910E1090910F102EE03EE00E94DF
:10E9E0005869882319F140911110509112106091CB
:10E9F000131070911410411551056105710591F0C6
:10EA000080910E1090910F102EE03EE00E94586908
:10EA1000882361F0109211101092121010921310AE
:10EA2000109214101092101081E0089580E0089563
:10EA3000DF92EF92FF920F931F937B018C01D42EF4
:10EA400080910A0E90910B0EA0910C0EB0910D0EBC
:10EA50008E159F05A007B107C1F00E94DD748823C1
:10EA6000E1F080910E1090910F10B801A7012EE0F7
:10EA70003EE00E94136A882381F0E0920A0EF09231
:10EA80000B0E00930C0E10930D0EDD2011F481E09F
:10EA900005C081E08093101001C080E01F910F91AC
:10EAA000FF90EF90DF9008958F929F92AF92BF9268
:10EAB000CF92DF92EF92FF920F931F93CF93DF934A
:10EAC0006C01142F70930F1060930E10FC01178AC5
:10EAD00082E090E0A0E0B0E080839183A283B383E2
:10EAE0001092101010921110109212101092131018
:10EAF000109214108FEF9FEFAFEFBFEF80930A0ECD
:10EB000090930B0EA0930C0EB0930D0E442321F4A2
:10EB100088249924540140C0453008F01EC160E0AB
:10EB200070E080E090E040E00E941875882309F4CE
:10EB300014C1C12FD0E02197FE0174E0EE0FFF1F3A
:10EB40007A95E1F7E25FF14FE254FE4F8081EE5B90
:10EB5000F14090E08F779070892B09F0FEC0E6536A
:10EB6000FE4F80819181A281B38184369105A105F8
:10EB7000B10508F4F2C064E0CC0FDD1F6A95E1F73F
:10EB8000CC52D04F88809980AA80BB808114910498
:10EB9000A104B10409F4E1C0C501B40140E00E9440
:10EBA0001875882309F4D9C08091190E90911A0E16
:10EBB0008050924009F0D1C020911E0E222309F40A
:10EBC000CCC080911C0E90911D0E892B09F4C5C0FC
:10EBD00080911B0E882309F4C0C0F601228B80911E
:10EBE0001B0E8483158661E070E007C04F5FF6015D
:10EBF00045874150483008F0B0C0F6014585848112
:10EC000090E09B01042E02C0220F331F0A94E2F70A
:10EC10008217930759F72091240E3091250E211564
:10EC2000310519F040E050E008C02091320E3091DB
:10EC3000330E4091340E5091350EF6012583368304
:10EC400047835087E0901C0EF0901D0E00E010E00E
:10EC5000E80CF91C0A1D1B1DE38AF48A058B168B30
:10EC600080911F0E9091200E918F808F60911E0ECB
:10EC700070E080E090E00E9432D76E0D7F1D801F13
:10EC8000911FF601628F738F848F958F20911F0ED5
:10EC90003091200E55E0220F331F5A95E1F7215095
:10ECA0003E4F232F3327269540E050E0260F371F95
:10ECB000481F591F26873787408B518B8091210E23
:10ECC0009091220E009719F0A0E0B0E008C080916A
:10ECD0002E0E90912F0EA091300EB091310E850125
:10ECE0007401E21AF30A040B150BA8019701280F0F
:10ECF000391F4A1F5B1FF601058404C056954795CE
:10ED0000379527950A94D2F721873287438754870E
:10ED1000253FFFE03F07F0E04F07F0E05F0720F4FA
:10ED20008CE0F601878B19C0255F3F4F4040504073
:10ED300018F480E1F6010EC080913A0E90913B0EDE
:10ED4000A0913C0EB0913D0EF601828F938FA48F5F
:10ED5000B58F80E2878B81E001C080E0DF91CF91A9
:10ED60001F910F91FF90EF90DF90CF90BF90AF90E9
:10ED70009F908F9008956F927F928F929F92AF9203
:10ED8000BF92CF92DF92EF92FF920F931F93CF9398
:10ED9000DF93EC015A016B01380149014230510502
:10EDA0006105710508F45EC089859A85AB85BC85CF
:10EDB0000196A11DB11D84179507A607B70708F492
:10EDC00051C08F89803129F4E52EF62E072F1127A7
:10EDD0000CC0803209F046C07A018B0187E016959D
:10EDE0000795F794E7948A95D1F78B899C89AD892B
:10EDF000BE89E80EF91E0A1F1B1FC801B70141E0BA
:10EE00000E941875882371F18F89803149F4F501CA
:10EE1000F070EE0FFF1FE25FF14F718260820DC054
:10EE2000F501EF77F070EE0FFF1FEE0FFF1FE25FAF
:10EE3000F14F60827182828293828A89823080F06F
:10EE40008D819E81AF81B885E80EF91E0A1F1B1FB8
:10EE5000E0921110F09212100093131010931410FE
:10EE600081E001C080E0DF91CF911F910F91FF9071
:10EE7000EF90DF90CF90BF90AF909F908F907F905A
:10EE80006F900895CF92DF92EF92FF920F931F93AE
:10EE9000CF93DF93EC017A018B01690189859A8513
:10EEA000AB85BC850196A11DB11D84179507A607EA
:10EEB000B70708F453C08F89803129F45527412FB3
:10EEC000302F2F2D0CC0803209F048C09A01AB01C1
:10EED00067E056954795379527956A95D1F78B89C1
:10EEE0009C89AD89BE89280F391F4A1F5B1F8091FD
:10EEF0000A0E90910B0EA0910C0EB0910D0E2817DA
:10EF000039074A075B0739F0CA01B90140E00E949E
:10EF10001875882319F18F89803159F4F701F07041
:10EF2000EE0FFF1FE25FF14F80819181A0E0B0E022
:10EF30000EC0F701EF77F070EE0FFF1FEE0FFF1F0F
:10EF4000E25FF14F80819181A281B381BF70F601B0
:10EF500080839183A283B38381E001C080E0DF914D
:10EF6000CF911F910F91FF90EF90DF90CF90089578
:10EF7000AF92BF92CF92DF92EF92FF920F931F93C7
:10EF8000DF93CF9300D000D0CDB7DEB76C017A010C
:10EF90008B0182E090E0A0E0B0E0F60180839183F5
:10EFA000A283B3835E010894A11CB11CC601B80101
:10EFB000A70195010E944277882341F1C601B8015B
:10EFC000A70100E010E020E030E00E94BB7688233B
:10EFD000E9F0E980FA800B811C81F6018789803194
:10EFE00051F4F8EFEF16FFEFFF06F0E00F07F0E047
:10EFF0001F07E0F209C088EFE8168FEFF8068FEFE1
:10F0000008078FE0180790F281E001C080E00F90C0
:10F010000F900F900F90CF91DF911F910F91FF9064
:10F02000EF90DF90CF90BF90AF9008954F925F9296
:10F030006F927F928F929F92AF92BF92CF92DF9208
:10F04000EF92FF920F931F93DF93CF9300D000D0E6
:10F05000CDB7DEB76C0149835A836B837C8339015A
:10F06000EE24FF2487012E010894411C511C812CA1
:10F07000E2E09E2EA12CB12C49815A816B817C81CA
:10F08000C60192010E944277882339F1D501C4015B
:10F09000F601058404C0880F991FAA1FBB1F0A949C
:10F0A000D2F7E80EF91E0A1F1B1F29813A814B81F6
:10F0B0005C818789803131F4285F3F4F4040504068
:10F0C000D8F205C0285F3F4F4F4F5F40A8F2F301D1
:10F0D000E082F1820283138381E00F900F900F9002
:10F0E0000F90CF91DF911F910F91FF90EF90DF90E4
:10F0F000CF90BF90AF909F908F907F906F905F90D8
:10F100004F9008952F923F924F925F926F927F920D
:10F110008F929F92AF92BF92CF92DF92EF92FF9227
:10F120000F931F93DF93CF93CDB7DEB72F970FB613
:10F13000F894DEBF0FBECDBF1C014A875B876C878A
:10F140007D873F872E87DC0119968D919D910D90CB
:10F15000BC91A02D0196A11DB11D8E839F83A88710
:10F16000B987F901008111812281338101151105CF
:10F170002105310549F0480159010894811C911C71
:10F18000A11CB11C1D8210C0D1018D909D90AD902D
:10F19000BC901D828A859B85AC85BD850197A105A4
:10F1A000B10511F491E09D83750164014424552457
:10F1B00032018E010F5F1F4FF10181859285A3857A
:10F1C000B485481659066A067B0608F090C08E8101
:10F1D0009F81A885B9858C159D05AE05BF0550F4A6
:10F1E000A2E08A2E912CA12CB12CF2E0CF2ED12CB2
:10F1F000E12CF12CC101B701A60198010E944277D0
:10F20000882309F474C089819A81AB81BC81A701EC
:10F2100096012F5F3F4F4F4F5F4F0097A105B105FC
:10F2200019F049015A010DC0281939094A095B0929
:10F230008A859B85AC85BD85281739074A075B07FA
:10F2400059F00894411C511C611C711C0894C11C8C
:10F25000D11CE11CF11CB0CFC101A601B7010FEF19
:10F260001FEF2FEF3FE00E94BB76882399F43FC049
:10F270002601370108944108510861087108C1014D
:10F28000B301A201970186010E94BB76882379F120
:10F29000730162018C149D04AE04BF0448F3AE8573
:10F2A000BF854D915D916D917C9141155105610531
:10F2B000710539F0C101950184010E94BB76882354
:10F2C000B1F0EE85FF8580829182A282B382FD81BA
:10F2D000FF2359F00894811C911CA11CB11CD10181
:10F2E0008D929D92AD92BC92139781E001C080E017
:10F2F0002F960FB6F894DEBF0FBECDBFCF91DF9132
:10F300001F910F91FF90EF90DF90CF90BF90AF9043
:10F310009F908F907F906F905F904F903F902F9035
:10F32000089510924B100895809386020895EFE699
:10F33000F0E0808182608083089580914910982F49
:10F3400080FF03C0459A8FEF02C0459881E080930B
:10F35000820291FF03C0479A8FEF02C0479881E075
:10F360008093830292FF03C02A988FEF02C02A9AEB
:10F3700081E08093840293FF03C028988FEF02C03E
:10F38000289A81E08093850208953D9A3F9A229AB7
:10F39000209A569A5E9A569A5E9A569A5E9A569A0B
:10F3A0005E9A3A98429A3B98439A3C98449A579A64
:10F3B0005F985E9A1092C1063E9A46985E9A1092A5
:10F3C000C206239A2B985E9A1092C306219A299816
:10F3D0005E9AA1E8B0E08C918F7E8C938C918860CE
:10F3E0008C93E0E8F0E080818D7F808380818E7F48
:10F3F000808380818F73808380818F7C80838C91D8
:10F40000887F82608C9380E090E490938900809361
:10F4100088001092850010928400EFE6F0E0808171
:10F420008260808381E08093860278940E949D7937
:10F4300008951F93FC011FB7F89480819181A281E8
:10F44000B3818093231090932410A0932510B09340
:10F450002610FB0180819181A281B38180932710C6
:10F4600090932810A0932910B0932A10FA0180815C
:10F470009181A281B38180932B1090932C10A09343
:10F480002D10B0932E10F90180819181A281B3815A
:10F4900080932F1090933010A0933110B0933210BE
:10F4A0001FBF1F910895FC012FB7F89480819181AF
:10F4B000A281B38180932F1090933010A0933110CC
:10F4C000B09332102FBF0895E82F8FB7F894F0E073
:10F4D000EE0FFF1FEE0FFF1FED5DFF4E208131810C
:10F4E000428153818FBFB901CA01089588E893E131
:10F4F000909334108093331080916F008D7F8093B0
:10F500006F000CC09091DA0D8091DB0D981731F0EF
:10F510008091DB0D8F5F8F708093DB0D9091DA0D02
:10F520008091DB0D981771F710921610109215103C
:10F5300080916F00826080936F00089502C00E94E6
:10F54000E4469091DA0D8091DB0D9817C1F708958C
:10F550000E949E7A0E943B3308951F920F920FB62D
:10F560000F920BB60F921124AF92BF92CF92DF92FF
:10F57000EF92FF920F931F932F933F934F935F93BD
:10F580006F937F938F939F93AF93BF93CF93DF93AB
:10F59000EF93FF938091331090913410892B51F1A8
:10F5A00010921610109215109091DA0D8091DB0DCB
:10F5B000981731F08091DB0D8F5F8F708093DB0D9A
:10F5C0008091331090913410019721F488E59CE0EC
:10F5D0000E94AE5380913310909134100197909314
:10F5E00034108093331088EC90E0909389008093DE
:10F5F000880066C68091151090911610892B09F02D
:10F60000A5C19091DA0D8091DB0D981719F4E0E017
:10F61000F0E014C08091DB0D90E02DE430E0829F9B
:10F62000F001839FF00D929FF00D1124E65FF64FDD
:10F63000E45BFF4F81E08083EC54F040F0931610C0
:10F64000E0931510309709F47BC1E45BFF4F81E034
:10F650008083EC54F04090A180914910981721F0DC
:10F66000909349100E949D7910925310109254105B
:10F670001092551010925610E0911510F09116103E
:10F6800060AD71AD2CE96134720718F060E47CE97B
:10F6900004C03EE46132730730F076956795769545
:10F6A000679584E007C047E26131740730F07695D2
:10F6B000679582E080934C1008C081E080934C10E5
:10F6C0006032710510F460E270E06052704058E002
:10F6D00060307507E8F0472F50E0440F551F440F86
:10F6E000551F4C59534F9A012E5F3F4FF901859199
:10F6F00094919C01AA27639FC001629F810D9A1F6C
:10F7000006948A1F9A1F1124FA01459154911EC034
:10F71000CB01969587958C7F8C599F4EFC01459126
:10F720005491FC01329625913491862F90E0877098
:10F730009070FC012E9FC0012F9F900D3E9F900D59
:10F740001124E3E096958795EA95E1F7481B590B5C
:10F7500044365105A8F4E9EBF1E007C08091C00000
:10F7600085FFFCCF31969093C60090819923B1F725
:10F7700082E294E04AE050E00E94303044E650E0FB
:10F78000509358104093571080914C10992787FD43
:10F79000909590935A1080935910E0911510F09124
:10F7A000161064AD75AD7093521060935110FCE962
:10F7B00061347F0718F060E47CE904C02EE4613214
:10F7C000720730F0769567957695679584E007C067
:10F7D00037E26131730730F07695679582E0809368
:10F7E0004C1008C081E080934C106032710510F419
:10F7F00060E270E06052704048E060307407E8F00A
:10F80000472F50E0440F551F440F551F4C59534F7D
:10F810009A012E5F3F4FF901859194919C01AA278F
:10F82000639FC001629F810D9A1F06948A1F9A1FD1
:10F830001124FA01459154911EC0CB0196958795EC
:10F840008C7F8C599F4EFC0145915491FC0132965E
:10F8500025913491862F90E087709070FC012E9F47
:10F86000C0012F9F900D3E9F900D112403E09695AF
:10F8700087950A95E1F7481B590B44365105A8F4C2
:10F88000E9EBF1E007C08091C00085FFFCCF319625
:10F890009093C60090819923B1F782E294E04AE008
:10F8A00050E00E94303044E650E0CA01A0E0B0E0F1
:10F8B00080934D1090934E10A0934F10B093501022
:10F8C0005093890040938800E0911510F091161034
:10F8D00080899189A289B389B695A79597958795CF
:10F8E000B095A095909581959F4FAF4FBF4F809356
:10F8F000351090933610A0933710B0933810809342
:10F90000391090933A10A0933B10B0933C10809321
:10F910003D1090933E10A0933F10B0934010809301
:10F92000411090934210A0934310B0934410109252
:10F93000451010924610109247101092481006C0C1
:10F9400080ED97E09093890080938800C091151016
:10F95000D0911610209709F4B3C4809186028823B1
:10F9600009F4E3C0488159816A817B818C819D8142
:10F97000AE81BF81481759076A077B0769F48091F8
:10F98000491090E0282F217030E09695879581707E
:10F99000907028173907B1F58091491084FF32C063
:10F9A00086B1869586958095E82FE17080FF2AC004
:10F9B00080914A1080FF26C01416150616061706F9
:10F9C0000CF58091231090912410A0912510B091F6
:10F9D00026108093171090931810A0931910B093CD
:10F9E0001A1080914B10816080934B1088899989FF
:10F9F000AA89BB898093451090934610A093471025
:10FA0000B09348104C815D816E817F81888199819E
:10FA1000AA81BB8184179507A607B70769F480916F
:10FA2000491090E0282F217030E0969587958170DD
:10FA3000907028173907D1F18091491085FF36C0A1
:10FA400086B18695869586958095817081958E275D
:10FA50008270E827E1FF2AC080914A1081FF26C00A
:10FA600014161506160617060CF5809127109091AE
:10FA70002810A0912910B0912A1080931B10909308
:10FA80001C10A0931D10B0931E1080914B1082602B
:10FA900080934B1088899989AA89BB8980934510E6
:10FAA00090934610A0934710B0934810809149104E
:10FAB00082FF39C086B182958F7080958170819563
:10FAC0008E278470E827E2FF2EC080914A1082FFC3
:10FAD0002AC088859985AA85BB85181619061A0635
:10FAE0001B060CF580912B1090912C10A0912D10DD
:10FAF000B0912E1080931F1090932010A09321108E
:10FB0000B093221080914B10846080934B108889B1
:10FB10009989AA89BB898093451090934610A09338
:10FB20004710B0934810E0934A1060E09EC1809166
:10FB3000C00087FF19C04091C600E0911E04F091FB
:10FB40001F0431969F012F773070319780912004E8
:10FB5000909121042817390739F0E256FC4F408371
:10FB600030931F0420931E0488819981AA81BB8150
:10FB70002091351030913610409137105091381047
:10FB8000820F931FA41FB51F8093351090933610DA
:10FB9000A0933710B0933810181619061A061B06D2
:10FBA0000CF45F9A8C819D81AE81BF8120914110C0
:10FBB000309142104091431050914410820F931F96
:10FBC000A41FB51F8093411090934210A09343103F
:10FBD000B0934410181619061A061B060CF4469A20
:10FBE00088859985AA85BB8520913D1030913E106E
:10FBF00040913F1050914010820F931FA41FB51FDA
:10FC000080933D1090933E10A0933F10B09340100E
:10FC1000181619061A061B060CF42B9A8C859D855E
:10FC2000AE85BF852091391030913A1040913B103C
:10FC300050913C10820F931FA41FB51F8093391061
:10FC400090933A10A0933B10B0933C1018161906ED
:10FC50001A061B060CF4299A2091351030913610A3
:10FC600040913710509138101216130614061506DD
:10FC700064F588899989AA89BB89281B390B4A0BA5
:10FC80005B0B209335103093361040933710509310
:10FC9000381020912310309124104091251050915C
:10FCA000261080918202992787FD9095A92FB92F60
:10FCB000820F931FA41FB51F8093231090932410CD
:10FCC000A0932510B09326105F9820914110309199
:10FCD000421040914310509144101216130614061E
:10FCE000150664F588899989AA89BB89281B390B6F
:10FCF0004A0B5B0B2093411030934210409343100A
:10FD000050934410209127103091281040912910D1
:10FD100050912A1080918302992787FD9095A92FF1
:10FD2000B92F820F931FA41FB51F809327109093A4
:10FD30002810A0932910B0932A10469820913D10C6
:10FD400030913E1040913F10509140101216130612
:10FD50001406150664F588899989AA89BB89281B28
:10FD6000390B4A0B5B0B20933D1030933E104093B0
:10FD70003F105093401020912B1030912C10409147
:10FD80002D1050912E1080918402992787FD909517
:10FD9000A92FB92F820F931FA41FB51F80932B107B
:10FDA00090932C10A0932D10B0932E102B9820918F
:10FDB000391030913A1040913B1050913C1012167E
:10FDC00013061406150664F588899989AA89BB89E2
:10FDD000281B390B4A0B5B0B2093391030933A10D8
:10FDE00040933B1050933C1020912F1030913010D5
:10FDF000409131105091321080918502992787FDF2
:10FE00009095A92FB92F820F931FA41FB51F809320
:10FE10002F1090933010A0933110B0933210299886
:10FE20008091451090914610A0914710B0914810D4
:10FE30000196A11DB11D8093451090934610A0938B
:10FE40004710B093481020914510309146104091D2
:10FE500047105091481088899989AA89BB89281729
:10FE600039074A075B0730F46F5F80914C106817C1
:10FE70000CF45DCE20914510309146104091471012
:10FE8000509148108C899D89AE89BF89821793074C
:10FE9000A407B50708F4E8C0E0904D10F0904E10AC
:10FEA00000914F1010915010AC8CBD8CCE8CDF8C1B
:10FEB000A8019701C601B501AA27279FB12D389F38
:10FEC000F001489FF00D479FE00DF11D289FB00DF8
:10FED000E11DFA1F379FB00DE11DFA1F469FB00DBF
:10FEE000E11DFA1F369FB10DEA1FFA1FB695EA1FF2
:10FEF000FA1F929FE00DF11D939FF00D11248CAD20
:10FF00009DAD8E0F9F1F909352108093511028AD7E
:10FF100039AD4AAD5BADA0E0B0E0281739074A071C
:10FF20005B0720F4309352102093511060915110D0
:10FF3000709152108CE96134780718F060E47CE924
:10FF400004C09EE46132790730F076956795769526
:10FF5000679584E007C0E7E261317E0730F076956F
:10FF6000679582E080934C1008C081E080934C102C
:10FF70006032710510F460E270E060527040F8E0A9
:10FF800060307F07E8F0472F50E0440F551F440FC3
:10FF9000551F4C59534F9A012E5F3F4FF9018591E0
:10FFA00094919C01AA27639FC001629F810D9A1FB3
:10FFB00006948A1F9A1F1124FA01459154911EC07C
:10FFC000CB01969587958C7F8C599F4EFC0145916E
:10FFD0005491FC01329625913491862F90E08770E0
:10FFE0009070FC012E9FC0012F9F900D3E9F900DA1
:10FFF0001124B3E096958795BA95E1F7481B590B04
:020000021000EC
:1000000044365105A8F4E9EBF1E007C08091C00047
:1000100085FFFCCF31969093C60090819923B1F76C
:1000200082E294E04AE050E00E94303044E650E042
:1000300050938900409388009A0140E050E08091FD
:100040004D1090914E10A0914F10B0915010820F12
:10005000931FA41FB51F80934D1090934E10A09333
:100060004F10B093501007C12091451030914610A9
:100070004091471050914810888D998DAA8DBB8D65
:1000800082179307A407B50708F0E9C060915310E1
:100090007091541080915510909156102C8D3D8D7B
:1000A0004E8D5F8DAA27639FB12D749FF001849FB1
:1000B000F00D839FE00DF11D649FB00DE11DFA1F4F
:1000C000739FB00DE11DFA1F829FB00DE11DFA1F55
:1000D000729FB10DEA1FFA1FB695EA1FFA1F569FCD
:1000E000E00DF11D579FF00D11248091511090915A
:1000F00052108E179F0738F4C05CDF4F68817981FA
:10010000C054D04003C0BC016E1B7F0BC05CDF4FEE
:10011000288139814A815B81CB01A0E0B0E0821760
:100120009307A407B50708F4B901FCE961347F0718
:1001300018F060E47CE904C02EE46132720730F00C
:10014000769567957695679584E007C037E26131CB
:10015000730730F07695679582E080934C1008C065
:1001600081E080934C106032710510F460E270E021
:100170006052704048E060307407E8F0472F50E06C
:10018000440F551F440F551F4C59534F9A012E5F72
:100190003F4FF901859194919C01AA27639FC0016B
:1001A000629F810D9A1F06948A1F9A1F1124FA01DB
:1001B000459154911EC0CB01969587958C7F8C59A3
:1001C0009F4EFC0145915491FC013296259134914A
:1001D000862F90E087709070FC012E9FC0012F9FAA
:1001E000900D3E9F900D112423E0969587952A95BA
:1001F000E1F7481B590B44365105A8F4E9EBF1E04F
:1002000007C08091C00085FFFCCF31969093C60057
:1002100090819923B1F782E294E04AE050E00E9495
:10022000303044E650E050938900409388009A01B2
:1002300040E050E08091531090915410A0915510DF
:10024000B0915610820F931FA41FB51F80935310B7
:1002500090935410A0935510B09356100CC08091F9
:100260005710909158109093890080938800809146
:10027000591080934C1020914510309146104091B8
:10028000471050914810E0911510F0911610808998
:100290009189A289B389281739074A075B0780F03B
:1002A00010921610109215109091DA0D8091DB0DBE
:1002B000981731F08091DB0D8F5F8F708093DB0D8D
:1002C000FF91EF91DF91CF91BF91AF919F918F916E
:1002D0007F916F915F914F913F912F911F910F915E
:1002E000FF90EF90DF90CF90BF90AF900F900BBE3C
:1002F0000F900FBE0F901F90189580914B10882380
:1003000009F48CC0EEE4F5E007C08091C00085FFE1
:10031000FCCF9093C600319694919923B1F7E0EA0F
:10032000F4E107C08091C00085FFFCCF9093C60028
:10033000319694919923B1F780914B1080FF1FC0A3
:1003400060911710709118108091191090911A10E7
:100350000E9422D42091B9083091BA084091BB087C
:100360005091BC080E9487D3AB01BC018CE994E199
:100370000E9486388CE894E160E00E94489B80915E
:100380004B1081FF1FC060911B1070911C10809159
:100390001D1090911E100E9422D42091BD08309112
:1003A000BE084091BF085091C0080E9487D3AB019E
:1003B000BC0188E894E10E94863888E794E160E017
:1003C0000E94489B80914B1082FF1FC060911F10BC
:1003D0007091201080912110909122100E9422D4BF
:1003E0002091C1083091C2084091C3085091C408BF
:1003F0000E9487D3AB01BC0184E794E10E94863858
:1004000084E694E160E00E94489B8091C00085FFF3
:10041000FCCF8AE08093C60010924B10089560E0F4
:1004200070E08FE793E420918B0230918C02409131
:100430008D0250918E020E9487D36093B410709306
:10044000B5108093B6109093B7100895FC0197FFF4
:1004500003C08091831003C0E657FF4E808190E077
:1004600008952F923F924F925F926F927F928F9258
:100470009F92AF92BF92CF92DF92EF92FF920F9333
:100480001F93DF93CF93CDB7DEB72E970FB6F894B7
:10049000DEBF0FBECDBF1C01FC01EE0FFF1FE55AF2
:1004A000FF4E008111817C01EE0CFF1CEE0CFF1C45
:1004B000970123593F4ED9018D919D910D90BC918B
:1004C000A02D89879A87AB87BC87B801882777FDDD
:1004D0008095982F0E9422D429853A854B855C858A
:1004E0000E94A6D26D837E838F839887F701E452A2
:1004F000FF4E608371838283938320E030E040E28B
:1005000051E40E948ED5181634F4F101E052FF4EEA
:1005100081E080830BC16D817E818F81988520E091
:1005200030E040E251EC0E9480D387FD02C0012BF5
:1005300031F4F101E052FF4E81E0808326C1F101E8
:10054000E052FF4E8081882379F081EE90E1E80E41
:10055000F91E20E030E040E050E0D7012D933D93BC
:100560004D935C93139710826D817E818F81988566
:1005700020918702309188024091890250918A022D
:100580000E9460D669837A838B839C836101CC0C43
:10059000DD1CCC0CDD1CF601EB51FF4E608371833A
:1005A00082839383F601EF51FF4E6D817E818F81AF
:1005B000988520813181428153810E94A7D27B019D
:1005C0008C01F601E055FF4E4080518062807380BF
:1005D000A30192010E9480D387FD13C0E4EBF0E1F8
:1005E000CE0EDF1ED6014D905D906D907C90C801BF
:1005F000B701A30192010E948ED5181614F02701AD
:1006000038016101CC0CDD1CCC0CDD1CF601EF5176
:10061000FF4EFE87ED874082518262827382C30162
:10062000B20120918B0230918C0240918D02509149
:100630008E020E9460D64B015C01F601E751FF4E2D
:10064000608371838283938360918F0270919002A3
:10065000809191029091920220ED3CEC4CE45DE39C
:100660000E9460D67B018C01F601E351FF4E698543
:100670007A858B859C8520813181428153810E94BE
:10068000A6D29B01AC01C801B7010E9460D67B01D4
:100690008C01E1EFF0E1CE0EDF1ED6016D917D9170
:1006A0008D919C9123E333E343E75FE30E9460D69F
:1006B0009B01AC01C801B7010E94A7D27B018C014C
:1006C000F601608371838283938369817A818B8150
:1006D0009C81A50194010E94A7D2A80197010E94C4
:1006E000A6D27B018C0120E030E04FE753E40E946A
:1006F0008ED5181634F56D817E818F81988520E026
:1007000030E040E050E00E948ED518167CF4C30122
:10071000B2012D813E814F8158850E94A6D2AD85C0
:10072000BE856D937D938D939C9313970F2EF0E070
:10073000EF2EF0E0FF2EFFE70F2FF3E41F2FF02D39
:100740002EC0C801B70120E030E040E050E00E9438
:1007500080D3882324F56D817E818F81988520E068
:1007600030E040E050E00E9480D387FF0EC0C3011C
:10077000B2012D813E814F8158850E94A6D2ED8520
:10078000FE8560837183828393830F2EF0E0EF2ECA
:10079000F0E0FF2EF0E00F2FF0E01F2FF02D220CE5
:1007A000331C220C331C8DEE90E1280E391E8985F6
:1007B0009A85AB85BC85F10180839183A283B38345
:1007C000B701C8012E960FB6F894DEBF0FBECDBF9D
:1007D000CF91DF911F910F91FF90EF90DF90CF901D
:1007E000BF90AF909F908F907F906F905F904F9051
:1007F0003F902F9008952F923F924F925F926F9269
:100800007F928F929F92AF92BF92CF92DF92EF92A0
:10081000FF920F931F93CF93DF93EC0121E030E021
:10082000A901440F551F440F551FFA01E35AFA4E10
:1008300085919491C817D9070CF059C0B90161503E
:100840007040660F771F660F771FCB01815A9A4E53
:10085000FC0105911491635A7A4EFB01C590D49026
:10086000FA01E15AFA4EE590F490FA01E35AFA4E91
:10087000A590B490B801882777FD8095982F0E94A5
:1008800022D41B012C01CC19DD09BE01882777FD7C
:100890008095982F0E9422D43B014C01E01AF10A66
:1008A0000027F7FC0095102FC801B7010E9422D441
:1008B0009B01AC01C401B3010E9460D67B018C0195
:1008C000AC18BD08CC24B7FCC094DC2CC601B50123
:1008D0000E9422D49B01AC01C801B7010E9487D3BA
:1008E0009B01AC01C201B1010E94A7D219C0822FA5
:1008F0008F5F2F5F3F4F2D33310509F091CF8D333F
:1009000029F0E0E070E080E060E00CC0EFE4F6E1A8
:1009100065917491882777FD8095982F0E9422D445
:10092000E62F692F2E2F372F482F562FB901CA01D6
:10093000DF91CF911F910F91FF90EF90DF90CF90BB
:10094000BF90AF909F908F907F906F905F904F90EF
:100950003F902F9008952CE933E549E45EE30E942F
:1009600060D608952CE933E549E45EE30E9487D31D
:1009700008952CE933E549E45EE30E9487D30895A6
:100980002CE933E549E45EE30E9460D608952F9296
:100990003F924F925F926F927F928F929F92AF920F
:1009A000BF92CF92DF92EF92FF920F931F93DF934C
:1009B000CF930F92CDB7DEB74C01662389F1E7E400
:1009C000F5E007C08091C00085FFFCCF9093C60082
:1009D000319694919923B1F782E294E070E04AE075
:1009E00050E00E940630E0E4F5E107C08091C000CD
:1009F00085FFFCCF9093C600319694919923B1F76F
:100A00008091C00085FFFCCF8AE08093C60087E319
:100A100095E10E940934E0E070E080E060E08AC087
:100A200021E030E06FC0A901F901EE0FFF1FEE0FCA
:100A3000FF1FE35AFA4E859194912F5F3F4F88161E
:100A400099060CF05FC09A0121503040220F331FED
:100A5000220F331FC901815A9A4EFC01059114914E
:100A6000235A3A4EF901C590D490440F551F440FB4
:100A7000551FFA01E15AFA4EE590F490FA01E35A53
:100A8000FA4EA590B490B801882777FD8095982FED
:100A90000E9422D41B012C018C189D08B4018827C8
:100AA00077FD8095982F0E9422D43B014C01E01ADB
:100AB000F10A0027F7FC0095102FC801B7010E942A
:100AC00022D49B01AC01C401B3010E9460D67B011A
:100AD0008C01AC18BD08CC24B7FCC094DC2CC6013A
:100AE000B5010E9422D49B01AC01C801B7010E944C
:100AF00087D39B01AC01C201B1010E94A7D2E62FAE
:100B0000692F09C029832D33310509F08CCFE0E02E
:100B100070E080E060E0F981FD3361F4EFE4F6E13C
:100B200065917491882777FD8095982F0E9422D433
:100B3000E62F692F2E2F372F482F562FB901CA01C4
:100B40000F90CF91DF911F910F91FF90EF90DF9069
:100B5000CF90BF90AF909F908F907F906F905F905D
:100B60004F903F902F90089580916510909166105E
:100B700060E00E94C78460936D1070936E10809344
:100B80006F109093701080917D1090917E100E9454
:100B9000FB8360937F1070938010809381109093FB
:100BA00082108FB7F89410929F108FBF0895CF9244
:100BB000DF92EF92FF920F931F93CF93DF93EC019D
:100BC000A82FB0E0FD01EE0FFF1FEE0FFF1FE3594E
:100BD000FF4EC080D180E280F380AA0FBB1FA55AD0
:100BE000BF4E6D917C91882777FD8095982F0E944C
:100BF00022D420E030E040E051E40E94A6D29B01E4
:100C0000AC01C701B6010E9480D38E01000F111FF5
:100C1000000F111F8823F4F4CC0FDD1FCC57DF4EDB
:100C2000C701B60120E030E040E850E40E94A7D2BE
:100C30000E94EFD3798368830E9458D00A571F4ED1
:100C40006058714C8F4F9F4FF8016083718382838E
:100C5000938307C00A571F4EF80110821182128237
:100C60001382DF91CF911F910F91FF90EF90DF9052
:100C7000CF90089510925C1010925B1080E090E08D
:100C80000E94D78510925C1010925B1010928A100F
:100C90005D981092641010926310109283105C980B
:100CA0000895CF93DF93DC019B01EA01809132022A
:100CB000882309F449C0E7E4F5E007C08091C0004B
:100CC00085FFFCCF9093C600319694919923B1F79C
:100CD00008C08091C00085FFFCCF9093C6002F5FB5
:100CE0003F4FF90194919923A1F7E9EFF4E107C08F
:100CF0008091C00085FFFCCF9093C60031969491FF
:100D00009923B1F7B7FF03C0E5EFF4E113C082E226
:100D100094E0BD014AE050E00E9406308091C0009E
:100D200085FFFCCF0EC08091C00085FFFCCF909363
:100D3000C600319694919923B1F78091C00085FF48
:100D4000FCCF8AE08093C6008091A710882349F4E5
:100D50001092320281E08093A710CE010E940934E4
:100D600002C00E943A86DF91CF91089590E06CE72F
:100D700076E14FE656E10E945186089590E06BE9D6
:100D800076E14EE856E10E94518608951F920F9237
:100D90000FB60F920BB60F9211242F933F934F93E0
:100DA0005F936F937F938F939F93AF93BF93EF93D3
:100DB000FF9390919B02992391F480918A108093E4
:100DC000A510882311F05D9A01C05D988091831071
:100DD0008093A410882311F05C9A01C05C988091E4
:100DE000A510891708F45D988091A410891708F45C
:100DF0005C989F5F9F7790939B0280919C0290915B
:100E00009D028630910509F497C087309105ACF4B6
:100E10008230910509F45CC08330910534F4009769
:100E200039F1019709F0ABC032C08430910509F463
:100E30007BC005970CF07DC05AC08930910509F43C
:100E400088C08A30910544F48730910509F479C04F
:100E5000089709F094C078C08B30910509F481C0DF
:100E60008B3091050CF478C00C9709F088C083C0D2
:100E700010927B0087E480937C0080917A008064EC
:100E800080937A000E94259681E090E01CC08091BA
:100E9000780090917900A0E0B0E020918B10309123
:100EA0008C1040918D1050918E10820F931FA41FB3
:100EB000B51F80938B1090938C10A0938D10B093DE
:100EC0008E1082E090E090939D0280939C0257C028
:100ED00010927B0086E480937C0080917A0080648D
:100EE00080937A000E94259683E090E0ECCF809179
:100EF000780090917900A0E0B0E020919B103091B3
:100F00009C1040919D1050919E10280F391F4A1F30
:100F10005B1F20939B1030939C1040939D10509327
:100F20009E1084E090E0CFCF0E94259685E090E06F
:100F3000CACF86E090E0C7CF0E94259687E090E078
:100F4000C2CF88E090E0BFCF0E94259689E090E074
:100F5000BACF8AE090E0B7CF0E9425968BE090E070
:100F6000B2CF10929D0210929C028091A6108F5FCA
:100F70008093A61004C010929D0210929C02809152
:100F8000A610803108F483C080919F10882399F4C3
:100F900080918B1090918C109093661080936510C7
:100FA00080919B1090919C1090937E1080937D1067
:100FB00081E080939F101092A61010928B101092D7
:100FC0008C1010928D1010928E1010928F10109223
:100FD0009010109291101092921010929310109203
:100FE00094101092951010929610109297101092E3
:100FF00098101092991010929A1010929B101092C3
:101000009C1010929D1010929E10209165103091AE
:1010100066108091A0109091A110821793071CF088
:1010200080E00E94BE8620919702309198028091C4
:10103000651090916610821793071CF080E00E9463
:10104000B68620917D1030917E108091A2109091F3
:10105000A3108217930744F08FEF9FEF63EE74E1C4
:1010600042ED54E10E9451862091990230919A02FA
:1010700080917D1090917E108217930744F08FEF3E
:101080009FEF60EC74E14FEA54E10E945186FF91BA
:10109000EF91BF91AF919F918F917F916F915F91F0
:1010A0004F913F912F910F900BBE0F900FBE0F905D
:1010B0001F9018952F923F924F925F926F927F925E
:1010C0008F929F92AF92BF92CF92DF92EF92FF9258
:1010D0000F931F93DF93CF93CDB7DEB728970FB64B
:1010E000F894DEBF0FBECDBF9A8389837C836B8368
:1010F0002D833E834F835887270138011601D7FE81
:1011000003C021E0C22ED12CF601EE0FFF1FEE0F1F
:10111000FF1FE855FF4EE080F18002811381C80176
:10112000B701A30192010E9480D3882321F0E981B5
:10113000FA8111821082E981FA8180819181823065
:101140009105C1F18330910534F4009759F001976E
:1011500009F086C010C083309105D1F1049709F0E1
:101160007FC077C0EB81FC811082118212821382D2
:1011700081E090E01AC0C301B20120E030E040E01D
:1011800050E00E948ED518160CF06AC0CC0CDD1C05
:10119000CC0CDD1C88EA90E1C80ED91EF601408215
:1011A00051826282738282E090E0E981FA819183C8
:1011B000808356C06D817E818F819885A8019701BB
:1011C0000E948ED588230CF44BC083E090E0EDCFD5
:1011D000B401882777FD8095982F0E9422D49B0127
:1011E000AC01C801B7010E94A6D29B01AC016D8180
:1011F0007E818F8198850E948ED588234CF00E9435
:1012000058D0EB81FC81608371838283938328C0F3
:101210000E9458D07B018C01B501882777FD80950D
:10122000982F28EE33E040E050E00E9432D7EB8167
:10123000FC812081318142815381260F371F481F55
:10124000591F2E153F054007510750F484E090E0E8
:10125000ACCFC10167E275E147E155E10E945186DB
:1012600028960FB6F894DEBF0FBECDBFCF91DF91A9
:101270001F910F91FF90EF90DF90CF90BF90AF90B4
:101280009F908F907F906F905F904F903F902F90A6
:1012900008954F925F926F927F928F929F92AF923A
:1012A000BF92CF92DF92EF92FF920F931F938091A4
:1012B0009F10882309F410C10E94B4850E9458D061
:1012C0002B013C01A0906D10B0906E10C0906F107B
:1012D000D090701060915B1070915C10882777FD42
:1012E0008095982F0E9422D47B018C018AEB90E19B
:1012F00062EC70E1A6019501CC24DD24E8E2AE2E7B
:10130000B12CB4E08B2E912C0E945A8880E090E0A2
:101310000E9431825B016C01E0906D10F0906E10C4
:1013200000916F10109170106091B8107091B91009
:10133000882777FD8095982F0E9422D49B01AC01CD
:10134000C801B7010E948ED51816CCF460919E0298
:1013500070919F02882777FD8095982F0E9422D454
:101360009B01AC01C801B7010E9480D388233CF4E3
:10137000C601B5010E94EFD37595679501C060E085
:1013800060938A108091861090918710A0918810A8
:10139000B09189100097A105B10521F1841595053B
:1013A000A605B705F8F46091841070918510882720
:1013B00077FD8095982F0E9422D49B01AC01C80133
:1013C000B7010E9480D388234CF480E090E060E66F
:1013D00076E141E556E10E94518604C080E090E04C
:1013E0000E94D7858091D2109091D310A091D410F3
:1013F000B091D510481659066A067B0608F46CC0F1
:1014000088E893E1A0E0B0E0480E591E6A1E7B1EFA
:101410004092D2105092D3106092D4107092D51096
:10142000A0907F10B0908010C0908110D09082105A
:101430006091631070916410882777FD8095982FD4
:101440000E9422D47B018C0186ED90E168ED70E171
:10145000A6019501CC24CA94DC2CF4E1AF2EB12C6A
:10146000E2E08E2E912C0E945A88E0907F10F0903E
:1014700080100091811010918210C801B70120E006
:1014800030E040EA50E40E948ED5181614F5C801E9
:10149000B70120E030E046E153E40E9480D3882386
:1014A000C4F46091631070916410882777FD809573
:1014B000982F0E9422D49B01AC01C801B7010E9461
:1014C00080D387FD02C080E001C08FE78093831046
:1014D00003C0109283105C981F910F91FF90EF90C2
:1014E000DF90CF90BF90AF909F908F907F906F9044
:1014F0005F904F9008950F931F93CF93DF9380E0F9
:1015000090E0A0E0B0E08093B0109093B110A09371
:10151000B210B093B31060E070E08FE793E42091D5
:101520008B0230918C0240918D0250918E020E946C
:1015300087D36093B4107093B5108093B6109093D6
:10154000B710559A549A249A87ED80937A00109296
:101550007E0080917E00806880937E0080917E0076
:10156000806480937E0080E888BD80916E008460F6
:1015700080936E006AEF70E080E090E00E9466D099
:1015800085E090E09093B9108093B81009C08091E5
:1015900097029091980240979093980280939702B7
:1015A000809197029091980260E00E94C78420E0A9
:1015B00030E040EA50E40E9480D387FDE8CF83E129
:1015C00091E090939F0280939E0209C08091A010A9
:1015D0009091A11040969093A1108093A0108091BB
:1015E000A0109091A11060E00E94C78420E030E834
:1015F00049E853E40E948ED5181644F3C09199022D
:10160000D0919A021C2F0D2FCE010E94FB83609770
:1016100020E030E040EA50E40E9480D387FDF2CF22
:101620001093990200939A02C091A210D091A31036
:101630001C2F0D2FCE010E94FB83609620E030E02E
:1016400046E153E40E948ED5181694F31093A2102D
:101650000093A310DF91CF911F910F9108952F92C6
:101660003F924F925F926F927F928F929F92AF9232
:10167000BF92CF92DF92EF92FF920F931F93DF936F
:10168000CF93CDB7DEB7E4970FB6F894DEBF0FBEA9
:10169000CDBF68A379A38AA39BA35CAB4BAB3DA34F
:1016A0002CA30E9458D06D8B7E8B8F8B988F2BA98B
:1016B0003CA9121613061CF0EDECF1E019C0E0EEA7
:1016C000F1E007C08091C00085FFFCCF3196909378
:1016D000C60090819923B1F78091C00085FFFCCFAF
:1016E0007DC48091C00085FFFCCF31969093C600E9
:1016F00090819923B1F78091C00085FFFCCF8AE0EB
:101700008093C6000E943A864BA95CA9452BA9F19B
:101710008FE7809383108D899E89AF89B88D898BDF
:101720009A8BAB8BBC8B7C018D011FA618AA19AAC2
:101730001AAA1B8E1A8E91E0998F1D861E861F860F
:10174000188A4FE7642E712C812C912C69867A8639
:101750008B869C8620E030E040E050E029833A838D
:101760004B835C830F2EF0E02F2EF0E43F2EFCE144
:101770004F2EF6E45F2EF02D04C08FE780938A1081
:10178000CACF0E9458D05B016C0180919F108823C2
:1017900009F4ABC20E94B4854BA95CA9452B69F042
:1017A00050917F105FA78091801088AB909181103D
:1017B00099ABA0918210AAAB0CC0B0916D10BFA7DD
:1017C000E0916E10E8ABF0916F10F9AB20917010C2
:1017D0002AAB69817A818B819C812FA538A949A97F
:1017E0005AA90E948ED5181644F08FA598A9A9A9C8
:1017F000BAA989839A83AB83BC83C201B1012FA5A7
:1018000038A949A95AA90E9480D387FD06C08FA58F
:1018100098A9A9A9BAA91C012D01398D332309F46E
:101820004AC06FA578A989A99AA928A139A14AA176
:101830005BA10E948ED518160CF057C2D801C701C3
:1018400088579C4EAF4FBF4F8A159B05AC05BD0511
:1018500008F04BC2D401C30129853A854B855C85CC
:10186000821B930BA40BB50B4BA95CA9452B39F03C
:10187000B595A795979587958093831006C0B595E4
:10188000A7959795879580938A10D601C5018E19E3
:101890009F09A00BB10B8D879E87AF87B88BA98A54
:1018A000BA8ACB8ADC8A28A139A14AA15BA1298303
:1018B0003A834B835C836FA578A989A99AA928A14B
:1018C00039A14AA15BA10E9480D388230CF00CC2ED
:1018D00089899A89AB89BC8988579C4EAF4FBF4F85
:1018E0008A159B05AC05BD0508F0FEC14A8D5B8DD0
:1018F000452B09F4D1C1D601C50129893A894B8903
:101900005C89821B930BA40BB50B2D853E854F85FF
:101910005889280F391F4A1F5B1F2C8F3D8F4E8F10
:101920005F8F2D853E854F855889281B390B4A0BC3
:101930005B0BCA01B90129853A854B855C850E94FC
:1019400032D72C8D3D8D4E8D5F8D0E949AD7620EC1
:10195000731E841E951E34E1631671048104910484
:1019600074F484E190E0A0E0B0E089879A87AB87C7
:10197000BC8794E1692E712C812C912C23C09CEEA4
:10198000691671048104910434F08BEE682E712C79
:10199000812C912C0BC0A0E86A167104810491047B
:1019A0002CF469867A868B869C860CC02EEF30E0FC
:1019B00040E050E0261937094809590929873A8734
:1019C0004B875C87E1EEF7E107C08091C00085FF9F
:1019D000FCCF9093C600319694919923B1F782E29F
:1019E00094E0B401A3012AE030E00E94D12FECED95
:1019F000F7E107C08091C00085FFFCCF9093C6003F
:101A0000319694919923B1F782E294E049855A8501
:101A10006B857C852AE030E00E94D12FE5EDF7E16F
:101A200007C08091C00085FFFCCF9093C60031961F
:101A300094919923B1F782E294E0B201A10122E0EE
:101A400030E00E94D930EEECF7E107C08091C00091
:101A500085FFFCCF9093C600319694919923B1F7FE
:101A600082E294E049815A816B817C8122E030E0FE
:101A70000E94D9308091C00085FFFCCF3AE03093BE
:101A8000C6004A8D5B8D433051050CF405C1698554
:101A90007A858B859C850E9422D420E030E040E846
:101AA00050E40E9460D67B018C0169817A818B8130
:101AB0009C81A20191010E94A6D22BED3FE049E456
:101AC00050E40E9460D620E030E040E05FE30E94F6
:101AD00060D69B01AC01C801B7010E9487D31B01EE
:101AE0002C016C8D7D8D8E8D9F8D0E9422D420E0E7
:101AF00030E04AE754E40E9487D37B018C01E8EC94
:101B0000F7E107C08091C00085FFFCCF9093C6002D
:101B1000319694919923B1F782E294E0B201A10148
:101B200022E030E00E94D930E2ECF7E107C080917A
:101B3000C00085FFFCCF9093C60031969491992305
:101B4000B1F782E294E0B801A70122E030E00E9400
:101B5000D9308091C00085FFFCCF5AE05093C60079
:101B6000C201B1012AE939E949E15FE30E9460D687
:101B70006D837E838F8398879B01AC010E94A7D2DF
:101B8000A80197010E9487D36BA77CA78DA79EA76A
:101B90006D817E818F819885A80197010E9460D612
:101BA00020E030E040E05EE30E9460D66FA378A7BB
:101BB00089A79AA7E4EBF7E107C08091C00085FFF1
:101BC000FCCF9093C600319694919923B1F7809100
:101BD000C00085FFFCCF8AE08093C600EEEAF7E103
:101BE00007C08091C00085FFFCCF9093C60031965E
:101BF00094919923B1F782E294E04D815E816F81E7
:101C0000788522E030E00E94D9308091C00085FFC5
